:100000000C94A3070C94C2070C94C2070C94C2076B
:100010000C94C2070C94C2070C94CD090C94030AEB
:100020000C94C2070C94C2070C94C2070C94C2072C
:100030000C94C2070C94C2070C94C2070C94700D68
:100040000C94C2070C94C2070C94C2070C94C2070C
:100050000C9428510C944A480C94C2070C94C20783
:100060000C94C2070C941F490C94C2070C941349BA
:100070000C94C2070C94C2070C94C2070C94C207DC
:100080000C94A05C0C94C2070C94C2070C94C20799
:100090000C945D490C94C2070C9451490C94C2070E
:1000A0000C94C2070C94C2070C94C2070C94C207AC
:1000B0000C94C2070C94C2070C94C2070C94C2079C
:1000C0000C94C2070C94C2070C94C2070C94C2078C
:1000D0000C94C2070C94C2070C94C2070C94C2077C
:1000E0000C94C2070C94E1500C94EB500C94D75034
:1000F0000C9491500C941C510C940D510C94015182
:100100000C94F5500C94C2070C94C2070C94C207CF
:100110000C94C2070C94C2070C94C2070C94C2073B
:1001200007634236B79BD8A71A39685618AEBAABE0
:10013000558C1D3CB7CC5763BD6DEDFD753EF61774
:100140007231BF000000803F08000000BE922449C9
:10015000123EABAAAA2ABECDCCCC4C3E00000080F9
:10016000BEABAAAAAA3E00000000BF000000803F6C
:100170000000000000084178D3BB4387D1133D192C
:100180000E3CC3BD4282AD2B3E68EC8276BED98F59
:10019000E1A93E4C80EFFFBE01C4FF7F3F0000009D
:1001A00000000A0025303278002025362E326620E5
:1001B0004F6E2D426F61726400202573002530322E
:1001C00078002025362E326620002025730048490D
:1001D00048363133302000424D5030383520004110
:1001E00044584C3334352000484D4338383533209B
:1001F000004C3347343230304420004E48444330C2
:100200003231362000756E6B6E6F776E20636D64D1
:100210000A002563006820202020202020202020A4
:1002200020202020202020202020202020202020CE
:10023000202D2068656C700A0D007620202020207B
:1002400020202020202020202020202020202020AE
:100250002020202020202D2076657273696F6E0A81
:100260000D0075202020202020202020202020206C
:1002700020202020202020202020202020202D2071
:10028000757074696D650A0D00616573205B6F6E32
:100290007C6F66665D2020202020202020202020EA
:1002A00020202020202D20696E7465677265747986
:1002B0000A0D0061646320202020202020202020BF
:1002C0002020202020202020202020202020202D21
:1002D0002073686F7720765F696E2C2061312C2047
:1002E000613220766F6C74616765730A0D0063611B
:1002F0006C69205B5B765F696E7C61317C61325D2D
:1003000020766F6C746167655D202D2063616C6978
:1003100062726174650A0D006465205B6D61736BC8
:100320005D20202020202020202020202020202090
:10033000202020202D2064656275670A0D006875F5
:100340006D20202020202020202020202020202060
:10035000202020202020202020202D2068756D695D
:10036000646974792073656E736F720A0D00687525
:100370006D70205B6F6E7C6F66665D202020202094
:10038000202020202020202020202D2068756D692D
:1003900064697479207065726D2073656E736F7215
:1003A000207077720A0D006964205B726573657452
:1003B0005D20202020202020202020202020202000
:1003C0002020202D2069642068616E646C696E674E
:1003D0000A0D006D63752020202020202020202081
:1003E0002020202020202020202020202020202D00
:1003F000206D637520696E666F0A0D006E65205B67
:10040000666C7573685D202020202020202020202D
:1004100020202020202020202D206E656967686222
:100420006F72207461626C650A0D006C6F67205BEF
:100430006175746F7C6F6E7C6F66665D2020202016
:10044000202020202020202D206D6F7465732064D3
:10045000617461206F6E205553420A0D006F772042
:10046000202020202020202020202020202020208C
:100470002020202020202020202D206F6E652D7729
:100480006972652073656E736F72730A0D00726511
:10049000205B6D61736B5D202020202020202020B8
:1004A000202020202020202020202D206D6F74650A
:1004B000207265706F72742073657474696E670A58
:1004C0000D007269205B696E745D20202020202061
:1004D00020202020202020202020202020202D200F
:1004E0007265706F727420696E74657276616C0AE1
:1004F0000D0072732020202020202020202020208A
:1005000020202020202020202020202020202D20DE
:10051000726164696F2073746174730A0D00737380
:1005200020202020202020202020202020202020CB
:10053000202020202020202020202D20737973745B
:10054000656D2073756D6D6172790A0D007077723B
:1005500031205B6F6E7C6F66665D2020202020203E
:100560002020202020202020202D2070696E312086
:100570007077720A0D007265737420656570726F12
:100580006D2020202020202020202020202020201E
:1005900020202D20726573746F72652065657072FE
:1005A0006F6D0A0D0070777273205B646565707CF7
:1005B000666F7263655F69646C655D202020202032
:1005C000202D206D637520736C656570206D6F64E0
:1005D000650A0D00626F6F742020202020202020EB
:1005E000202020202020202020202020202020200B
:1005F0002D207265626F6F740A0D0075706772202E
:1006000020202020202020202020202020202020EA
:10061000202020202020202D207265626F6F742002
:1006200076696120626F6F746C6F616465720A0D28
:100630000074657374205B6F66667C317C327C333A
:100640005D2020202020202020202020202D20740C
:10065000657374206D6F6465730A0D00557074695D
:100660006D6520256420646179732C202530326407
:100670003A253032643A253032640A00204E6576DD
:1006800065722D7573656420737461636B203E2001
:1006900025642062797465730A0025352E32662040
:1006A0000025372E33662025372E3366002530325D
:1006B0007800525F49442000525F542000525F543A
:1006C000312000525F545F4D43552000525F565F0A
:1006D0004D43552000525F50302000525F50305F34
:1006E000542000525F50312000525F50315F54203F
:1006F00000525F555054494D452000525F524820EA
:1007000000525F565F494E2000525F413120005237
:100710005F41322000525F502000525F5041200064
:10072000525F49443D09093078257800525F543DB5
:1007300009093078257800525F54313D0909307835
:10074000257800525F545F4D43553D093078257838
:1007500000525F565F4D43553D0930782578005271
:100760005F50303D09093078257800525F50305F86
:10077000543D09093078257800525F50313D090910
:100780003078257800525F50315F543D0909307848
:10079000257800525F555054494D453D0930782524
:1007A0007800525F52483D09093078257800525F41
:1007B000565F494E3D09093078257800525F413136
:1007C0003D09093078257800525F41323D090930F2
:1007D00078257800525F503D09093078257800521D
:1007E0005F50413D0909307825780025730A004E95
:1007F00065772064656275673D307825580A004347
:10080000757272656E742064656275673D30782517
:10081000580A00445F4F5045523D307825780A0011
:10082000445F52583D307825780A00445F54583D63
:10083000307825780A00445F504B543D6E3078255F
:10084000780A00445F4F573D307825780A00445FAE
:100850004C45443D307825780A00445F504F574559
:10086000523D307825780A00445F4556454E543D48
:10087000307825780A00445F50305F4C45443D3065
:100880007825780A00445F50315F4C45443D30780C
:1008900025780A00445F4145533D307825780A00A9
:1008A000445F5057525F313D307825780A00445FED
:1008B000505245533D307825780A00445F41434308
:1008C000454C3D307825780A00445F434F4D5041F8
:1008D00053533D307825780A0025630025630025B1
:1008E00063004F4B0A002563007478206C656E200E
:1008F000202020207268206D6973732020202072D0
:1009000068207374616C652020207268206D6973A3
:10091000630A00252D31306C7520252D31306C7522
:1009200020252D31306C7520252D31306C75200A35
:10093000002563004D43553D2530366C7800204638
:100940007573653A2065653D253032782068663DCF
:1009500025303278206C663D25303278206C623D3F
:100960002530327800204F534343414C3D256420CD
:10097000002563002563002563002563004E65772D
:10098000207265706F72743D307825582000557361
:10099000696E67207265706F72743D3078255820DB
:1009A000002563004E6577207265706F7274206950
:1009B0006E74657276616C3D252D64207365630AE3
:1009C0000043757272656E74207265706F72742068
:1009D000696E74657276616C3D252D642073656364
:1009E0000A0025630025630053797374656D2053F5
:1009F000756D6D6172790A0049443D004932433A90
:100A000020004E65696768626F72207461626C6570
:100A10002073697A653D25640A0052494D4520617D
:100A20006464723D252D642E252D640A0052657084
:100A30006F727420496E74657276616C3D252D6409
:100A40000A005265706F7274204D61736B3D30788F
:100A5000252D782000565F494E3D252D352E3266D6
:100A60000A00565F4D43553D252D352E32660A004E
:100A70005553425F5057523D25730A00496E7472B8
:100A80002E20546F74616C3A2050303D252D6C64DB
:100A90002050313D252D6C640A00496E74722E2061
:100AA0005365633A20202050303D252D372E336684
:100AB0002050313D252D372E33660A004C6F6720BC
:100AC0006D6F64653D006175746F0A0025730A00DF
:100AD00048554D5F5057525F414C574159533D2542
:100AE000730A00496E7075742050313D25730A00F9
:100AF00044656275673D3078252D780A005077721D
:100B0000313D25730A0025630025630052483D25C9
:100B10002D342E31662000545F52483D252D342E51
:100B200031662000256300256C6420432000256C7D
:100B3000642050612020252D372E3266206D00253F
:100B400063005854414C5F5452494D3D2564004563
:100B500072726F72203020566F6C74004572726F23
:100B600072203020566F6C74004572726F722030A4
:100B700020566F6C740025352E3266200025372EE6
:100B800033662025372E33660025730A00546573BB
:100B90007420312025730A00546573742032202597
:100BA000730A005465737420332025730A0054655A
:100BB000737420342025730A0025730A0025730AF4
:100BC0000025730A0025730A002563002563005081
:100BD0003A20256C642050612020252D372E326666
:100BE000206D0A00532025642E256420636C6F63FA
:100BF0006B20256C7520747820256C752072782008
:100C0000256C752072747820256C7520727278209E
:100C1000256C75207265786D697420256C7520616E
:100C2000636B747820256C75206E6F61636B7478CC
:100C300020256C752061636B727820256C7520749B
:100C4000696D65646F757420256C752062616461DF
:100C5000636B727820256C7520746F6F6C6F6E6794
:100C600020256C7520746F6F73686F727420256C0B
:100C7000752062616473796E636820256C752062EB
:100C8000616463726320256C7520636F6E74656E9A
:100C900074696F6E64726F7020256C752073656E59
:100CA00064696E6764726F7020256C75206C6C745B
:100CB0007820256C75206C6C727820256C750A0084
:100CC000452025642E256420636C6F636B20256CA2
:100CD000752063707520256C75206C706D20256CF7
:100CE000752069727120256C7520676C65642025FC
:100CF0006C7520796C656420256C7520726C656458
:100D000020256C7520747820256C75206C697374AF
:100D1000656E20256C752073656E736F7273202568
:100D20006C752073657269616C20256C750A000A08
:100D30002A2A2A2A2A2A2A426F6F74696E67202576
:100D4000732A2A2A2A2A2A2A0A0052616E646F6D9F
:100D50002045554936342061646472657373206799
:100D6000656E6572617465640A004D41432061647B
:100D70006472657373200025783A000A0025732099
:100D800025732C206368616E6E656C20257520705C
:100D90006F776572202575002C20636865636B2072
:100DA0007261746520257520487A000A004F6E6CC8
:100DB000696E650A00257325730A006C6F63616CA8
:100DC000686F73740041544D454741313238726643
:100DD000613100020000FFFE000001454550524F06
:100DE0004D20697320636F72727570742C20726568
:100DF00077726974696E67207769746820646566C4
:100E000061756C74732E0A006E616E00696E660007
:100E100000407A10F35A00A0724E18090010A5D4B1
:100E2000E80000E87648170000E40B54020000CA0E
:100E30009A3B000000E1F505000080969800000054
:100E400040420F000000A0860100000010270000B3
:100E50000000E803000000006400000000000A0039
:100E6000000000000100000000002C76D888DC673C
:100E70004F0823DFC1DFAE59E1B1B796E5E3E45394
:100E8000C63AE651997696E8E6C28426EB898C9BB1
:100E900062ED407C6FFCEFBC9C9F40F2BAA56FA551
:100EA000F490055A2AF75C936B6CF9676DC11BFCD3
:100EB000E0E40D47FEF520E6B500D0ED902E0300EE
:100EC000943577050080841E080000204E0A00003B
:100ED00000C80C333333330F986E12831141EF8DFA
:100EE0002114893BE65516CFFEE6DB18D1844B383A
:100EF0001BF77C1D901DA4BBE424203284725E226B
:100F00008100C9F124ECA1E53D27494E46494E49EF
:100F100054594E414E000020410000C84200401C80
:100F20004620BCBE4CCA1B0E5AAEC59D74CDCCCC5F
:100F30003D0AD7233C17B7D13877CC2B329595E6AD
:100F4000241FB14F0A0011241FBECFEFD1E4DEBF32
:100F5000CDBF16E0A0E0B2E0EEE2F0EF00E00BBFA4
:100F600002C007900D92AC38B107D9F71DE2ACE88A
:100F7000B6E001C01D92A633B107E1F70E94C8692F
:100F80000C9415780C940000E0915B17F0E0EF7181
:100F9000F070E055F84E808380915B178F5F8093EF
:100FA0005B17809170248860809370244EEB54E02E
:100FB000CA0161E10E94FE3880E090E008954F92FE
:100FC0005F926F927F928F929F92AF92BF92CF92D9
:100FD000DF92EF92FF920F931F93CF93DF93CDB7E2
:100FE000DEB760970FB6F894DEBF0FBECDBF4B01E2
:100FF000809192069091930681FD74980E948A3F99
:101000003C0188E996E00E94FA390AC0C8010296BC
:10101000B4010E94D5360097F1F4C8010E94A03AAD
:101020008C01009799F725C1C8010296B4010E946E
:10103000CC36D3018C918150F801808780E091E01B
:10104000A0E0B0E081879287A387B48788E996E023
:10105000B8010E94693AC8010D9660E074E649E55E
:1010600059E098010E948B3C84E00E94AE40D80178
:1010700015969C938E93149783E00E94AE402C01AA
:10108000F80197838683D301CC908085C81ADD242C
:10109000EE24FF2486E0CC0CDD1CEE1CFF1C8A95A0
:1010A000D1F7618572858385948520EC30E040E03E
:1010B00050E00E941571DC01CB01892F9A2FAB2FD4
:1010C000BB27C80ED91EEA1EFB1EF801C186D286B8
:1010D000E386F486D3018C9180878091920690916B
:1010E000930681FD08C08091DE0480FD04C081FF6D
:1010F000B8C01D9BB6C0EDB7FEB772970FB6F89497
:10110000FEBF0FBEEDBFADB6BEB60894A11CB11CAC
:1011100080E092E092838183C3010196D50113960A
:101120009C938E931297F401808114968C9314975C
:1011300015961C921597818116968C931697179683
:101140001C92D3018C91F50180871186D8011496E9
:101150008D919C9115979387828755864486BB27EE
:10116000AF2D9E2D8D2D97878687C701B60124E66A
:1011700030E040E050E00E941571672F782F892FF2
:1011800099270E945B71DC01CB01F501918B808B6B
:101190000E9406752091FA048DB79EB742960FB64D
:1011A000F8949EBF0FBE8DBF2223A9F000D000D0BF
:1011B000EDB7FEB731968CEC9BE0ADB7BEB712969B
:1011C0009C938E931197228313820E9418750F901F
:1011D0000F900F900F908091F91B85FF42C00E94E5
:1011E0003345C30104960E94F444EDB7FEB73C9723
:1011F0000FB6F894FEBF0FBEEDBF31966E01089496
:10120000C11CD11CADB7BEB71296DC92CE9211971D
:1012100080E190E0938382838CE392E095838483E2
:10122000D80114968D919C91159797838683169675
:101230008D919C91179791878087D3018C9182879C
:1012400013860E946D75EDB7FEB73C960FB6F89405
:10125000FEBF0FBEEDBF82E00E940F45C6010E9497
:10126000F444809192069091930681FF0BC0749A8A
:1012700009C08BE095E00E9487398C01009709F046
:10128000D3CEEFCF60960FB6F894DEBF0FBECDBFC2
:10129000DF91CF911F910F91FF90EF90DF90CF9052
:1012A000BF90AF909F908F907F906F905F904F9086
:1012B0000895CF93DF93EC0180919206909193066D
:1012C00087FF2EC08DB79EB70C970FB6F8949EBFC0
:1012D0000FBE8DBFEDB7FEB731968FE492E0ADB78C
:1012E000BEB712969C938E9311978A818283138244
:1012F0008B81848315828885868317828C819D816A
:10130000918780878E819F81938782870E9406754F
:101310008DB79EB70C960FB6F8949EBF0FBE8DBFCB
:1013200088E996E0BE010E94343A8BE095E0BE0168
:101330000E94B239DF91CF91089587EE93E0811535
:10134000910511F00197F1F70895882369F06D98E0
:101350007598ED9A80916A00886080936A00809108
:1013600068008160809368008091DE049091DF04C2
:1013700091FF10C06E988EB18F6B8EB9EE9A8091EE
:101380006A00806280936A00809168008160809327
:1013900068000895769AEE9808951F920F920FB6FE
:1013A0000F9211248F939F93AF93BF938091680006
:1013B00080FF20C08091502490915124A09152240C
:1013C000B09153240196A11DB11D80935024909398
:1013D0005124A0935224B09353248091920690916B
:1013E000930690FF07C0749882E090E09093080500
:1013F00080930705BF91AF919F918F910F900FBE82
:101400000F901F9018951F920F920FB60F921124F4
:101410008F939F93AF93BF938091680080FF20C00C
:101420008091542490915524A0915624B091572432
:101430000196A11DB11D8093542490935524A0932F
:101440005624B0935724809192069091930691FF71
:1014500007C0739882E090E0909308058093070599
:10146000BF91AF919F918F910F900FBE0F901F90E2
:10147000189580937C0080917B00877F80937B0010
:1014800080917C00806C80937C0085E080937A0062
:1014900080917A00806880937A0080917B0087FF3A
:1014A000FCCF80917B0085FFFCCF80917A00806427
:1014B00080937A0080917A0086FDFCCF10927900AB
:1014C0001092780084E090E060E070E020917A0073
:1014D000206420937A0020917A0026FDFCCF209191
:1014E000780030917900620F731F019779F710929D
:1014F0007C0080917A008F7780937A00769567954B
:101500007695679580E090E00E949B6E462F572F5E
:10151000682F792FCB01BA01089580E00E94390A23
:101520002091030530910405409105055091060571
:101530000E944D6F21EE3AE744E95EE30E94CB6DD5
:10154000462F572F682F792FCB01BA01089580E1DC
:1015500080935101809351019091510195FF03C0F7
:101560008F5F8F31B9F76BE4869FB0011124882714
:1015700077FD8095982F0E949D6E20E030E64FE920
:1015800054E40E94CB6D462F572F682F792FCB0143
:10159000BA0120E030E04AE754E40E94336E462F5F
:1015A000572F682F792FCB01BA0108958091E2045B
:1015B00083FF4DC080917B00886080937B0089EC25
:1015C00080937C0085E080937A0080917A00806827
:1015D00080937A0080917B0087FFFCCF80917B0015
:1015E00085FFFCCF80917A00806480937A0080919F
:1015F0007A0086FDFCCF80917A00806480937A0027
:1016000080917A0086FDFCCF60917800709179001E
:1016100080E090E00E949B6E27ED33EA40E95FE3B3
:101620000E944D6F26E636E648E853E40E94CA6DF4
:10163000DC01CB018093501790935117A093521760
:10164000B093531780917A008F7780937A00089532
:10165000CF92DF92EF92FF921F93CF93DF93CDB79C
:10166000DEB729970FB6F894DEBF0FBECDBF6C0171
:1016700010928C068FEF8983ACE6EA2EA7E1FA2E52
:1016800010E03FC0183009F440C0CE010196BE0101
:101690006E5F7F4F0E94714289818F3F11F08E3FB4
:1016A00019F480938C0631C0CE010296C114D10486
:1016B00079F40E948A4280936D24DE011296E5E659
:1016C000F4E288E09D9191938150E1F711E01DC013
:1016D0000E948A42F7018083DE01129620E030E00A
:1016E000C70108974D91FC01E20FF31F40832F5F64
:1016F0003F4F28303105B1F71F5F89E090E0E80ED9
:10170000F91E8981882309F0BDCF812F29960FB654
:10171000F894DEBF0FBECDBFDF91CF911F91FF9038
:10172000EF90DF90CF90089500D082EA91E0EDB77E
:10173000FEB7928381830E9418750F900F900895D1
:101740002F923F924F925F926F927F928F929F92D1
:10175000AF92BF92CF92DF92EF92FF920F931F93BF
:10176000CF93DF9300D000D0CDB7DEB78C010097C8
:1017700041F489E290E06BE270E04AE250E027E059
:101780000AC08130910549F489E290E06BE270E093
:101790004AE250E026E00E944641C8010E94280B20
:1017A0006DE8862E66E0962E800E911ED4018C93F5
:1017B0000115110599F02CE6A22E27E1B22E00E0CA
:1017C00010E03DEB632E31E0732E42EC442E41E0FD
:1017D000542E5AEC252E51E0352E10C185E694E2A8
:1017E0000E94AD43FC01BF01882777FD8095982FAB
:1017F0000E949D6EF82EE92E05E614E2AA24BB2471
:1018000094EAC92E91E0D92ED8018D918D0100D096
:1018100000D0EDB7FEB73196ADB7BEB71296DC92E9
:10182000CE921197828313826B837C830E941875FA
:101830000894A11CB11C0F900F900F900F906B811A
:101840007C81B8E0AB16B104F9F600D000D000D02E
:101850000DB71EB70F5F1F4F89EA91E0EDB7FEB7D6
:10186000928381839701862F972FA32FBE2DBC01D2
:10187000CD0120E030E048EC52E40E94336EDC0100
:10188000CB01F80182839383A483B5830E941875EA
:101890002DB73EB72A5F3F4F0FB6F8943EBF0FBE3D
:1018A0002DBF80916D24882319F08EE792E002C04D
:1018B00087E892E000D000D029EB31E0ADB7BEB7A9
:1018C00012963C932E93119714969C938E93139794
:1018D0000E9418750F900F900F900F900E94940B1C
:1018E00094C0C801B3E0880F991FBA95E1F7800F43
:1018F000911F8C59984E0E94AD43FC01BF0188276F
:1019000077FD8095982F0E949D6E6C0120E030E05D
:1019100088EFE82E8FEFF82EEA0CFB1C00D000D0E9
:10192000ADB7BEB71196EDB7FEB772826182F7010F
:10193000E20FF31F808112968C93129713961C92DC
:1019400029833A836B837C830E94187529813A81AD
:101950002F5F3F4F0F900F900F900F906B817C8106
:1019600028303105D9F600D000D000D0EDB6FEB653
:101970000894E11CF11CADB7BEB712965C924E9272
:101980001197862F972FAC2DBD2DBC01CD0120E0E6
:1019900030E048EC52E40E94336EDC01CB01F701E9
:1019A00082839383A483B5830E9418752DB73EB7B5
:1019B0002A5F3F4F0FB6F8943EBF0FBE2DBFD50133
:1019C0008C91882319F08EE792E002C087E892E0BC
:1019D00000D000D0EDB7FEB732822182948383839A
:1019E0000E9418750F900F900F900F900E94940B0B
:1019F0000F5F1F4F29E030E0A20EB31ED4018C917F
:101A000090E0081719070CF46CCF0F900F900F900F
:101A10000F90DF91CF911F910F91FF90EF90DF908A
:101A2000CF90BF90AF909F908F907F906F905F907E
:101A30004F903F902F900895CF93DF9300D0CDB774
:101A4000DEB780916624898380916C248A83CE01DD
:101A500001960E94E7360F900F90DF91CF91089585
:101A6000CF93DF93EC01809165248F3FB1F5809196
:101A700066248F3F91F5809167248F3F71F58091A7
:101A800068248F3F51F5809169248F3F31F5809113
:101A90006A248F3F11F580916B248F3FF1F4809180
:101AA0006C248F3FD1F489E290E06BE270E04AE26F
:101AB00050E027E00E94464180E090E00E94280B21
:101AC000C357D94F888385E694E260E070E049E02F
:101AD00050E00E945E760E941C0DDF91CF91089528
:101AE0001F920F920FB60F920BB60F9211242F93E5
:101AF0003F934F935F936F937F938F939F93AF9396
:101B0000BF93EF93FF938091702482608093702441
:101B10008091DE0486FD2B9A87FD2B9A8091070524
:101B2000909108051816190614F4749A739A809106
:101B300092069091930685FF02C0749873988091E5
:101B4000090590910A05019790930A05809309056C
:101B5000009709F068C080919606909197069C01C5
:101B60002F5F3F4F30939706209396064091FB1FBF
:101B70005091FC1F6091FD1F7091FE1F4F5F5F4FE2
:101B80006F4F7F4F4093FB1F5093FC1F6093FD1FCF
:101B90007093FE1F20E130E030930A052093090581
:101BA0002091DE0420FD02C01D9B05C0109290060E
:101BB00010928F0606C021E030E03093900620930B
:101BC0008F062091E0043091E10421153105A1F048
:101BD0000296B9010E943471009771F47798809150
:101BE00092069091930693FF07C0749884E090E06A
:101BF00090930805809307052115310581F08091A8
:101C0000960690919706B9010E943471009739F4B5
:101C100086EA94E062E140E050E00E94FE38809164
:101C2000DE0486FD2B988FE295E060E040E050E016
:101C30000E94FE38FF91EF91BF91AF919F918F91DC
:101C40007F916F915F914F913F912F910F900BBEBC
:101C50000F900FBE0F901F90189580915B17909179
:101C60000F20891B08950E942D0E882379F0E091A2
:101C70000F20F0E0EF71F070E055F84E808190E0B9
:101C800020910F202F5F20930F2008958FEF9FEF5B
:101C90000895CF93DF93EC0110929506109294066D
:101CA00088819981009731F022E08E3B920709F0FC
:101CB000B7C009C00E942D0E882341F48EEB92E03C
:101CC00099838883B1C0613109F0AEC0F8947894EB
:101CD0000E94330E90E09093A1068093A0068D3071
:101CE00009F47CC08F3F31F38231910569F18F3760
:101CF000910521F08830910509F053C08091A2062A
:101D00009091A306181619060CF060C06091302D52
:101D10007091312D88E090E00E94DA746091302D4E
:101D20007091312D80E290E00E94DA746091302D44
:101D30007091312D88E090E00E94DA748091A206C3
:101D40009091A30601973EC06091302D7091312D86
:101D50008DE090E00E94DA741092A5061092A4061D
:101D600014C0805F9F4DFC0180816091302D709187
:101D7000312D90E00E94DA748091A4069091A5061E
:101D800001969093A5068093A4068091A406909155
:101D9000A5062091A2063091A306821793070CF3A3
:101DA00015C06091302D7091312D0E94DA748091B0
:101DB000A2069091A3062091A006FC01E05FFF4DD2
:101DC000208301969093A3068093A2068091A20699
:101DD0009091A3068F33910509F06CCF10920F20DC
:101DE00010925B178091A2069091A306FC01E05F20
:101DF000FF4D108290939506809394061092A3064F
:101E00001092A20680916E2490916F24009709F49D
:101E100051CF60919E0640E050E00E94FE384ACFCC
:101E20001982188283E001C081E0DF91CF9108958B
:101E3000789480918F0690919006009731F0809170
:101E4000DE049091DF0490FF03C083B7817F03C05D
:101E500083B7817F866083BFF89483B7816083BF37
:101E60007894889583B78E7F83BF78940895CF93B5
:101E7000DF93EC0188819981009721F029E08D366C
:101E8000920789F40E94180F8091440E9091450E9C
:101E900065E840E050E00E94FE388DE699E09983C5
:101EA000888381E003C01982188283E0DF91CF919B
:101EB0000895CF93DF938EE40E942B448823B1F4DE
:101EC0000E947A448091F91B9091FA1B8160909353
:101ED000FA1B8093F91B00D08EEC91E0EDB7FEB7B2
:101EE000928381830E9418750F900F908EEE0E944E
:101EF0002B448823B1F40E947A448091F91B90917D
:101F0000FA1B82609093FA1B8093F91B00D087ED37
:101F100091E0EDB7FEB7928381830E9418750F9010
:101F20000F9086EA0E942B448823B1F40E947A44E1
:101F30008091F91B9091FA1B84609093FA1B809317
:101F4000F91B00D08FED91E0EDB7FEB7928381834E
:101F50000E9418750F900F908CE30E942B448823E9
:101F6000B1F40E947A448091F91B9091FA1B886029
:101F70009093FA1B8093F91B00D088EE91E0EDB7A7
:101F8000FEB7928381830E9418750F900F9082EDA7
:101F90000E942B448823B1F40E947A448091F91B5B
:101FA0009091FA1B80619093FA1B8093F91B00D0EB
:101FB00081EF91E0EDB7FEB7928381830E9418759F
:101FC0000F900F90C7E0D0E08CE70E942B4488234D
:101FD000B9F40E947A448091F91B9091FA1B8062B7
:101FE0009093FA1B8093F91B00D08BEF91E0EDB733
:101FF000FEB7928381830E9418750F900F9002C0E4
:10200000219711F70E94940BDF91CF910895CF9300
:10201000DF9300D0CDB7DEB74A8369830E94504476
:102020006981862F0E9482444A81842F0E948244C3
:102030000E947A440F900F90DF91CF910895AF9254
:10204000BF92DF92EF92FF920F931F93CF93DF9394
:1020500000D00F92CDB7DEB7082FD22E4A835B8314
:1020600069830E9450446981862F0E948244802F98
:1020700081600E9477444A81042F5B81152FEE24F2
:10208000FF24AD2CBB240894A108B1080FC0EA14AA
:10209000FB0419F40E949D4402C00E949344F8017D
:1020A00080830894E11CF11C0F5F1F4FED1478F33F
:1020B0000E947A440F900F900F90DF91CF911F9163
:1020C0000F91FF90EF90DF90BF90AF900895CF9366
:1020D000DF9300D0CDB7DEB71A8219828EEE6AEA9E
:1020E000AE014F5F5F4F22E00E941F10398120E058
:1020F0008A8190E0822B932B9093D1178093D017F5
:102100008EEE6CEAAE014F5F5F4F22E00E941F101F
:10211000398120E08A8190E0822B932B9093D31712
:102120008093D2178EEE6EEAAE014F5F5F4F22E0D2
:102130000E941F10398120E08A8190E0822B932B2E
:102140009093D5178093D4178EEE60EBAE014F5F5E
:102150005F4F22E00E941F10398120E08A8190E0C9
:10216000822B932B9093E3178093E2178EEE62EB12
:10217000AE014F5F5F4F22E00E941F10398120E0C7
:102180008A8190E0822B932B9093E5178093E4173C
:102190008EEE64EBAE014F5F5F4F22E00E941F1096
:1021A000398120E08A8190E0822B932B9093E7176E
:1021B0008093E6178EEE66EBAE014F5F5F4F22E035
:1021C0000E941F10398120E08A8190E0822B932B9E
:1021D0009093D7178093D6178EEE68EBAE014F5FC2
:1021E0005F4F22E00E941F10398120E08A8190E039
:1021F000822B932B9093D9178093D8178EEE6AEB8E
:10220000AE014F5F5F4F22E00E941F10398120E036
:102210008A8190E0822B932B9093DD178093DC17BB
:102220008EEE6CEBAE014F5F5F4F22E00E941F10FD
:10223000398120E08A8190E0822B932B9093DF17E5
:102240008093DE178EEE6EEBAE014F5F5F4F22E0A4
:102250000E941F10398120E08A8190E0822B932B0D
:102260009093E1178093E0170F900F90DF91CF913B
:1022700008952F923F924F925F926F927F928F922A
:102280009F92AF92BF92CF92DF92EF92FF920F9305
:102290001F93CF93DF93CDB7DEB76C970FB6F8944B
:1022A000DEBF0FBECDBF882E4A8F2B8FFE01319629
:1022B00083E0DF011D928A95E9F78091F417882366
:1022C00039F46C8F0E94671081E08093F4176C8D55
:1022D000662309F478C08EEE64EF4EE20E94071088
:1022E00069E07AE180E090E00E9418448EEE66EFAB
:1022F000AE014F5F5F4F22E00E941F10898190E086
:10230000A0E0B0E0BA2FA92F982F88274A8150E08B
:1023100060E070E0842B952BA62BB72B2091E6175D
:102320003091E717A90160E070E0841B950BA60BC4
:10233000B70B2091E4173091E51740E050E0BC0165
:10234000CD010E9415716B017C01AFE0F594E7941B
:10235000D794C794AA95D1F76091DE177091DF17D3
:10236000882777FD8095982FBBE0660F771F881F21
:10237000991FBA95D1F72091E0173091E1174427C2
:1023800037FD4095542F2C0D3D1D4E1D5F1D0E94A5
:102390007D712C0D3D1D3093DB172093DA17285FDC
:1023A0003F4F14E0359527951A95E1F76901EE2422
:1023B000D7FCE094FE2CC092E817D092E917E09287
:1023C000EA17F092EB17082D0295000F000F007C22
:1023D0000C5C282D30E0398F288F63E070E0082CEA
:1023E00002C0660F771F0A94E2F7882777FD809571
:1023F000982F25E335E040E050E00E941571DC01A4
:10240000CB010296A11DB11D888B998BAA8BBB8B2A
:1024100020E533EC40E050E004C0559547953795F2
:1024200027958A94D2F72C8B3D8B4E8B5F8B10E0D7
:102430001C861D861E861F86E8E02E2E312C488DB8
:10244000598D241A350A73C18EEE64EF402F0E9415
:102450000710688979898A899B890E9418448EEEC1
:1024600066EFAE014F5F5F4F23E00E941F10809127
:10247000DA179091DB17805A9F409C01442737FD63
:102480004095542F2C833D834E835F83CA01B9014D
:102490000E9415712B013C016091D4177091D517E2
:1024A000882777FD8095982F0E9415716B017C011C
:1024B000BDE0F594E794D794C794BA95D1F76091AD
:1024C000D6177091D717882777FD8095982FA3018D
:1024D0009201ECE05595479537952795EA95D1F708
:1024E0000E941571DC01CB01CD01BB2797FDB09592
:1024F000AB2FC80ED91EEA1EFB1E82E090E0A0E0C2
:10250000B0E0C80ED91EEA1EFB1EE2E0F594E79487
:10251000D794C794EA95D1F720E030E840E050E046
:10252000C20ED31EE41EF51E2091E2173091E31770
:1025300040E050E0C701B6010E941571DC01CB01FB
:10254000FFE0B695A79597958795FA95D1F7888777
:102550009987AA87BB8789809924AA24BB24540120
:10256000992488248A8190E0A0E0B0E0BA2FA92FB6
:10257000982F8827882A992AAA2ABB2A8B8190E03B
:10258000A0E0B0E0882A992AAA2ABB2A022C04C01B
:10259000B594A794979487940A94D2F7C090D017D3
:1025A000D090D117EE24D7FCE094FE2CE2E0CC0CC6
:1025B000DD1CEE1CFF1CEA95D1F76091D8177091D5
:1025C000D917882777FD8095982FA30192010E9443
:1025D00015712B013C01F7E175946794579447946A
:1025E000FA95D1F76091D2177091D317882777FDAC
:1025F0008095982F2C813D814E815F810E941571BD
:10260000DC01CB01EBE0B595A79597958795EA9509
:10261000D1F7480E591E6A1E7B1EC40CD51CE61C41
:10262000F71C088C04C0CC0CDD1CEE1CFF1C0A94AB
:10263000D2F722E030E040E050E0C20ED31EE41EAC
:10264000F51EF2E0F594E794D794C794FA95D1F784
:102650008C189D08AE08BF08C501B4012C893D89BE
:102660004E895F890E94157197FD0DC0660F771F17
:10267000881F991F288539854A855B850E945B7173
:1026800049015A010CC0288539854A855B850E941D
:102690005B7149015A01880C991CAA1CBB1C552767
:1026A000B7FC5A954B2D3A2D292DCA01B9010E942C
:1026B00015712EED3BE040E050E00E9415716C0179
:1026C000FF24D7FCF094EF2CC501B40123E433EED2
:1026D0004FEF5FEF0E941571DC01CB01CD01BB27ED
:1026E00097FDB095AB2FC80ED91EEA1EFB1E8FECCE
:1026F0009EE0A0E0B0E0C80ED91EEA1EFB1EE4E09A
:10270000F594E794D794C794EA95D1F7C80CD91CEF
:10271000EA1CFB1C2C853D854E855F852C0D3D1DDF
:102720004E1D5F1D2C873D874E875F871F5F3A8D4B
:10273000131709F089CE112391F0212F30E040E0EA
:1027400050E06C857D858E859F850E945B7120930E
:10275000EC173093ED174093EE175093EF174B8D16
:102760004423E9F16091EC177091ED178091EE1719
:102770009091EF17611571058105910581F10E9416
:102780009D6E20E836EE45EC57E40E94336E21E062
:102790003EED42E45EE30E94B06FB62FA72F382FC4
:1027A000292F60E070E080E89FE3FD01A9010F2F71
:1027B0001E2F252F342FA90198010E94CA6D2BE4EA
:1027C0003AE34DEB57E30E94336EDC01CB0180937B
:1027D000F0179093F117A093F217B093F3176C963C
:1027E0000FB6F894DEBF0FBECDBFDF91CF911F9122
:1027F0000F91FF90EF90DF90CF90BF90AF909F90A0
:102800008F907F906F905F904F903F902F900895A2
:10281000CF93DF9300D000D000D0CDB7DEB7FE015C
:10282000319686E0DF011D928A95E9F780915A176B
:10283000882399F486EA61E340E00E94071086EA63
:102840006CE24AE00E94071081E080935A176CE71F
:102850007EE380E090E00E94184486EA6DE248E062
:102860000E9407106CE77EE380E090E00E9418442D
:1028700086EA62E3AE014F5F5F4F26E00E941F10C1
:1028800086EA6DE247E00E9407109A8180E0698144
:1028900070E0682B792B70935517609354179C81C7
:1028A00080E04B8150E0482B592B509357174093B1
:1028B00056173E8120E08D8190E0822B932B9093E0
:1028C0005917809358172DB73EB7285030400FB690
:1028D000F8943EBF0FBE2DBFEDB7FEB7319628E886
:1028E00032E0ADB7BEB712963C932E931197738327
:1028F000628355834483978386830E9406752DB730
:102900003EB7285F3F4F0FB6F8943EBF0FBE2DBFB6
:1029100026960FB6F894DEBF0FBECDBFDF91CF91E4
:1029200008950F931F93CF93DF9300D000D000D072
:10293000CDB7DEB78E010F5F1F4F86E0D8011D9225
:102940008A95E9F78CE362E041E00E9407108CE38E
:1029500060E048E50E94071062E174E380E090E0E7
:102960000E9418448CE363E0A80126E00E941F1037
:102970008CE362E043E00E940710998180E06A8165
:1029800070E0682B792B70933B1760933A179B810B
:1029900080E04C8150E0482B592B50933D174093D9
:1029A0003C173D8120E08E8190E0822B932B909309
:1029B0003F1780933E17EDB7FEB738970FB6F894E0
:1029C000FEBF0FBEEDBF319626E932E0ADB7BEB710
:1029D00012963C932E93119773836283558344839D
:1029E000978386830E940675EDB7FEB738960FB6BB
:1029F000F894FEBF0FBEEDBF26960FB6F894DEBF6B
:102A00000FBECDBFDF91CF911F910F910895CF934E
:102A1000DF93EC0188819981009731F029E08735B7
:102A2000920709F071C00BC08AEB96E060E870E095
:102A30000E94923B87E599E09983888369C08AEB7D
:102A400096E00E94BD3B009709F462C08091920617
:102A50009091930694FF3FC08091F91B81FF3BC08A
:102A600083E061E048E021E00E9439118DB79EB714
:102A70000A970FB6F8949EBF0FBE8DBFEDB7FEB795
:102A800031968FEC9BE0ADB7BEB712969C938E93B8
:102A900011978091EC179091ED17A091EE17B091DE
:102AA000EF1782839383A483B5838091F01790916D
:102AB000F117A091F217B091F31786839783A0873F
:102AC000B1870E9418758DB79EB70A960FB6F89415
:102AD0009EBF0FBE8DBF809192069091930695FF89
:102AE00006C08091F91B82FF02C00E9408148091E9
:102AF00092069091930696FF97CF8091F91B83FFE2
:102B000093CF0E94911490CF1982188283E001C064
:102B100081E0DF91CF910895FF920F931F93CF93A0
:102B2000DF93729A8091DE0483FD06C0C0E5D0E099
:102B30000E949D092197E1F78EE40E942B4488238F
:102B400009F08BC0C0E5D0E00E949D092197E1F714
:102B50008FE40E942B440E949344C82F829586954F
:102B6000869583708130A9F4409103205091042010
:102B700060910520709106204F5F5F4F6F4F7F4F30
:102B80004093032050930420609305207093062007
:102B900016C08230A0F0409107205091082060912B
:102BA000092070910A204F5F5F4F6F4F7F4F409316
:102BB0000720509308206093092070930A200E94F8
:102BC00093441C2F1F7300E0080F111D0E949344B3
:102BD000F82E0E949D44DF2D90E0C92FC80FD11D13
:102BE000D695C795D695C7950E947A448091DE0404
:102BF00083FF7298B80180E090E00E949B6E20E114
:102C000034E048EC5BE30E944D6FDC01CB01809324
:102C1000F5179093F617A093F717B093F817BE0126
:102C200080E090E00E949B6E24EA3CEF44E25CE38B
:102C30000E944D6F20E030E040E252E40E94CA6DF5
:102C4000DC01CB018093712490937224A0937324B0
:102C5000B093742480E090E015C08091FF1F9091A4
:102C60000020A0910120B09102200196A11DB11D6C
:102C70008093FF1F90930020A0930120B093022027
:102C800081E090E0DF91CF911F910F91FF90089527
:102C90007298729A8EE40E942B4480EA0E948244C9
:102CA00080E00E94824480E00E9482448FE40E947F
:102CB0002B440E949344829586958695837081303B
:102CC000A9F4409103205091042060910520709157
:102CD00006204F5F5F4F6F4F7F4F4093032050930D
:102CE0000420609305207093062016C08230A0F067
:102CF00040910720509108206091092070910A208E
:102D00004F5F5F4F6F4F7F4F4093072050930820D6
:102D10006093092070930A2000D000D0EDB7FEB771
:102D2000319624EA32E0ADB7BEB712963C932E93AB
:102D30001197828313820E9406750F900F900F9057
:102D40000F908EE40E942B4480E80E94824480E031
:102D50000E94824480E00E9482440E947A4480E083
:102D600090E0089500D085E092E0ADB7BEB712962E
:102D70009C938E9311970E9418752091FA040F90DE
:102D80000F902223A9F000D000D0EDB7FEB7319606
:102D900082E192E0ADB7BEB712969C938E931197E5
:102DA000228313820E9418750F900F900F900F903E
:102DB000089500D085E192E0EDB7FEB7928381835C
:102DC0000E9418758AE392E0EDB7FEB79283818383
:102DD0000E94187582E692E0EDB7FEB79283818378
:102DE0000E94187589E892E0EDB7FEB7928381835F
:102DF0000E94187583EB92E0EDB7FEB79283818352
:102E00000E9418758EEE92E0EDB7FEB79283818333
:102E10000E94187588E193E0EDB7FEB79283818335
:102E20000E9418758EE393E0EDB7FEB7928381831D
:102E30000E9418758EE693E0EDB7FEB7928381830A
:102E40000E94187587EA93E0EDB7FEB792838183FD
:102E50000E94187583ED93E0EDB7FEB792838183EE
:102E60000E9418758CEF93E0EDB7FEB792838183D3
:102E70000E9418758BE294E0EDB7FEB792838183D0
:102E80000E9418758DE594E0EDB7FEB792838183BB
:102E90000E9418758EE894E0EDB7FEB792838183A7
:102EA0000E94187582EC94E0EDB7FEB7928381839F
:102EB0000E94187582EF94E0EDB7FEB7928381838C
:102EC0000E9418758EE195E0EDB7FEB7928381837D
:102ED0000E9418758DE495E0EDB7FEB7928381836B
:102EE0000E94187586E795E0EDB7FEB7928381835F
:102EF0000E94187585EA95E0EDB7FEB7928381834D
:102F00000E94187584ED95E0EDB7FEB7928381833A
:102F10000E9418758BEF95E0EDB7FEB79283818321
:102F20000E94187581E396E0EDB7FEB79283818326
:102F30000E9418750F900F90089584EB92E00E9404
:102F40003F7508954F925F926F927F928F929F92FA
:102F5000AF92BF92CF92DF92EF92FF920F931F93A7
:102F6000CF93DF9300D000D0CDB7DEB76091FB1FC9
:102F70007091FC1F8091FD1F9091FE1F8090FB1FA0
:102F80009090FC1FA090FD1FB090FE1F4090FB1F73
:102F90005090FC1F6090FD1F7090FE1F2091FB1F42
:102FA0003091FC1F4091FD1F5091FE1F29833A83F1
:102FB0004B835C834DB75EB74A5050400FB6F894D0
:102FC0005EBF0FBE4DBF0DB71EB70F5F1F4F2CE585
:102FD00036E0EDB7FEB732832183A0E8CA2EA1E523
:102FE000DA2EA1E0EA2EF12CA70196010E945B7176
:102FF000F80133832283C501B401A70196010E9421
:103000005B71B0E1CB2EBEE0DB2EE12CF12CA701F1
:1030100096010E945B71332727FD3095F8013583B7
:103020002483C301B201A70196010E945B712CE3C6
:10303000C22ED12CE12CF12CA70196010E945B71CC
:10304000332727FD3095F8013783268369817A81FC
:103050008B819C81A70196010E945B71772767FD98
:103060007095F801718760870E9418752DB73EB77B
:10307000265F3F4F0FB6F8943EBF0FBE2DBF0F9097
:103080000F900F900F90DF91CF911F910F91FF90B4
:10309000EF90DF90CF90BF90AF909F908F907F90F8
:1030A0006F905F904F900895E6E3FDE280819181FB
:1030B00022E482349207B9F000D000D08CE796E089
:1030C000ADB7BEB712969C938E931197E653FD420F
:1030D0001496FC93EE9313970E9418750F900F901F
:1030E0000F900F9008953A96B1E4E53FFB07F0F298
:1030F0000895EF92FF920F931F93CF93DF930E9457
:103100008D0ADC01CB0100D000D000D02AE936E0E6
:10311000EDB7FEB73283218383839483A583B6837F
:103120000E9418758DB79EB706960FB6F8949EBF8D
:103130000FBE8DBF81E00E94390A2091FF043091BB
:10314000000540910105509102050E944D6F8B01D1
:10315000D82FC92F82E00E94390AAB01BC01EDB71C
:10316000FEB73A970FB6F894FEBF0FBEEDBFEDB6AF
:10317000FEB60894E11CF11C21EA36E0328321837B
:103180009E01802F912FA32FB22FF701828393836B
:10319000A483B583CB01BA012091FB043091FC04D8
:1031A0004091FD045091FE040E944D6FDC01CB0163
:1031B000F70186839783A087B1870E9418758DB722
:1031C0009EB70A960FB6F8949EBF0FBE8DBF0E94A1
:1031D000940BDF91CF911F910F91FF90EF90089585
:1031E000EF92FF920F931F93CF93DF93882389F081
:1031F00085E694E26FEF70E049E050E00E94907441
:1032000085E694E260E070E049E050E00E945E767E
:1032100022C005E614E2C0E0D0E03DEAE32E36E04D
:10322000F32ED8018D918D0100D000D0EDB7FEB7FF
:103230003196ADB7BEB71296FC92EE92119782838B
:1032400013820E94187521960F900F900F900F9087
:10325000C830D10531F70E94940BDF91CF911F91B7
:103260000F91FF90EF900895CF92DF92EF92FF922F
:103270006091F8047091F90480E090E00E948274FB
:1032800065ED72E00E949774009709F07BC083E1BE
:103290009AE09093E3048093E20482EE94E06DE080
:1032A00070E042E050E00E945E768CE390E0909304
:1032B000E1048093E00480EE94E06BE070E042E093
:1032C00050E00E945E768AE090E09093DF04809365
:1032D000DE048EED94E069E070E042E050E00E9490
:1032E0005E76109293061092920682E996E06BE168
:1032F00070E042E050E00E945E760F2EF2E2CF2EA8
:10330000FFEFDF2EFCECEF2EFBE3FF2EF02DC09243
:10331000FF04D0920005E0920105F09202058FEFC4
:1033200094E063E170E044E050E00E945E76C09279
:10333000FB04D092FC04E092FD04F092FE048BEFBB
:1033400094E06FE070E044E050E00E945E768DEE25
:1033500097E4AAE8BCE38093030590930405A09347
:103360000505B093060583E095E067E170E044E071
:1033700050E00E945E7681E00E94F01880E090E0CC
:103380000E94300DFF90EF90DF90CF90089588233A
:1033900009F401C18091E20480FF0BC000D082EBF0
:1033A00096E0EDB7FEB7928381830E9418750F9067
:1033B0000F908091E20481FF0BC000D088EB96E073
:1033C000EDB7FEB7928381830E9418750F900F901E
:1033D0008091E20482FF0BC000D08DEB96E0EDB748
:1033E000FEB7928381830E9418750F900F90809191
:1033F000E20483FF0BC000D083EC96E0EDB7FEB78C
:10340000928381830E9418750F900F908091E2043F
:1034100084FF0BC000D08CEC96E0EDB7FEB7928332
:1034200081830E9418750F900F908091E20485FFB0
:103430000BC000D085ED96E0EDB7FEB79283818397
:103440000E9418750F900F908091E20486FF0BC0C8
:1034500000D08BED96E0EDB7FEB7928381830E949A
:1034600018750F900F908091E20487FF0BC000D079
:1034700083EE96E0EDB7FEB7928381830E941875C4
:103480000F900F908091E2049091E30490FF0BC0A5
:1034900000D089EE96E0EDB7FEB7928381830E945B
:1034A00018750F900F908091E2049091E30491FFC2
:1034B0000BC000D081EF96E0EDB7FEB79283818319
:1034C0000E9418750F900F908091E2049091E30490
:1034D00092FF0BC000D08BEF96E0EDB7FEB7928362
:1034E00081830E9418750F900F908091E204909153
:1034F000E30493FF0BC000D081E097E0EDB7FEB787
:10350000928381830E9418750F900F908091E2043E
:103510009091E30494FF0BC000D089E097E0EDB7F1
:10352000FEB7928381830E9418750F900F9080914F
:10353000E2049091E30495FF0BC000D08FE097E088
:10354000EDB7FEB7928381830E9418750F900F909C
:103550008091E2049091E30496FF0BC000D085E1D6
:1035600097E0EDB7FEB7928381830E9418750F90A4
:103570000F908091E2049091E30497FF4AC100D03C
:103580008AE197E0EDB7FEB7928381830E941875B8
:103590000F900F903EC100D000D080E297E0EDB7D1
:1035A000FEB79283818381E090E0948383830E94BD
:1035B00018750F900F900F900F900E94940B00D0F1
:1035C00000D08CE297E0EDB7FEB79283818382E072
:1035D00090E0948383830E9418750F900F900F9052
:1035E0000F900E94940B00D000D087E397E0EDB7D6
:1035F000FEB79283818384E090E0948383830E946A
:1036000018750F900F900F900F900E94940B00D0A0
:1036100000D083E497E0EDB7FEB79283818388E022
:1036200090E0948383830E9418750F900F900F9001
:103630000F900E94940B00D000D081E597E0EDB789
:10364000FEB79283818380E190E0948383830E941C
:1036500018750F900F900F900F900E94940B00D050
:1036600000D08FE597E0EDB7FEB79283818380E2CB
:1036700090E0948383830E9418750F900F900F90B1
:103680000F900E94940B00D000D08BE697E0EDB72E
:10369000FEB79283818380E490E0948383830E94C9
:1036A00018750F900F900F900F900E94940B00D000
:1036B00000D089E797E0EDB7FEB79283818380E879
:1036C00090E0948383830E9418750F900F900F9061
:1036D0000F900E94940B00D000D085E897E0EDB7E2
:1036E000FEB79283818380E091E0948383830E947C
:1036F00018750F900F900F900F900E94940B00D0B0
:1037000000D083E997E0EDB7FEB79283818380E034
:1037100092E0948383830E9418750F900F900F900E
:103720000F900E94940B00D000D082EA97E0EDB792
:10373000FEB79283818380E094E0948383830E9428
:1037400018750F900F900F900F900E94940B00D05F
:1037500000D08EEA97E0EDB7FEB79283818380E0D8
:1037600098E0948383830E9418750F900F900F90B8
:103770000F900E94940B00D000D08CEB97E0EDB737
:10378000FEB79283818380E090E1948383830E94DB
:1037900018750F900F900F900F900E94940B00D00F
:1037A00000D088EC97E0EDB7FEB79283818380E08C
:1037B00090E2948383830E9418750F900F900F906E
:1037C0000F900E94940B00D000D084ED97E0EDB7ED
:1037D000FEB79283818380E090E4948383830E9488
:1037E00018750F900F900F900F900E94940B00D0BF
:1037F00000D08FED97E0EDB7FEB79283818380E034
:1038000090E8948383830E9418750F900F900F9017
:103810000F900E94940B08952F923F924F925F92C7
:103820006F927F928F929F92AF92BF92CF92DF92D0
:10383000EF92FF920F931F93CF93DF9300D0CDB7FA
:10384000DEB79A838983DC018D919C911197009753
:1038500011F00C94AB2D6091F8047091F90480E1A3
:1038600090E20E94827480E190E260E470E00E9445
:10387000A074009759F46091302D7091312D8AE039
:1038800090E00E94DA7481E00C94B12D81309105B2
:1038900049F42090102033244424552466247724AE
:1038A0004301BEC18230910599F4309110202091DE
:1038B0001120932F80E0820F911D1C01892F880F0A
:1038C000880B482E582E682E782E882E982EA8C148
:1038D0008330910509F09CC0209110208090112028
:1038E000B090122030E040E050E060E070E080E016
:1038F00090E000E10E940B69922EA32E142FF52E6A
:10390000E62EC72E282ED92E282D30E040E050E09C
:1039100060E070E080E090E008E00E940B69290D13
:10392000B1E0291508F0B0E03A0DE1E03A1508F0F1
:10393000E0E0B30FF1E0B31708F0F0E0EF2B410F38
:1039400031E0411708F030E0E40FF1E0E41708F04F
:10395000F0E03F2B5F0D41E05F1508F040E0A32F42
:10396000A50F31E0A51708F030E0432B6E0D31E0D4
:103970006E1508F030E0F42FF60F41E0F61708F06E
:1039800040E0342B7C0D41E07C1508F040E0532FE3
:10399000570F31E0571708F030E0432B820D31E02C
:1039A000821508F030E0480F61E0481708F060E049
:1039B000362BD90ED30EB20E81E0B21608F080E09D
:1039C000182F1B0F71E01B1708F070E07E0F61E0ED
:1039D0007E1708F060E06A0F31E06A1708F030E007
:1039E0003F0F21E03F1708F020E0250F91E0251759
:1039F00008F090E0940F81E0941708F080E02B2C01
:103A0000312E472E562E632E722E892E982EFDC0F3
:103A10008430910509F0FBC0209110208090112086
:103A2000A0901220B090132030E040E050E060E021
:103A300070E080E090E008E10E940B69722E932E06
:103A4000142FF52EE62EC72E282ED92E282D30E045
:103A500040E050E060E070E080E090E000E10E9433
:103A60000B69270DF1E0271508F0F0E0390DE1E0D2
:103A7000391508F0E0E0F30FA1E0F31708F0A0E03B
:103A8000EA2B410F31E0411708F030E0E40FA1E0EC
:103A9000E41708F0A0E03A2B5F0D41E05F1508F055
:103AA00040E0B32FB50F31E0B51708F030E0432BFD
:103AB0006E0D31E06E1508F030E0A42FA60F41E046
:103AC000A61708F040E0342B7C0D41E07C1508F08F
:103AD00040E0532F570F31E0571708F030E0432BE9
:103AE000820D31E0821508F030E0480F61E04817A0
:103AF00008F060E0362BD90ED30E222E2B0C81E07D
:103B0000221608F080E0B82EBF0E81E0BF1608F044
:103B100080E0982E9E0E81E09E1608F080E0C82E70
:103B2000CB0E11E0CB1608F010E01A0F81E01A1747
:103B300008F080E0F82EF50E81E0F51608F080E040
:103B4000E82EE40E81E0E41608F080E0D80E2A2D7D
:103B500030E040E050E060E070E080E090E008E0BD
:103B60000E940B69220DE1E0221508F0E0E03B0D18
:103B7000F1E03B1508F0F0E0E30FA1E0E31708F0F7
:103B8000A0E0FA2B490D31E0491508F030E0F40FC0
:103B9000A1E0F41708F0A0E03A2B5C0D41E05C15C1
:103BA00008F040E0A32FA50F31E0A51708F030E0A2
:103BB000432B610F31E0611708F030E0542F560FAE
:103BC00041E0561708F040E0342B7F0D41E07F15AF
:103BD00008F040E0632F670F31E0671708F030E02E
:103BE000432B8E0D31E08E1508F030E0480F71E068
:103BF000481708F070E0372BD90E222E3E2E4F2E9C
:103C00005A2E652E762E842E932E9D0C09C0FAE036
:103C10002F2E332444245524662477248824992481
:103C20000E94940BB3E62B1689F4EDE63E1671F470
:103C3000F8E64F1659F4552049F4662039F47720F8
:103C400029F4882019F4992009F40EC59101A201E4
:103C5000B301C40113E6A12E0DE6B02EE8E6CE2E88
:103C6000DD24EE24FF2400E010E00E94856982300C
:103C700008F04FC283E3281689F491E7391671F4EE
:103C8000442061F4552051F4662041F4772031F44A
:103C9000882021F4992011F40C94BB2C9101A201ED
:103CA000B301C401A3E3AA2EB1E7BB2ECC24DD24CB
:103CB000EE24FF2400E010E00E948569823008F0C5
:103CC00012C1A5E62A1681F4B4E63B1669F4442035
:103CD00059F4552049F4662039F4772029F48820D6
:103CE00019F4992009F456C69101A201B301C40147
:103CF000E5E6AE2EF4E6BF2ECC24DD24EE24FF2430
:103D000000E010E00E948569823008F06BC0E5E7B2
:103D10002E1679F4332069F4442059F4552049F4DF
:103D2000662039F4772029F4882019F4992009F4C1
:103D30007DC79101A201B301C40105E7A02EBB24F8
:103D4000CC24DD24EE24FF2400E010E00E948569ED
:103D5000823090F4F8E62F1611F00C94A92D332040
:103D600011F00C94A92D442011F00C94A92D55208C
:103D700011F00C94A92D88C386E7281679F4332016
:103D800069F4442059F4552049F4662039F4772029
:103D900029F4882019F4992009F457C794E62916C4
:103DA00011F00C94A92DA1E63A1611F00C94A92D4E
:103DB000442011F00C94A92D552011F00C94A92D3C
:103DC000662011F00C94A92D772011F00C94A92DE8
:103DD000882011F00C94A92D992011F00C94A92D94
:103DE0000C94BB2CB5E62B1689F4EEE63E1671F466
:103DF000442061F4552051F4662041F4772031F4D9
:103E0000882021F4992011F40C94ED289101A2014D
:103E1000B301C401B5E6AB2E1EE6B12ECC24DD24E1
:103E2000EE24FF2400E010E00E948569823018F53E
:103E3000F4E62F1611F00C94A92D89E6381611F02E
:103E40000C94A92D442011F00C94A92D552011F0AB
:103E50000C94A92D662011F00C94A92D772011F057
:103E60000C94A92D882011F00C94A92D992011F003
:103E70000C94A92DBBC697E7291689F4AFE63A162C
:103E800071F4442061F4552051F4662041F4772008
:103E900031F4882021F4992011F40C948F28B1E397
:103EA0002B1611F00C94A92DE0E73E1611F00C949E
:103EB000A92D442011F00C94A92D552011F00C943B
:103EC000A92D662011F00C94A92D772011F00C94E7
:103ED000A92D882011F00C94A92D992011F00C9493
:103EE000A92D0C947729F3E62F1691F484E6381661
:103EF00079F491E6491661F4552051F4662041F4B5
:103F0000772031F4882021F4992011F40C94BB2CF3
:103F10009101A201B301C401E3E6AE2EF4E6BF2E87
:103F2000A1E6CA2EDD24EE24FF2400E010E00E946A
:103F30008569823008F080C0A9E62A1689F4B2E7C4
:103F40003B1671F4442061F4552051F4662041F48D
:103F5000772031F4882021F4992011F40C94702AF0
:103F60009101A201B301C40119E6A12E02E7B02E0E
:103F7000CC24DD24EE24FF2400E010E00E948569BB
:103F8000823018F5E5E62E1611F00C94A92D3B149D
:103F900011F00C94A92D442011F00C94A92D55205A
:103FA00011F00C94A92D662011F00C94A92D772006
:103FB00011F00C94A92D882011F00C94A92D9920B2
:103FC00011F00C94A92D0C940A2AF3E72F1689F40A
:103FD00082E7381671F4442061F4552051F46620CC
:103FE00041F4772031F4882021F4992011F40C94C5
:103FF000C92A93E7291611F00C94A92D391611F04E
:104000000C94A92D442011F00C94A92D552011F0E9
:104010000C94A92D662011F00C94A92D772011F095
:104020000C94A92D882011F00C94A92D992011F041
:104030000C94A92D0C94D82AA3E72A1689F4B5E686
:104040003B1671F4E1E64E1659F4552049F466200A
:1040500039F4772029F4882019F4992009F404C64A
:104060009101A201B301C401F3E7AF2EA5E6BA2E78
:10407000B1E6CB2EDD24EE24FF2400E010E00E9408
:104080008569823018F5F8E72F1611F00C94A92DE8
:1040900084E6381611F00C94A92D4C1411F00C94F0
:1040A000A92D552011F00C94A92D662011F00C9427
:1040B000A92D772011F00C94A92D882011F00C94D3
:1040C000A92D992011F00C94A92DC6C292E62916AB
:1040D00089F4A5E63A1671F4B4E64B1659F4552066
:1040E00049F4662039F4772029F4882019F49920BE
:1040F00009F450C4E2E72E1611F00C94A92D3E16D7
:1041000011F00C94A92DF5E64F1611F00C94A92D81
:1041100007C189E6281691F49CE6391679F4A1E6E0
:104120004A1661F4B3E65B1649F4662039F4772049
:1041300029F4882019F4992009F4C2C29101A2013E
:10414000B301C401B9E6AB2E1CE6B12E01E6C02EC8
:10415000E3E6DE2EEE24FF2400E010E00E948569F5
:10416000823008F02BC1E5E72E1681F43D1471F47E
:10417000FDE64F1659F4552049F4662039F47720AE
:1041800029F4882019F4992009F44AC79101A20161
:10419000B301C401E5E7AE2EF3E6BF2EADE6CA2EAD
:1041A000DD24EE24FF2400E010E00E9485698230C7
:1041B00008F083C02B1489F482E3381671F499E671
:1041C000491659F4552049F4662039F4772029F42A
:1041D000882019F4992009F443C29101A201B30186
:1041E000C401B3E6AB2E12E3B12E09E6C02EDD24E6
:1041F000EE24FF2400E010E00E948569823028F55B
:10420000ADE62A1611F00C94A92DB5E73B1611F076
:104210000C94A92DE8E64E1611F00C94A92D55200A
:1042200011F00C94A92D662011F00C94A92D772083
:1042300011F00C94A92D882011F00C94A92D99202F
:1042400011F00C94A92D0C94CA2CF4E62F1689F4C5
:1042500083E6381671F49CE6491659F4552049F462
:10426000662039F4772029F4882019F4992009F47C
:1042700018C6A7E62A1611F00C94A92DBFE63B1626
:1042800011F00C94A92DECE64E1611F00C94A92D0A
:10429000552011F00C94A92D662011F00C94A92D35
:1042A000772011F00C94A92D882011F00C94A92DE1
:1042B000992011F00C94A92DF7C5F1E32F1681F484
:1042C0003F1671F481E7481659F4552049F46620E9
:1042D00039F4772029F4882019F4992009F4A0C62C
:1042E0009101A201B301C401E1E3AE2EF1E3BF2EBF
:1042F000A1E7CA2EDD24EE24FF2400E010E00E9496
:104300008569823010F590E3291611F00C94A92DDF
:104310003B1411F00C94A92D4C1411F00C94A92D00
:10432000552011F00C94A92D662011F00C94A92DA4
:10433000772011F00C94A92D882011F00C94A92D50
:10434000992011F00C94A92D08C6A0E72A1691F423
:10435000B5E63B1679F4E2E74E1661F4552051F4C8
:10436000662041F4772031F4882021F4992011F45B
:104370000C940A2AF4E72F1611F00C94A92D8FE65D
:10438000381611F00C94A92D481611F00C94A92D93
:1043900092E6591611F00C94A92D662011F00C9498
:1043A000A92D772011F00C94A92D882011F00C94E0
:1043B000A92D992011F00C94A92D8CC4A1E32A16E3
:1043C00091F4B2E73B1679F4E7E74E1661F4F0E7B3
:1043D0005F1649F4662039F4772029F4882019F40F
:1043E000992009F445C19101A201B301C401A1E3DF
:1043F000AA2EB2E7BB2E17E7C12E00E7D02EEE247F
:10440000FF2400E010E00E948569823008F088C037
:1044100081E6281691F49DE6391679F4A5E74A1647
:1044200061F4B8E65B1649F4662039F4772029F484
:10443000882019F4992009F487C69101A201B301DB
:10444000C40111E6A12E0DE6B02EE5E7CE2EF8E66A
:10445000DF2EEE24FF2400E010E00E948569823008
:1044600020F5E0E72E1611F00C94A92DFCE63F167E
:1044700011F00C94A92D85E6481611F00C94A92D85
:104480005D1411F00C94A92D662011F00C94A92D47
:10449000772011F00C94A92D882011F00C94A92DEF
:1044A000992011F00C94A92D9EC390E7291691F440
:1044B000ADE63A1679F4B5E74B1661F4E8E65E1618
:1044C00049F4662039F4772029F4882019F49920DA
:1044D00009F453C6F3E72F1611F00C94A92D85E6C5
:1044E000381611F00C94A92D92E7491611F00C948E
:1044F000A92DA0E75A1611F00C94A92D662011F0F1
:104500000C94A92D772011F00C94A92D882011F07E
:104510000C94A92D992011F00C94A92D0C94142D14
:10452000B4E72B1689F4E3E73E1671F4F5E64F166F
:1045300059F45B1649F4662039F4772029F4882071
:1045400019F4992009F4C9C39101A201B301C4016E
:10455000E4E7AE2EF3E7BF2EA5E6CA2EB4E7DB2EC6
:10456000EE24FF2400E010E00E9485698230C8F547
:104570002B1491F482E7381679F497E7491661F421
:10458000A0E75A1649F4662039F4772029F48820E8
:1045900019F4992009F4F6C6B4E72B1611F00C941F
:1045A000A92DE3E73E1611F00C94A92DF5E64F1660
:1045B00011F00C94A92D82E7581611F00C94A92D36
:1045C000662011F00C94A92D772011F00C94A92DE0
:1045D000882011F00C94A92D992011F00C94A92D8C
:1045E00083C692E7291691F4A7E63A1679F4B0E764
:1045F0004B1661F4E5E75E1649F4662039F477203E
:1046000029F4882019F4992009F41AC4FCE62F161D
:1046100011F00C94A92D81E6381611F00C94A92DF7
:1046200094E7491611F00C94A92DA8E75A1611F039
:104630000C94A92D662011F00C94A92D772011F06F
:104640000C94A92D882011F00C94A92D992011F01B
:104650000C94A92D0C946F2D0E9408140C94AB2D72
:104660000E94590F0C94AB2D0E9491140C94AB2D09
:104670006091F8047091F90480E090E00E948274E7
:104680008C016CED72E00E949774009719F4779892
:104690000C94AB2DC8016FED72E00E9497740097E7
:1046A00019F4779A0C94AB2D779903C08CED92E0B6
:1046B00002C08FED92E000D000D02BEE37E003C3B4
:1046C0006091F8047091F90480E090E00E94827497
:1046D0008C0166EF72E00E949774009709F043C066
:1046E0006091F8047091F90480E090E00E94827477
:1046F0008C01009711F40C94AB2D69EF72E00E94CD
:104700009774009729F482E29FEFACECBBE318C0EA
:10471000C8010E9475736B017C0120E030E040E02D
:1047200050E00E942F6E8823D1F081E00E94390A68
:104730009B01AC01C701B6010E94336EDC01CB01C5
:104740008093FF0490930005A0930105B0930205A8
:104750008FEF94E063E170E044E050E040C600D0A9
:104760008FE49BE09DC0C8016FEF72E00E949774D8
:10477000009709F045C06091F8047091F90480E059
:1047800090E00E9482748C01009711F40C94AB2D80
:1047900069EF72E00E949774009729F482E29FEF1C
:1047A000ACECBBE318C0C8010E9475736B017C01BF
:1047B00020E030E040E050E00E942F6E8823C1F0FE
:1047C00082E00E94390A9B01AC01C701B6010E9438
:1047D000336EDC01CB018093FB049093FC04A09327
:1047E000FD04B093FE048BEF94E06FE070E0B4CF73
:1047F00000D08CE59BE0EDB7FEB79283818356C075
:10480000C80162E073E00E949774009709F054C0F9
:104810006091F8047091F90480E090E00E94827445
:104820008C01009711F40C94AB2D69EF72E00E949B
:104830009774009729F48DEE97E4AAE8BCE320C0B2
:10484000C8010E9475736B017C0120E030E040E0FC
:1048500050E00E942F6E882301F180E00E94390A07
:104860004B015C01C701B60121EE3AE744E95EE382
:104870000E94CA6DA50194010E94336EDC01CB0138
:104880008093030590930405A0930505B093060556
:1048900083E095E067E170E05FCF00D089E69BE0C0
:1048A000ADB7BEB712969C938E9311970E94187560
:1048B0000F900F900C94AB2D0E948D0AAB01BC01A0
:1048C00000D000D000D086E79BE0EDB7FEB7928322
:1048D000818343835483658376830E941875EDB783
:1048E000FEB736960FB6F894FEBF0FBEEDBF81E05F
:1048F0000E94390A2091FF04309100054091010582
:10490000509102050E944D6F6B01182F092F82E014
:104910000E94390AAB01BC018DB79EB70A970FB64A
:10492000F8949EBF0FBE8DBFEDB6FEB60894E11C95
:10493000F11C8DE79BE0ADB7BEB712969C938E93AA
:10494000119798018C2D9D2DA32FB22FF7018283F3
:104950009383A483B583CB01BA012091FB043091EA
:10496000FC044091FD045091FE040E944D6FDC0157
:10497000CB01F70186839783A087B1870E941875C2
:104980008DB79EB70A960FB6F8949EBF0FBE8DBF27
:104990000C94A62D6091F8047091F90480E090E0E9
:1049A0000E948274009771F160E070E040E150E095
:1049B0000E943472AB01BC018091920690919306E3
:1049C0008417950799F1509393064093920682E9D4
:1049D00096E06BE170E042E050E00E945E768091EC
:1049E00092069091930600D000D02FEE37E0ADB73D
:1049F000BEB712963C932E93119714969C938E9368
:104A000013970EC0809192069091930600D000D02B
:104A10002FEF37E0EDB7FEB7328321839483838392
:104A20000E9418750F900F900F900F900E94940B9A
:104A300000D000D083E198E0ADB7BEB712969C934A
:104A40008E93119781E090E014969C938E93139728
:104A50000E94187580E298E0EDB7FEB792838183DB
:104A600082E090E0948383830E9418758BE298E043
:104A7000ADB7BEB712969C938E93119784E090E0E9
:104A800014969C938E9313970E94187586E398E072
:104A9000EDB7FEB79283818388E090E094838383AF
:104AA0000E94187583E498E0ADB7BEB712969C9348
:104AB0008E93119780E190E014969C938E931397B8
:104AC0000E9418758EE498E0EDB7FEB7928381835B
:104AD00080E290E0948383830E9418758AE598E0D1
:104AE000ADB7BEB712969C938E93119780E490E079
:104AF00014969C938E9313970E94187588E698E0FD
:104B0000EDB7FEB79283818380E890E0948383833E
:104B10000E94187586E798E0ADB7BEB712969C93D1
:104B20008E93119780E091E014969C938E93139747
:104B30000E94187585E898E0EDB7FEB792838183EF
:104B400080E092E0948383830E94187584E998E062
:104B5000ADB7BEB712969C938E93119780E094E008
:104B600014969C938E9313970E94187580EA98E090
:104B7000EDB7FEB79283818380E098E094838383CE
:104B80000E9418758EEA98E0ADB7BEB712969C9356
:104B90008E93119780E090E114969C938E931397D7
:104BA0000E9418758BEB98E0EDB7FEB79283818376
:104BB00080E090E2948383830E94187589EC98E0EA
:104BC000ADB7BEB712969C938E93119780E090E498
:104BD00014969C938E9313970E9418750F900F90C4
:104BE0000F900F90B8C70E94D916B5C76091F8040E
:104BF0007091F90480E090E00E94827469EF72E0A5
:104C00000E949774009711F481E001C080E00E9437
:104C1000F0182091FA04222309F49DC700D000D097
:104C2000EDB7FEB7319689ED98E09EC20E94A217BB
:104C30002091FA04222309F48EC700D000D0EDB7EA
:104C4000FEB731968CED98E08FC20E949D1720919F
:104C5000FA04222309F47FC700D000D0EDB7FEB7D5
:104C600031968FED98E080C26091F8047091F9045C
:104C700080E090E00E9482748C016CED72E00E94F2
:104C80009774009731F48091DE049091DF04846082
:104C90009CC3C8016FED72E00E9497749C018091E3
:104CA000DE049091DF042115310511F48B7F8DC353
:104CB00082FF03C08CED92E002C08FED92E000D045
:104CC00000D029E83BE0EDB7FEB73283218394831F
:104CD000838382CF0C9400003EC76091F8047091EA
:104CE000F90480E090E00E9482748C0167E073E038
:104CF0000E949774009739F4219A8091DE04909174
:104D0000DF04806162C3C80169E073E00E949774A8
:104D1000009739F4229A8091DE049091DF0480623A
:104D200054C3C8016BE073E00E949774009739F494
:104D3000239A8091DE049091DF04806446C3C80109
:104D40006DE073E00E949774009739F4239A809184
:104D5000DE049091DF04806838C3C8016FED72E013
:104D60000E9497749C018091DE049091DF042115CC
:104D7000310539F48F709093DF048093DE042B9A11
:104D800028C384FF03C08CED92E002C08FED92E057
:104D900000D000D02DE83BE0ADB7BEB712963C93F3
:104DA0002E93119714969C938E9313970E941875C7
:104DB0008091DE040F900F900F900F9085FF03C03D
:104DC0008CED92E002C08FED92E000D000D028E997
:104DD0003BE0EDB7FEB732832183948383830E9447
:104DE00018758091DE040F900F900F900F9086FF42
:104DF00003C08CED92E002C08FED92E000D000D0B5
:104E000023EA3BE0ADB7BEB712963C932E931197C1
:104E100014969C938E9313970E9418758091DE04CC
:104E20000F900F900F900F9087FF03C08CED92E0D2
:104E300002C08FED92E000D000D02EEA3BE043CFDD
:104E400000D082EE98E0ADB7BEB712969C938E93D9
:104E500011970E9418752091FA040F900F90222349
:104E6000A9F000D000D0EDB7FEB7319686EE98E0FD
:104E7000ADB7BEB712969C938E931197228313827F
:104E80000E9418750F900F900F900F9088E10FB649
:104E9000F89480936000109260000FBE0C94007C28
:104EA0005AC60E94974557C66091F8047091F9045C
:104EB00080E090E00E9482747C016CED72E00E94C0
:104EC0009774009749F40E945A4B8091DE049091A8
:104ED000DF0481608D7F79C2C7016FED72E00E94AF
:104EE0009774009741F40E944B4C8091DE0490919E
:104EF000DF048C7F6AC20FE013E0C701B8010E9493
:104F00009774009749F40E944B4C8091DE04909175
:104F1000DF048E7F826059C28091DE0481FF0BC066
:104F200000D000D089EB9BE0EDB7FEB79283818380
:104F30001483038351CE80FF03C08CED92E002C046
:104F40008FED92E000D000D02DEB3BE0ADB7BEB7C7
:104F500012963C932E9311973BCE00D089EE98E0A9
:104F6000EDB7FEB7928381830E9418758DB79EB707
:104F700040970FB6F8949EBF0FBE8DBFEDB7FEB73A
:104F8000319683E199E0ADB7BEB712969C938E93AC
:104F9000119780910B2090910C20A0910D20B09141
:104FA0000E2082839383A483B5838091FF1F909109
:104FB0000020A0910120B091022086839783A087D2
:104FC000B1878091032090910420A0910520B09199
:104FD000062082879387A487B587809107209091C8
:104FE0000820A0910920B0910A2086879787A08B7E
:104FF000B18B0E9418752091FA04EDB7FEB7729636
:105000000FB6F894FEBF0FBEEDBF222309F4A3C56F
:1050100000D000D0EDB7FEB7319681E399E0A4C08F
:10502000F89409E081E090E0FC0100935700C895F6
:10503000F02C20E030E0F90100935700C895E02CF7
:105040007894F89423E030E0F90100935700C89574
:10505000102D82E090E0FC0100935700C895002DD0
:10506000789400D000D000D024E339E0EDB7FEB74B
:10507000328321838091AC179091AD17A091AE1728
:10508000B091AF1783839483A583B6830E9418756C
:1050900000D000D0EDB7FEB731968EE399E0ADB702
:1050A000BEB712969C938E9311970283138214833A
:1050B0001582E6821782F08611860E941875EDB778
:1050C000FEB73A960FB6F894FEBF0FBEEDBF0E9432
:1050D00054182091660000D000D0EDB7FEB731968D
:1050E00085E699E0ADB7BEB712969C938E93119763
:1050F000228313820E9418750F900F900F900F90CB
:105100000E94940B2091FA04222309F424C500D0B4
:1051100000D0EDB7FEB7319681E799E025C080E079
:1051200090E00E94A00B81E090E00E94A00B2091F3
:10513000FA04222309F40FC500D000D0EDB7FEB762
:10514000319684E799E010C00E9448160E94940BA3
:105150002091FA04222309F4FEC400D000D0EDB758
:10516000FEB7319687E799E0ADB7BEB712969C932C
:105170008E931197228313822FCD6091F804709142
:10518000F90480E090E00E9482748C016CED72E082
:105190000E949774009731F48091DE049091DF04AF
:1051A000886013C1C8016FED72E00E9497749C0182
:1051B0008091DE049091DF042115310511F4877F81
:1051C00004C183FF03C08CED92E002C08FED92E03A
:1051D00000D000D021EC3BE076CD6091F8047091D6
:1051E000F90480E090E00E94827464E173E00E9420
:1051F0009774009731F5F89488E996E00E94FA399F
:105200000CC0C8010D960E94123D8BE095E0B801DC
:105210000E94B239C8010E94A03A8C01009789F718
:1052200004C088E996E00E94273A88E996E00E9447
:10523000823A0097B1F788E996E00E94F6397894AF
:1052400046C088E996E00E94FA397C010AE113E041
:105250003BC08DB79EB70C970FB6F8949EBF0FBE9C
:105260008DBFEDB7FEB73196ADB7BEB712961C93A2
:105270000E931197D70112968C9112978283138205
:1052800013968C9113978483158218968C91189796
:105290008683178214968D919C91159791878087AC
:1052A00016968D919C911797938782870E94067519
:1052B000EDB7FEB73C960FB6F894FEBF0FBEEDBF3C
:1052C000C7010E94A03A7C01E114F10411F620917B
:1052D000FA04222309F43FC400D000D0EDB7FEB792
:1052E00031968AE799E040CF0E94341934C4609126
:1052F000F8047091F90480E090E00E9482748C01BF
:105300006CED72E00E949774009731F48091DE0496
:105310009091DF0492600EC0C8016FED72E00E94B0
:1053200097749C018091DE049091DF042115310572
:1053300071F49D7F9093DF048093DE048EED94E002
:1053400069E070E042E050E00E945E7617C091FF95
:1053500003C08CED92E002C08FED92E000D000D04F
:1053600025EC3BE0EDB7FEB7328321839483838342
:105370000E9418750F900F900F900F9081E00E947F
:10538000A509E9C36091F8047091F90480E090E008
:105390000E9482748C016EEE72E00E9497740097F6
:1053A00031F48091DE049091DF049E7F0EC0C8012D
:1053B00063EE72E00E9497749C018091DE049091EC
:1053C000DF042115310571F491609093DF0480931F
:1053D000DE048EED94E069E070E042E050E00E946F
:1053E0005E76B9C390FF03C083EE92E002C08EEEFA
:1053F00092E000D000D021E433E0ADB7BEB7129602
:105400003C932E93119714969C938E9313970E941E
:105410000675E4CB6091F8047091F90480E090E0A7
:105420000E948274009769F160E070E040E150E012
:105430000E943472DC01CB019093E3048093E20478
:1054400000D000D04DB75EB74F5F5F4F2DE739E01A
:10545000EDB7FEB732832183FA01938382830E94E2
:1054600018750F900F900F900F9082EE94E06DE002
:1054700070E042E050E00E945E7681E00E94C71931
:105480006AC380E00E94C7190E94940B00D000D02C
:105490008EE899E0ADB7BEB712969C938E931197A4
:1054A0008091E2049091E30414969C938E93139759
:1054B0000E9418750F900F900F900F9081E00E943E
:1054C000C7190E94940B2091FA04222309F443C3C4
:1054D00000D000D0EDB7FEB7319681EA99E044CE16
:1054E0006091F8047091F90480E090E00E94827469
:1054F000009751F160E070E04AE050E00E943472A1
:10550000DC01CB019093E1048093E00400D000D053
:105510004DB75EB74F5F5F4F24EA39E0EDB7FEB796
:1055200032832183FA01938382830E9418750F903E
:105530000F900F900F9080EE94E06BE070E042E0EF
:1055400050E00E945E7618C000D000D081EC99E057
:10555000ADB7BEB712969C938E9311978091E004DD
:105560009091E10414969C938E9313970E94187562
:105570000F900F900F900F902091FA04222309F4BE
:10558000EAC200D000D0EDB7FEB7319682EE99E0C6
:10559000EBCD0E944B3D2091FA04222309F4DBC29B
:1055A00000D000D0EDB7FEB7319685EE99E0DCCDA6
:1055B00000D088EE99E0EDB7FEB7928381830E9418
:1055C00018750F900F900E949D1700D088EF99E0FA
:1055D000ADB7BEB712969C938E9311970E94187523
:1055E0000F900F9080E00E94F01800D08CEF99E0AF
:1055F000EDB7FEB7928381830E9418750F900F90CC
:105600000E94590F0E94A21700D000D082E09AE0B9
:10561000ADB7BEB712969C938E93119780E490E03D
:1056200014969C938E9313970E94187500D0EDB733
:10563000FEB731968AE19AE0ADB7BEB712969C9359
:105640008E931197809175248283138280917624A2
:10565000848315820E9418750F900F908DE29AE056
:10566000EDB7FEB7928381838091E0049091E104CD
:10567000948383830E94187582E49AE0ADB7BEB725
:1056800012969C938E9311978091E2049091E3047B
:1056900014969C938E9313970E9418750F900F90F9
:1056A0000F900F9081E00E94C7190E948D0AAB01F4
:1056B000BC0100D000D000D085E59AE0EDB7FEB780
:1056C0009283818343835483658376830E94187514
:1056D000EDB7FEB736960FB6F894FEBF0FBEEDBF1E
:1056E0000E94D60A0E94A70AAB01BC0100D000D0DC
:1056F00000D082E69AE0ADB7BEB712969C938E9327
:105700001197EDB7FEB743835483658376830E9478
:1057100018758DB79EB706960FB6F8949EBF0FBE4C
:105720008DBF1D9B03C083EF92E002C08FED92E01E
:1057300000D000D020E73AE0ADB7BEB712963C9358
:105740002E93119714969C938E9313970E9418751D
:105750008091502490915124A0915224B0915324CF
:1057600040915424509155246091562470915724AF
:1057700000D000D000D00DB71EB70F5F1F4F2CE731
:105780003AE0EDB7FEB732832183F8018283938339
:10579000A483B58346835783608771870E941875F9
:1057A000EDB7FEB731968AE99AE0ADB7BEB712966B
:1057B0009C938E93119780915D2490915E24A0918B
:1057C0005F24B091602482839383A483B583809106
:1057D000612490916224A0916324B0916424868313
:1057E0009783A087B1870E941875EDB7FEB73896EA
:1057F0000FB6F894FEBF0FBEEDBF8CEB9AE092831C
:1058000081830E9418758091DE040F900F9081FFB4
:105810000EC000D086EC9AE0ADB7BEB712969C934E
:105820008E9311970E9418750F900F9017C080FFEC
:1058300003C08CED92E002C08FED92E000D000D06A
:105840002CEC3AE0EDB7FEB7328321839483838357
:105850000E9418750F900F900F900F908091DE04AA
:1058600083FF03C08CED92E002C08FED92E000D088
:1058700000D020ED3AE0ADB7BEB712963C932E9320
:10588000119714969C938E9313970E94187580918C
:10589000DE049091DF040F900F900F900F9091FF16
:1058A00003C08CED92E002C08FED92E000D000D0FA
:1058B00023EE3AE0EDB7FEB73283218394838383EE
:1058C0000E941875809192069091930620EF3AE01D
:1058D000ADB7BEB712963C932E93119714969C9336
:1058E0008E9313970E9418750F900F900F900F9042
:1058F000779903C08CED92E002C08FED92E000D06A
:1059000000D02DEF3AE0EDB7FEB7328321839483C8
:1059100083830E9418758091DE049091DF040F90BC
:105920000F900F900F9090FF03C083EE92E002C0A3
:105930008EEE92E000D000D021E433E0ADB7BEB7E8
:1059400012963C932E93119714969C938E931397D3
:105950000E9406752091FA040F900F900F900F90FF
:10596000222309F4F8C000D000D0EDB7FEB731967D
:1059700086E09BE0F9CB0E9479182091FA0422235B
:1059800009F4E9C000D000D0EDB7FEB7319689E048
:105990009BE0EACB0E948C150097B9F500D000D0AF
:1059A00000D08CE09BE0EDB7FEB7928381838091BD
:1059B000F5179091F617A091F717B091F817838318
:1059C0009483A583B6830E94187587E19BE0ADB7E9
:1059D000BEB712969C938E931197809171249091EB
:1059E0007224A0917324B0917424EDB7FEB7838321
:1059F0009483A583B6830E9418758DB79EB70696CB
:105A00000FB6F8949EBF0FBE8DBF0E94940B2091DD
:105A1000FA04222309F49FC000D000D0EDB7FEB7EE
:105A2000319684E29BE0A0CB83E061E048E021E096
:105A30000E94391100D000D000D087E29BE0EDB782
:105A4000FEB7928381838091E8179091E917A09126
:105A5000EA17B091EB1783839483A583B6830E94E2
:105A6000187500D000D0EDB7FEB731968EE29BE0FE
:105A7000ADB7BEB712969C938E9311978091EC1799
:105A80009091ED17A091EE17B091EF178283938359
:105A9000A483B5838091F0179091F117A091F2172C
:105AA000B091F31786839783A087B1870E941875FA
:105AB000EDB7FEB73A960FB6F894FEBF0FBEEDBF36
:105AC0000E94940B2091FA04222309F444C000D0D0
:105AD00000D0EDB7FEB731968FE39BE045CB6091E8
:105AE000F8047091F90480E090E00E9482746AE406
:105AF00073E00E9497740097A1F46091F80470918C
:105B0000F90480E090E00E948274009721F10E94E5
:105B10007973803100F590915201982B9093520146
:105B20001AC08091520100D000D022E43BE0EDB7D2
:105B3000FEB73283218390E08F70907094838383CB
:105B40000E9418750F900F900F900F900E94940B69
:105B500002C00E94B216A981BA8111961C921E92AF
:105B600083E00F900F90DF91CF911F910F91FF90E5
:105B7000EF90DF90CF90BF90AF909F908F907F90ED
:105B80006F905F904F903F902F900895F89491E21E
:105B9000E0E0F0E0909357008491E2E0F0E0909331
:105BA00057004491E4E0F0E090935700E49190E0D6
:105BB000A0E0B0E0DC019927882750E060E070E0C9
:105BC000762F652F542F4427840F951FA61FB71FCC
:105BD0008E0F911DA11DB11D8093AC179093AD1731
:105BE000A093AE17B093AF1778940895CF93DF9337
:105BF00000D000D000D0CDB7DEB7CE0101966DE069
:105C000070E042E050E00E94407689819A812FEF57
:105C10008F3F920749F482EE94E06DE070E042E03D
:105C200050E00E945E7604C09093E3048093E20407
:105C3000CE0101966BE070E042E050E00E944076B9
:105C400089819A812FEF8F3F920779F48CE390E05E
:105C50009093E1048093E00480EE94E06BE070E0C8
:105C600042E050E00E945E7604C09093E10480938D
:105C7000E004CE01019669E070E042E050E00E944D
:105C8000407689819A812FEF8F3F920779F48AE0DD
:105C900090E09093DF048093DE048EED94E069E061
:105CA00070E042E050E00E945E7604C09093DF0412
:105CB0008093DE04CE0101966BE170E042E050E09B
:105CC0000E94407689819A812FEF8F3F920769F475
:105CD000109293061092920682E996E06BE170E0D2
:105CE00042E050E00E945E7604C090939306809359
:105CF000920685E694E260E070E049E050E00E94A0
:105D000040760E941C0DCE01039663E170E044E0F2
:105D100050E00E9440768B819C81AD81BE818F3F97
:105D20002FEF92072FEFA2072FEFB20749F48FEF63
:105D300094E063E170E044E050E00E945E7608C0C9
:105D40008FEF94E063E170E044E050E00E94407621
:105D5000CE0103966FE070E044E050E00E94407690
:105D60008B819C81AD81BE818F3F2FEF92072FEFFA
:105D7000A2072FEFB20749F48BEF94E06FE070E0D9
:105D800044E050E00E945E7608C08BEF94E06FE044
:105D900070E044E050E00E944076CE01039667E157
:105DA00070E044E050E00E9440768B819C81AD81A0
:105DB000BE818F3F2FEF92072FEFA2072FEFB20781
:105DC00049F483E095E067E170E044E050E00E9430
:105DD0005E7608C083E095E067E170E044E050E063
:105DE0000E94407626960FB6F894DEBF0FBECDBF58
:105DF000DF91CF9108956C9A6B9A6A9A6F9A729A12
:105E0000749A739A779A809880B3897F80BB87E071
:105E100080937E00549A0E94C62D0E94F62D81E048
:105E20000E94A50980E090E00E94300D0E94254468
:105E30008091DE0486FD239A0895CF93DF93EC01D1
:105E400088819981009731F029E08834920709F020
:105E50007BC071C00E94FB2E8091DE0480FD02C0D9
:105E60000E944B4C809170008C7F809370008091D9
:105E7000B60080628093B6001092B20082E08093F8
:105E8000B1008091B60090E0877090700097C9F7DC
:105E90008091700081608093700080E090E064ECFD
:105EA00077E00E941D4A0E949D1780E00E94F01832
:105EB0000E94590F8091F91B85FF02C00E94424544
:105EC0000E94B44E80939A060E940D4D80939B06CB
:105ED00000D000D000D0EDB7FEB731962FE433E00C
:105EE000ADB7BEB712963C932E931197828313825F
:105EF00080919A06848315820E94067510929D06F1
:105F000010929C068DB79EB706960FB6F8949EBF6A
:105F10000FBE8DBF84ED94E090936F2480936E2428
:105F200083E290E090939F0680939E0688E499E038
:105F3000998388830DC0633259F48CE996E060E060
:105F400070E00E940C1CE6CF1982188283E001C029
:105F500081E0DF91CF9108958536910564F120911C
:105F600092063091930620FF10C000D000D021E6A9
:105F700033E0EDB7FEB732832183948383830E949D
:105F800006750F900F900F900F9080910B209091BD
:105F90000C20A0910D20B0910E200196A11DB11DE5
:105FA00080930B2090930C20A0930D20B0930E2093
:105FB00081E090E0089580E090E008954F925F9234
:105FC0006F927F928F929F92AF92BF92CF92DF9209
:105FD000EF92FF920F931F93CF93DF93CDB7DEB76E
:105FE000CB57D0400FB6F894DEBF0FBECDBF2C010B
:105FF000633851F486EA96E0EC966FAFEC970E9416
:106000003837EC966FADEC97D2018D919C9111973A
:10601000B8E087339B07E9F0E8E088339E0718F47F
:10602000009761F09AC6F9E081319F0709F46EC6C6
:1060300029E08831920709F090C681C686EA96E089
:1060400061E870E043E155E00E941D3787E398E086
:1060500071C6623109F086C60E94D60A8091E204B8
:106060009091E30492FF02C00E948C158091E2049B
:106070009091E30493FF0CC00E948D0ADC01CB01D8
:106080008093582490935924A0935A24B0935B246E
:106090008091E20480FF60C000D000D000D0EDB756
:1060A000FEB7319672E0C72ED12CCC0EDD1EADB7F7
:1060B000BEB71296DC92CE92119788E790E0938358
:1060C000828385E793E0958384830E946D758C01BC
:1060D00085E6A82E84E2B82EEDB7FEB736960FB649
:1060E000F894FEBF0FBEEDBFEE24FF2498E7892E83
:1060F000912C29E7622E23E0722ED5012D915D01AE
:10610000EDB7FEB738970FB6F894FEBF0FBEEDBFE0
:106110003196C601800F911FADB7BEB712969C9302
:106120008E9311979382828275826482268317826E
:106130000E946D75080F191F0894E11CF11CEDB742
:10614000FEB738960FB6F894FEBF0FBEEDBFF8E06D
:10615000EF16F10491F602C000E010E08091E20435
:106160009091E304009781F12DB73EB7285030405D
:106170000FB6F8943EBF0FBE2DBFEDB7FEB73196F8
:10618000CE010296800F911FADB7BEB712969C93B9
:106190008E93119788E790E0938382838EE793E054
:1061A0009583848380918F06909190069783868350
:1061B0000E946D75080F191FEDB7FEB738960FB620
:1061C000F894FEBF0FBEEDBF8091E20481FF51C085
:1061D00089E290E06BE270E04AE250E027E00E9442
:1061E000464185E694E20E94AD432DB73EB72A5062
:1061F00030400FB6F8943EBF0FBE2DBFEDB6FEB6D1
:106200000894E11CF11C9E012E5F3F4F200F311FAF
:10621000ADB7BEB712963C932E93119728E730E0A6
:10622000F7013383228325E833E0358324839C01FF
:10623000B901882777FD8095982F0E949D6E20E0F8
:1062400030E048EC52E40E94336EDC01CB01F701F0
:1062500086839783A087B1870E946D75080F191FE9
:106260002DB73EB7265F3F4F0FB6F8943EBF0FBE27
:106270002DBF8091E20482FF57C089E290E06BE27B
:1062800070E04AE250E026E00E94464181E090E062
:106290000E94280B80938E0684E697E10E94AD430E
:1062A0004DB75EB74A5050400FB6F8945EBF0FBE70
:1062B0004DBFEDB6FEB60894E11CF11C9E012E5FA9
:1062C0003F4F200F311FADB7BEB712963C932E93B0
:1062D000119728E730E0F701338322832FE833E07A
:1062E000358324839C01B901882777FD8095982FF9
:1062F0000E949D6E20E030E048EC52E40E94336E34
:10630000DC01CB01F70186839783A087B1870E94C8
:106310006D75080F191F2DB73EB7265F3F4F0FB69B
:10632000F8943EBF0FBE2DBF8091E20483FF36C0BC
:106330004DB75EB74A5050400FB6F8945EBF0FBEDF
:106340004DBFEDB7FEB73196CE010296800F911F7B
:10635000ADB7BEB712969C938E93119788E790E0E5
:10636000938382838AE993E0958384838091501795
:1063700090915117A0915217B0915317868397832C
:10638000A087B1870E946D75080F191FEDB7FEB782
:106390003A960FB6F894FEBF0FBEEDBF8091E204AF
:1063A00084FF32C00E94A70AAB01BC012DB73EB7E3
:1063B0002A5030400FB6F8943EBF0FBE2DBFEDB748
:1063C000FEB73196CE010296800F911FADB7BEB7D2
:1063D00012969C938E93119788E790E09383828323
:1063E00088EA93E095838483468357836087718727
:1063F0000E946D75080F191FEDB7FEB73A960FB6DC
:10640000F894FEBF0FBEEDBF8091E20485FF38C057
:10641000F8944091502450915124609152247091ED
:10642000532478942DB73EB72A5030400FB6F894D5
:106430003EBF0FBE2DBFEDB7FEB73196CE0102961F
:10644000800F911FADB7BEB712969C938E93119794
:1064500088E790E09383828386EB93E0958384833F
:1064600046835783608771870E946D75080F191FD7
:10647000EDB7FEB73A960FB6F894FEBF0FBEEDBF6C
:106480008091E20486FF8DC08091E0049091E10448
:10649000009709F486C0F89480905024909051247D
:1064A000A0905224B0905324789480915C179091DE
:1064B0005D17A0915E17B0915F17A5019401281B8D
:1064C000390B4A0B5B0BCA01B9010E949B6EE62E89
:1064D000C72EF82ED92E6091E0047091E10480E07F
:1064E00090E00E949B6E9B01AC018E2D9C2DAF2DE8
:1064F000BD2DBC01CD010E94336EE82EC92E4DB7D3
:106500005EB74A5050400FB6F8945EBF0FBE4DBF05
:10651000EDB7FEB73196CE010296800F911FADB751
:10652000BEB712969C938E93119788E790E0938361
:1065300082838FEB93E095838483862F972FAE2DF4
:10654000BC2D86839783A087B187EC966FAFEC97BD
:10655000EB967FAFEB970E946D75080F191FEC96B5
:106560006FADEC97EB967FADEB97862F972FAE2D07
:10657000BC2D80935D2490935E24A0935F24B09300
:10658000602480925C1790925D17A0925E17B09283
:106590005F17EDB7FEB73A960FB6F894FEBF0FBE81
:1065A000EDBF8091E20487FF3EC0F89440915424EF
:1065B00050915524609156247091572478942DB7AA
:1065C0003EB72A5030400FB6F8943EBF0FBE2DBFE5
:1065D000EDB7FEB73196CE010296800F911FADB791
:1065E000BEB712969C938E93119788E790E09383A1
:1065F00082838CEC93E09583848346835783608702
:1066000071870E946D75080F191FEDB7FEB73A9696
:106610000FB6F894FEBF0FBEEDBFC8010E94AC2FAD
:10662000009709F013CD8091E2049091E30490FF6C
:106630008DC08091E0049091E104009709F486C038
:10664000F8948090542490905524A0905624B090B3
:10665000572478948091601790916117A0916217E8
:10666000B0916317A5019401281B390B4A0B5B0BF2
:10667000CA01B9010E949B6EE62EC72EF82ED92EB4
:106680006091E0047091E10480E090E00E949B6ED4
:106690009B01AC018E2D9C2DAF2DBD2DBC01CD01DC
:1066A0000E94336EE82EC92E4DB75EB74A50504057
:1066B0000FB6F8945EBF0FBE4DBFEDB7FEB7319673
:1066C000CE010296800F911FADB7BEB712969C9374
:1066D0008E93119788E790E09383828385ED93E012
:1066E00095838483862F972FAE2DBC2D8683978329
:1066F000A087B187EC966FAFEC97EB967FAFEB97E7
:106700000E946D75080F191FEC966FADEC97EB9614
:106710007FADEB97862F972FAE2DBC2D80936124F4
:1067200090936224A0936324B093642480926017B2
:1067300090926117A0926217B0926317EDB7FEB7FF
:106740003A960FB6F894FEBF0FBEEDBF8091E204FB
:106750009091E30491FF3CC04091FB1F5091FC1FBE
:106760006091FD1F7091FE1F2DB73EB72A5030403B
:106770000FB6F8943EBF0FBE2DBFEDB7FEB73196F2
:10678000CE010296800F911FADB7BEB712969C93B3
:106790008E93119788E790E09383828382EE93E053
:1067A0009583848346835783608771870E946D75C4
:1067B000080F191FEDB7FEB73A960FB6F894FEBF53
:1067C0000FBEEDBFC8010E94AC2F009709F03ECC70
:1067D0008091E2049091E30492FF3CC02DB73EB754
:1067E0002A5030400FB6F8943EBF0FBE2DBFEDB714
:1067F000FEB73196CE010296800F911FADB7BEB79E
:1068000012969C938E93119788E790E093838283EE
:106810008BEE93E0958384838091F5179091F61722
:10682000A091F717B091F81786839783A087B18757
:106830000E946D75080F191FEDB7FEB73A960FB697
:10684000F894FEBF0FBEEDBFC8010E94AC2F0097A9
:1068500009F0FCCB8091E2049091E30493FF3CC0EB
:106860002DB73EB72A5030400FB6F8943EBF0FBE4A
:106870002DBFEDB7FEB73196CE010296800F911F66
:10688000ADB7BEB712969C938E93119788E790E0B0
:106890009383828386EF93E0958384838091582449
:1068A00090915924A0915A24B0915B2486839783B8
:1068B000A087B1870E946D75080F191FEDB7FEB74D
:1068C0003A960FB6F894FEBF0FBEEDBFC8010E9406
:1068D000AC2F009709F0BACB8091E2049091E304C9
:1068E00094FF4CC081E00E94390AAB01BC012DB776
:1068F0003EB72A5030400FB6F8943EBF0FBE2DBFB2
:10690000EDB6FEB60894E11CF11CCE010296800F94
:10691000911FADB7BEB712969C938E93119788E7DF
:1069200090E0F7019383828383E094E095838483EE
:10693000CB01BA012091FF0430910005409101057F
:10694000509102050E944D6FDC01CB01F701868357
:106950009783A087B1870E946D75080F191F2DB707
:106960003EB7265F3F4F0FB6F8943EBF0FBE2DBF18
:10697000C8010E94AC2F009709F068CB8091E20417
:106980009091E30495FF4BC082E00E94390AAB016D
:10699000BC018DB79EB70A970FB6F8949EBF0FBE85
:1069A0008DBFEDB6FEB60894E11CF11CCE01029637
:1069B000800F911FADB7BEB712969C938E9311971F
:1069C00088E790E0F7019383828380E194E09583E8
:1069D0008483CB01BA012091FB043091FC044091E7
:1069E000FD045091FE040E944D6FDC01CB01F701C4
:1069F00086839783A087B1870E946D75080F191F42
:106A00002DB73EB7265F3F4F0FB6F8943EBF0FBE7F
:106A10002DBFC8010E94AC2F009709F017CB8091C1
:106A2000E2049091E30496FF06C083E061E046E053
:106A300020E00E9439118091E2049091E30497FFD5
:106A400006C083E061E046E021E00E9439118091B8
:106A5000E2049091E30496FF3CC04DB75EB74A5004
:106A600050400FB6F8945EBF0FBE4DBFEDB7FEB7F6
:106A70003196CE010296800F911FADB7BEB7129628
:106A80009C938E93119788E790E0938382838DE1A6
:106A900094E0958384838091EC179091ED17A091F9
:106AA000EE17B091EF1786839783A087B1870E9476
:106AB0006D75080F191FEDB7FEB73A960FB6F8942B
:106AC000FEBF0FBEEDBFC8010E94AC2F009709F0BA
:106AD000BDCA8091E2049091E30497FF3CC02DB7BA
:106AE0003EB72A5030400FB6F8943EBF0FBE2DBFC0
:106AF000EDB7FEB73196CE010296800F911FADB76C
:106B0000BEB712969C938E93119788E790E093837B
:106B1000828385E294E0958384838091F01790913D
:106B2000F117A091F217B091F31786839783A0878E
:106B3000B1870E946D75080F191FEDB7FEB73A9621
:106B40000FB6F894FEBF0FBEEDBFC8010E94AC2F78
:106B5000009709F07BCA779A8091920690919306EC
:106B600093FD749A809192069091930682FD08C0DD
:106B70008091DE0480FD04C081FF31C01D9B2FC0C9
:106B800000D000D080E394E0ADB7BEB712969C93DE
:106B90008E931197CE01029614969C938E93139721
:106BA0000E9406752091FA040F900F900F900F909D
:106BB0002223A9F000D000D0EDB7FEB7319689ECC2
:106BC0009BE0ADB7BEB712969C938E93119722832C
:106BD00013820E9418750F900F900F900F90809164
:106BE000B1068983FE01E00FF11F128280919206A7
:106BF0009091930680FF12C000D000D087E394E00C
:106C0000EDB7FEB792838183C80102969483838394
:106C10000E9406750F900F900F900F9062E0C62EA5
:106C2000D12CC00ED11ECE010196B6010E94524059
:106C30008091DE0482FF49C084EE94E0BE016F5F64
:106C40007F4FA60120E530E20E94A7448091920682
:106C50009091930692FF39C040E5E42E40E2F42E75
:106C600000E010E058E4A52E54E0B52ED7018D9138
:106C70007D0100D000D0EDB7FEB73196ADB7BEB7FD
:106C80001296BC92AE921197828313820E9406756F
:106C90000F5F1F4F0F900F900F900F900031110555
:106CA00029F78AE090E00E94387500D000D08DE48A
:106CB00094E0EDB7FEB792838183D482C3820E94B1
:106CC00006750F900F900F900F9080919206909103
:106CD000930682FD73980E945A4B86EA96E00E94C2
:106CE0003B3780918F0690919006009711F00E949B
:106CF0004B4C8091B1068F5F8093B10680919206D4
:106D00009091930682FFA2C9739AA0C982EB96E084
:106D10000E94BD3B009731F10E945A4B8091DE04E6
:106D200087FD2B9882EB96E060E470E00E94923B36
:106D300088E199E0D20111969C938E9313C082EB67
:106D400096E00E94BD3B009769F00E944B4C8091F9
:106D5000DE0487FF7BC92B9A79C9F2011182108268
:106D600083E001C081E0C558DF4F0FB6F894DEBF65
:106D70000FBECDBFDF91CF911F910F91FF90EF908C
:106D8000DF90CF90BF90AF909F908F907F906F904B
:106D90005F904F9008950895FC01DB018C918083F2
:106DA00011968C91119781830895FC01DB019081EC
:106DB0008C91981741F421E030E0918111968C91EB
:106DC0001197981711F020E030E0C9010895BC0137
:106DD00085E794E20E94CC360895DC011996ED9186
:106DE000FC911A970280F381E02D309709F0099504
:106DF00008950F931F93CF93DF9300D0CDB7DEB7E5
:106E00008C0188E10E94C140BC01CE0101960E9424
:106E1000CC36D8011996ED91FC911A970190F0812A
:106E2000E02DC801BE016F5F7F4F09950F900F9055
:106E3000DF91CF911F910F910895EF92FF920F93E1
:106E40001F93CF93DF93EC018B017A0149E155E069
:106E50000E944937FA86E986C8016DE175E00E9413
:106E6000A737DF91CF911F910F91FF90EF90089579
:106E70000E9462370895CF93DF93EC0188E165E7C4
:106E800074E20E94B740CE010E946537DF91CF9136
:106E90000895EF92FF920F931F93CF93DF93EC012E
:106EA0008B017A010E948337F886EF82C80161E284
:106EB00075E00E94A737DF91CF911F910F91FF904E
:106EC000EF9008950E948C3708950E94C351089551
:106ED000DC011796ED91FC9118970190F081E02D5F
:106EE00009950895DC011796ED91FC9118970280A1
:106EF000F381E02D309709F00995089582E49EE032
:106F00000E94F6390895FC017383628382E49EE057
:106F1000BF010E94693A0895BC0182E49EE00E948C
:106F2000343A0895CF93DF93EC0182E49EE00E940F
:106F3000FA3908C0FC01228133812C173D0721F06A
:106F40000E94A03A0097B1F7DF91CF9108950F9377
:106F50001F93CF93DF938B010E949237EC01009730
:106F600031F01D830C83C8010E9406548E83DF918B
:106F7000CF911F910F9108951F93CF93DF93EC0151
:106F8000162F888580FF1DC0EC81FD813097C9F0E8
:106F9000D093450EC093440E82E08887CE010696BA
:106FA0000995992787FD909502978230910510F0F9
:106FB000133829F4CE01BE010E94E53702C081E0FA
:106FC0008887DF91CF911F910895CF92DF92EF9242
:106FD000FF920F931F93CF93DF93EC017B01C0903F
:106FE000440ED090450E0091460E1091470EF801C8
:106FF00003C00190F081E02DEC17FD0719F03097E8
:10700000C1F746C0209709F443C08885882309F159
:1070100018860BC0C017D10729F0C80167E8AE0178
:107020000E94BC37F801008111810115110591F70B
:10703000EC81FD81309769F0CE15DF0551F0D093DA
:10704000450EC093440ECE01069663E840E050E042
:107050000995E091460EF091470ECE17DF0791F4A7
:10706000888199819093470E8093460E0DC0808150
:1070700091818C179D0729F4888199819183808360
:1070800003C0FC01309799F7D092450EC092440E90
:10709000DF91CF911F910F91FF90EF90DF90CF90F4
:1070A00008951F93CF93DF931092480EC091460E20
:1070B000D091470E11E00EC08985882341F01887D2
:1070C0001986CE0162E840E050E00E94BC3709908A
:1070D000D881C02D209781F7DF91CF911F9108951E
:1070E0008091490E982F9F5F9093490E089560916B
:1070F000440E7091450E0E94E53708958AE880930A
:10710000490E10924A0E10924B0E1092470E10929A
:10711000460E1092450E1092440E08958091480E2E
:10712000882311F00E94513870914B0E772309F497
:1071300055C020914A0E30E0F901EE0FFF1FEE0F0F
:10714000FF1FE20FF31FE45BF14F60816093EC0ED1
:10715000418152815093EE0E4093ED0E83819481D4
:107160009093F00E8093EF0E2F5F3F4F2F71307092
:1071700020934A0E715070934B0E009741F5809109
:10718000460E9091470E18C08091480E882311F04A
:107190000E9451384091ED0E5091EE0E8091F10E0B
:1071A0009091F20E6091EC0E0E94BC37E091F10ECE
:1071B000F091F20E808191819093F20E8093F10E06
:1071C0008091F10E9091F20E0097F1F607C06138B0
:1071D00019F421E0FC0120870E94BC378091480E01
:1071E00020914B0E90E0820F911D08958091480EE2
:1071F00020914B0E90E0820F911D08959C0170919B
:107200004B0E7032D9F080914A0E870F8F718093A8
:10721000F30E90E0FC01EE0FFF1FEE0FFF1FE80FD3
:10722000F91FE45BF14F60835283418334832383EE
:107230007F5F70934B0E80E090E0089581E090E0D6
:107240000895CF93DF93C091440ED091450E0E94D4
:10725000BC37D093450EC093440EDF91CF91089573
:10726000FC01AB019091460E8091470EA92FB82FDB
:1072700003C00D90BC91A02DAE17BF0791F01097E1
:10728000C1F7309771F090838183F093470EE093BC
:10729000460E81E0808717821682CF0161E80E9446
:1072A00021390895FC01009741F08085815082309A
:1072B00020F481E081878093480E089521E030E03A
:1072C000FC018085882311F420E030E0C901089595
:1072D000CF93DF93EC014A815B818C819D8160E0DB
:1072E00070E00E9490742A813B8188819981289F57
:1072F000A001299F500D389F500D11248E819F8130
:1073000060E070E00E949074DF91CF910895DC01FD
:1073100012962D913C91139780E090E01DC0149639
:10732000ED91FC911597E80FF91F4081442399F4E2
:1073300021E020832D913C911197829FA001839F92
:10734000500D929F500D112416968D919C91179778
:10735000840F951F089501968217930701F780E027
:1073600090E00895FC0146815781A281B38120E01D
:1073700030E019C04617570781F4A481B581A20FE8
:10738000B31F8C91181614F481508C930480F581EE
:10739000E02DE20FF31F8081089580819181480FD5
:1073A000591F2F5F3F4F2A173B0721F78FEF089593
:1073B000FC014681578164177507A8F0A081B1814F
:1073C00082819381A89F9001A99F300DB89F300DB5
:1073D0001124240F351F81E090E06217730728F015
:1073E00080E090E0089580E090E00895FC01118233
:1073F00010820895FC01808191810895FB01208114
:107400003181FC01318320830895FC0180819181C9
:10741000009711F40895C901FC01208131812115E3
:107420003105C9F70895DC01ED91FC911197309772
:1074300029F40BC0DF010190F081E02D8081918162
:107440000097C1F711961C921E92CF010895DC019E
:10745000ED91FC911197309729F0808191811196DF
:107460009C938E93CF010895CF93DF93EC01E88135
:10747000F9813097B9F0A0E0B0E002C0DF01FC0173
:1074800080819181E617F70759F4109719F49983D1
:10749000888303C011969C938E931182108202C040
:1074A000009761F7DF91CF9108950F931F93CF93CA
:1074B000DF938C01EB010E94343AF80180819181C5
:1074C00099838883D183C083DF91CF911F910F91DE
:1074D00008950F931F93CF93DF938C01EB010E94CC
:1074E000343A19821882C8010E94053A009711F4B3
:1074F000F80101C0FC01D183C083DF91CF911F91BE
:107500000F910895DC01ED91FC91119780E090E0DE
:1075100004C001960190F081E02D3097D1F70895D5
:10752000FB01BA01309719F40E94553A0895808101
:107530009181DA0111969C938E9351834083089533
:10754000009721F0FC0180819181089580E090E016
:1075500008958091F40E9091F50E009729F4109201
:10756000F70E1092F60E08950E94CB48BC01E091F0
:10757000F40EF091F50E4281538180819181480F84
:10758000591F461B570B0CC082819381208131818A
:10759000820F931F861B970B8417950708F4AC0185
:1075A0000480F581E02D309779F7460F571F5093EF
:1075B000F70E4093F60E08958FE295E00E9452393F
:1075C0000895EF92FF920F931F93CF93DF937C0167
:1075D000FC0180819181009729F08A35910509F09D
:1075E0006DC00BC01092F50E1092F40E8AE590E07B
:1075F000F7019183808381E065C0673859F5A091D8
:10760000F40EB091F50E04C014960D90BC91A02D0F
:10761000109741F316968D919C91179784179507B3
:1076200099F3A093F40EB093F50E0DC08681978167
:107630008417950739F48481958115969C938E93D0
:107640001497FD01DF011496ED91FC911597309789
:1076500069F7CCCF623851F6C091F40ED091F50E97
:1076600000E010E028C0CE010E94EB570097F1F037
:107670008E819F8168E8AE010E94FE380097A1F4D8
:107680001F821E828C819D810115110521F0F80158
:107690009583848304C09093F50E8093F40E1D822D
:1076A0001C820E94A93AD8CF0E94DC3A9C818D812D
:1076B0008E01C92FD82F2097B1F698CFF7011182EC
:1076C000108283E0DF91CF911F910F91FF90EF9097
:1076D0000895CF93DF93EC010E94DC3A8E819F8165
:1076E0003091F40E2091F50E009759F0E32FF22F10
:1076F00006C0EC17FD0789F00480F581E02D309776
:10770000C1F78091440E9091450E9F838E833C83F8
:107710002D83D093F50EC093F40E0E94A93ADF9109
:10772000CF910895CF93DF93EC010E94CB57CE0108
:107730000E94693BDF91CF910895CF93DF93EC01D5
:107740000E94D757CE010E94693BDF91CF910895E7
:10775000CF93DF93EC010E94E157CE010E94693B79
:10776000DF91CF910895FC0180819181860F971F51
:10777000918380830E94A93A089521E030E0FC01C2
:1077800086819781009711F020E030E0C9010895CB
:10779000FC012281338180819181280F391FC90129
:1077A0000895FC0180819181089581E090E020910D
:1077B000F40E3091F50E2115310511F480E090E0C2
:1077C00008958091F40E9091F50E009729F0809124
:1077D000F60E9091F70E089580E090E00895CF9313
:1077E000DF93EC01E091F40EF091F50E8E179F07F8
:1077F00041F48C819D819093F50E8093F40E14C01A
:10780000FC01309731F0848195818C179D07C1F779
:1078100007C01D821C821F821E82DF91CF910895B6
:107820008C819D81958384830E94A93AF2CFEF9247
:10783000FF920F931F93CF93DF937C018A01FC018A
:1078400080819181009729F08B34910509F049C01E
:107850001AC089EF9EE00E94FA39EC0109C06C81E0
:107860007D81CE0102960E94923B0990D881C02D65
:107870002097A9F781E08093F80E8BE490E0F70160
:107880009183808333C0683889F589EF9EE00E9438
:10789000FA39EC0123C0CE01029608171907D9F472
:1078A00089EF9EE0BE010E94343A0091440E10918F
:1078B000450E8A859B859093450E8093440EEC85FA
:1078C000FD85309719F08E859F8509951093450E9B
:1078D0000093440ED2CF0990D881C02D2097D9F6BD
:1078E000CCCFF7011182108283E001C081E0DF91EB
:1078F000CF911F910F91FF90EF9008951092F80E85
:1079000089EF9EE00E94F63988E495E060E070E03F
:107910000E94303908950F931F93CF93DF93EC01AA
:107920000091440E1091450E1B870A875D874C8796
:107930003F872E878091F80E882379F088E495E0C0
:107940009093450E8093440ECE0102960E94923B86
:107950001093450E0093440E02C07D836C8389EF23
:107960009EE0BE010E94343A89EF9EE0BE010E9473
:10797000693ADF91CF911F910F9108950F931F9353
:10798000CF93DF93EC018091F80E882391F0009162
:10799000440E1091450E88E495E09093450E809337
:1079A000440ECE0102960E949D3B1093450E00931B
:1079B000440E89EF9EE0BE010E94343A89EF9EE0BA
:1079C000BE010E94693ADF91CF911F910F910895F6
:1079D0000F931F93CF93DF93EC018091F80E8823D0
:1079E00091F00091440E1091450E88E495E090933B
:1079F000450E8093440ECE0102960E94A83B109340
:107A0000450E0093440E89EF9EE0BE010E94343A79
:107A100089EF9EE0BE010E94693ADF91CF911F91EC
:107A20000F910895CF93DF93EC018091F80E882396
:107A300029F0CE0102960E94EF3B04C01F821E82F5
:107A40001986188689EF9EE0BE010E94343ADF91C4
:107A5000CF910895CF93DF93EC018091F80E8823A6
:107A600029F0CE0102960E94BD3B12C089EF9EE034
:107A70000E94FA3906C08C179D0741F0FC018081F5
:107A800091810097C1F781E090E002C080E090E032
:107A9000DF91CF910895CF93DF93D0917524C0915A
:107AA00076240E94F748AB01BC018DB79EB7825582
:107AB00090400FB6F8949EBF0FBE8DBFEDB7FEB7D6
:107AC000319684EE9BE0ADB7BEB712969C938E9331
:107AD0001197D2831382C4831582468357836087AC
:107AE00071878091682690916926A0916A26B0914D
:107AF0006B2682879387A487B58780916C269091A7
:107B00006D26A0916E26B0916F2686879787A08BF1
:107B1000B18B8091702690917126A0917226B091C0
:107B20007326828B938BA48BB58B80917426909156
:107B30007526A0917626B0917726868B978BA08F9D
:107B4000B18F8091782690917926A0917A26B09174
:107B50007B26828F938FA48FB58F80917C26909106
:107B60007D26A0917E26B0917F26868F978FA0A339
:107B7000B1A38091802690918126A0918226B09118
:107B8000832682A393A3A4A3B5A380918426909176
:107B90008526A0918626B091872686A397A3A0A7C5
:107BA000B1A78091882690918926A0918A26B091CC
:107BB0008B2682A793A7A4A7B5A780918C26909126
:107BC0008D26A0918E26B0918F2686A797A7A0AB71
:107BD000B1AB8091902690919126A0919226B09180
:107BE000932682AB93ABA4ABB5AB809194269091D6
:107BF0009526A0919626B091972686AB97ABA0AF1D
:107C0000B1AF8091982690919926A0919A26B09133
:107C10009B2682AF93AFA4AFB5AFEDB7FEB7FF968B
:107C200080919C2690919D26A0919E26B0919F26A2
:107C300080839183A283B383EDB7FEB7ED5BFF4FE3
:107C40008091A0269091A126A091A226B091A32672
:107C500080839183A283B383EDB7FEB7E95BFF4FC7
:107C60008091A4269091A526A091A626B091A72642
:107C700080839183A283B383EDB7FEB7E55BFF4FAB
:107C80008091A8269091A926A091AA26B091AB2612
:107C900080839183A283B383EDB7FEB7E15BFF4F8F
:107CA0008091AC269091AD26A091AE26B091AF26E2
:107CB00080839183A283B3830E941875D091752429
:107CC000C09176248DB79EB78E5A9F4F0FB6F89409
:107CD0009EBF0FBE8DBF0E94F748AB01BC01ADB780
:107CE000BEB7D2970FB6F894BEBF0FBEADBFEDB70B
:107CF000FEB7319680EC9CE012969C938E93119780
:107D0000D2831382C4831582468357836087718729
:107D10008091B0269091B126A091B226B091B32661
:107D200082879387A487B5878091B4269091B526E2
:107D3000A091B626B091B72686879787A08BB18B86
:107D40008091B8269091B926A091BA26B091BB2611
:107D5000828B938BA48BB58B8091BC269091BD2692
:107D6000A091BE26B091BF26868B978BA08FB18F36
:107D70008091C0269091C126A091C226B091C326C1
:107D8000828F938FA48FB58F8091C4269091C52642
:107D9000A091C626B091C726868F978FA0A3B1A3C6
:107DA0008091C8269091C926A091CA26B091CB2671
:107DB00082A393A3A4A3B5A38091CC269091CD26B2
:107DC000A091CE26B091CF2686A397A3A0A7B1A756
:107DD0008091D8269091D926A091DA26B091DB2601
:107DE00082A793A7A4A7B5A78091DC269091DD2652
:107DF000A091DE26B091DF2686A797A7A0ABB1ABF6
:107E00000E9418758DB79EB7C2960FB6F8949EBFA4
:107E10000FBE8DBFDF91CF91089580E38093FF0E59
:107E20000895CF93DF936091FF0E70E0C0E3D0E040
:107E3000C61BD70B6E5F704FAE010E948774CE01D8
:107E4000DF91CF910895CF92DF92EF92FF920F933F
:107E50001F93CF93DF937C01C090FD0ED090FE0E58
:107E60006091FF0E70E08601005D1F4F061B170B2F
:107E700001381105D8F4C0E3D0E0C61BD70B6E5F04
:107E8000704FAE010E948774C7018C0F9D1F6091D7
:107E9000000F7091010F2091FB0E3091FC0E620FCC
:107EA000731FA6010E948774C80102C080E090E0A1
:107EB000DF91CF911F910F91FF90EF90DF90CF90C6
:107EC00008959091FF0E980F9093FF0E08954091A2
:107ED000FD0E5091FE0E9C014817590798F08091B5
:107EE000FB0E9091FC0E820F931F9093FC0E8093DB
:107EF000FB0E421B530B5093FE0E4093FD0E81E090
:107F000090E0089580E090E008959093FE0E8093B5
:107F1000FD0E08958091FB0E9091FC0E8E5C904FAB
:107F200008958091FF0E90E08E5F904F089581E05C
:107F300090E02091000F3091010F4FE02233340781
:107F400011F480E090E008950E94973F009769F057
:107F500082E39FE06091000F7091010F4091FD0E50
:107F60005091FE0E0E94877408954091FB0E50912F
:107F7000FC0E41155105C1F08091FD0E9091FE0E51
:107F8000C096A2E3BFE020E330E007C0FD01E40FAC
:107F9000F51F60816D932F5F3F4F28173907B4F3AA
:107FA0001092FC0E1092FB0E08958091000F90919C
:107FB000010F08958091FD0E9091FE0E089590910D
:107FC000FF0E80E3891B089520E38091FF0E281B9C
:107FD0008091FD0E9091FE0E820F911D08951F93CA
:107FE000CF93DF93EC011091FF0E812F90E08C175F
:107FF0009D076CF00E94E43F8C0F9D1F8138910516
:1080000030F41C1B1093FF0E81E090E002C080E072
:1080100090E0DF91CF911F910895CF93DF93EFE729
:10802000F4E21192119284E2EF3AF807D1F7C0E03E
:10803000D0E0CE01880F991F89589B4D67E175E00C
:108040000E94CC362196C430D10599F7DF91CF91AB
:1080500008951092FC0E1092FB0E1092FE0E1092DC
:10806000FD0E80E38093FF0E82E39FE09093010F6B
:108070008093000F0E940D4008950F931F93CF939C
:10808000DF93EC018B010E942940D093010FC09334
:10809000000F1093FE0E0093FD0EDF91CF911F9104
:1080A0000F910895EF92FF920F931F93CF93DF9359
:1080B00000D0CDB7DEB78C0169837A830E94294056
:1080C0006981E62E7A81F72E81E8E816F10418F02E
:1080D00030E8E32EF12C8091000F9091010FB80150
:1080E000A7010E948774F092FE0EE092FD0EC70178
:1080F0000F900F90DF91CF911F910F91FF90EF9014
:108100000895FC01AFE7B4E280E30D900192815045
:10811000E1F7FB01A7E7B4E288E00D9001928150FE
:10812000E1F70895AFE7B4E2FC0180E301900D921E
:108130008150E1F7A7E7B4E2FB0188E001900D92DE
:108140008150E1F70895E82FF0E0EE0FFF1FE158AE
:10815000FB4D7183608381E090E00895E82FF0E0AB
:10816000EE0FFF1FE158FB4D80819181089590E053
:10817000880F991F895B9B4D0E94CC3681E090E06F
:10818000089590E0880F991F895B9B4D0895811594
:10819000910511F00197F1F70895E091B224F09163
:1081A000B32490818091B12489230895E091AF2474
:1081B000F091B02480819091B124892B8083E0914B
:1081C000B424F091B52480819091B124892B8083CF
:1081D0000895E091AF24F091B02490818091B12472
:1081E000809589238083E091B424F091B524908117
:1081F0008091B12480958923808308951F93CF9324
:10820000DF93E091AF24F091B02490818091B1246C
:10821000809589238083E091B424F091B5248081F6
:108220009091B124892B80838FEB93E00E94C7400B
:108230001FB7F894E091B424F091B5249081809117
:10824000B12480958923808383E890E00E94C74011
:10825000E091B224F091B324D081C091B1241FBF2A
:1082600078948BE393E00E94C740E091B224F091B0
:10827000B32480819091B124892319F08D2F8C2310
:1082800001C081E0DF91CF911F9108955093B524F3
:108290004093B4247093B0246093AF249093B3249C
:1082A0008093B22481E090E002C0880F991F2A9544
:1082B000E2F78093B1240E94FE400895CF93DF93AC
:1082C000C82FDFB7F894E091B424F091B5248081F1
:1082D0009091B124892B808383E090E00E94C74075
:1082E000CC2351F0E091B424F091B5249081809199
:1082F000B12480958923808387E190E00E94C74064
:10830000E091B224F091B32480819091B12489232B
:1083100009F4C0E089E590E00E94C740E091B424F0
:10832000F091B52490818091B12480958923808338
:10833000DFBF8BE390E00E94C7408C2FDF91CF918D
:108340000895CF93DF93C82FD8E08C2F81700E94BF
:108350005E41C6958111C068D150B9F78C2FDF916D
:10836000CF9108958FEF0E94A1410895DF92EF927F
:10837000FF920F931F93CF93DF93182FEB010E946F
:10838000FE40882381F580EF0E94A141EE2400E4A5
:1083900098E0D92E81E00E945E41F82E81E00E9493
:1083A0005E41882319F0FF2069F020C0FF2051F4BE
:1083B000011728F0888180FF05C0101719F0E02E02
:1083C000FF24F3948F2D0E945E41888186958883D7
:1083D000FF2011F0806888830150DA94D9F6219645
:1083E0000023B1F605C0EE24EA9402C08EEFE82E19
:1083F0008E2DDF91CF911F910F91FF90EF90DF9025
:1084000008950F931F93CF93DF93182FEB010E94D2
:10841000FE40209751F085E50E94A14108E0899136
:108420000E94A1410150D9F703C08CEC0E94A141E8
:10843000812F0E94A141DF91CF911F910F9108954B
:108440000F931F93CF93DF93E82FDB01EA01B9016C
:108450004C9150E011969C91119780E0482B592B3C
:10846000E03181F4CA018E7F33E0880F991F3A957D
:10847000E1F716962C9116974CE050E0421B5109FB
:10848000480F591F57FF06C081E0888350954195DA
:108490005F4F01C01882E83299F414968C911497BA
:1084A00090E09C01207630702036310549F086FF3F
:1084B00002C04E7F05C085FF02C04C7F01C0487FCF
:1084C000CA0124E0969587952A95E1F7FB01808300
:1084D0004F70F801408380E0DF91CF911F910F91A1
:1084E00008950F931F93CF93DF93EC018B01888145
:1084F000B8010E94B641888381508D3F30F4F80165
:108500008081883211F0803191F7DF91CF911F91F6
:108510000F910895CF93DF93EC010E94FE4084EB0E
:10852000BE010E94014281E00E945E41C82F0E946C
:10853000FE4081E0CC2309F480E0DF91CF910895E3
:108540001F93CF93DF93182FEB010E94FE400E94F0
:10855000CD40882349F084E4BE010E9401421130DD
:1085600029F00E94D64002C082E001C080E0DF9185
:10857000CF911F9108956F927F928F929F92BF9299
:10858000CF92DF92EF92FF920F931F93CF93DF93DF
:10859000CDB7DEB729970FB6F894DEBF0FBECDBFBB
:1085A0007C014B013A0169010E94FE408EEBB7014C
:1085B0000E9401428E010F5F1F4FE9E0BE2E0E9414
:1085C000B241F80181938F01BA94C9F7CE010196A7
:1085D00069E070E00E94855C882361F4F701808186
:1085E000BE016F5F7F4FA401930186010E9420426C
:1085F00080E001C083E029960FB6F894DEBF0FBE7D
:10860000CDBFDF91CF911F910F91FF90EF90DF9041
:10861000CF90BF909F908F907F906F9008958F9292
:108620009F92AF92BF92CF92DF92EF92FF920F9301
:108630001F93CF93DF93CDB7DEB729970FB6F8948A
:10864000DEBF0FBECDBFD82E5B014A0179018EEB94
:1086500060E070E00E9401428E010F5F1F4FF9E061
:10866000CF2E0E94B241F80181938F01CA94C9F7BD
:10867000CE01019669E070E00E94855C882359F480
:108680008D2DBE016F5F7F4FA501940187010E9470
:10869000204280E001C083E029960FB6F894DEBF47
:1086A0000FBECDBFDF91CF911F910F91FF90EF9043
:1086B000DF90CF90BF90AF909F908F900895EF92F2
:1086C000FF921F93CF93DF93CDB7DEB728970FB6F6
:1086D000F894DEBF0FBECDBF182F262FDE011196F6
:1086E000E2E5F5E088E001900D928150E1F7E42E9B
:1086F000FF24E7FCF09441E752E0E49EC001E59ED0
:10870000900DF49E900D112464E670E00E94487173
:10871000CB0134E6239F90011124820F931FFE01A9
:10872000319640E0219130E0E216F30611F4019613
:1087300003C04F5F4830B1F7112319F09095819530
:108740009F4F28960FB6F894DEBF0FBECDBFDF91C6
:10875000CF911F91FF90EF9008950F931F93CF93A8
:10876000DF93CDB7DEB72B970FB6F894DEBF0FBE01
:10877000CDBF182F092F885F612F792F0E94A0424B
:10878000882309F048C066E471E48FE090E00E941D
:108790001844812F902FBE016D5F7F4FAE014E5F59
:1087A0005F4F9E012F5F3F4F0E94BB42882399F588
:1087B000DE011496E2E5F5E088E001900D9281502B
:1087C000E1F7E9814E2F50E021E732E0429FC001FE
:1087D000439F900D529F900D112464E670E00E941B
:1087E0004871CB013A8124E6329F90011124820F17
:1087F000931FDE01149620E03D91E31711F40196DA
:1088000003C02F5F2830C1F72B81222331F09095D0
:1088100081959F4F02C084E391E22B960FB6F894A6
:10882000DEBF0FBECDBFDF91CF911F910F91089595
:10883000DC01CB0181159105A105B10529F081501D
:108840009040A040B040D9F708951092B90080E25E
:108850008093B800089594EA9093BC009091BC0076
:1088600097FFFCCF9091B900987F983011F090312C
:1088700099F48093BB0084E88093BC008091BC0095
:1088800087FFFCCF9091B900987F983139F081E053
:10889000903429F480E0089581E0089580E00895FF
:1088A00044EA34E824E94093BC009091BC0097FF6F
:1088B000FCCF9091B900987F983011F0903199F7E2
:1088C0008093BB003093BC009091BC0097FFFCCF1D
:1088D0009091B900987F903211F0983539F4209337
:1088E000BC009091BC0094FDFCCFDDCF08950E94A8
:1088F0002B44089584E98093BC008091BC0084FDE2
:10890000FCCF08958093BB0084E88093BC008091E5
:10891000BC0087FFFCCF9091B900987F81E098322E
:1089200009F480E0089584EC8093BC008091BC0041
:1089300087FFFCCF8091BB00089584E88093BC0042
:108940008091BC0087FFFCCF8091BB000895FC01A3
:1089500080E1919190933F018150D9F780913C0142
:108960008F7D80933C0180913C01877F80933C0107
:10897000FB0180E1919190933E018150D9F7809164
:108980003C01806880933C0180913D0180FFFCCFD9
:108990004051504080913C01806280933C01809125
:1089A0003C01877F80933C0112C0FB0180E19191E3
:1089B00090933E018150D9F780913C01806880936B
:1089C0003C0180913D0180FFFCCF40515040141686
:1089D00015065CF3F90180E190913E01919381507D
:1089E000D9F781E090E008950F931F93CF93DF9321
:1089F0008C018CE70E9450448CE70E948244C0E1C5
:108A0000D0E0F80181918F010E9482442197C9F73B
:108A10000E947A44DF91CF911F910F910895813088
:108A200039F48CE790E060E070E040E050E006C090
:108A30008CE790E060E070E040EC50E00E940710AE
:108A40000895813039F48CE790E060E070E04EE00A
:108A500050E006C08CE790E060E070E048E050E055
:108A60000E94071008958CE790E060E070E041E01C
:108A700050E00E9407106AE67AE080E090E00E94F1
:108A8000184408958CE790E060E070E048E350E01F
:108A90000E9407108CE790E060E070E049E350E04E
:108AA0000E9407108CE790E060E070E044E150E045
:108AB0000E9407108CE790E060E070E048E750E02B
:108AC0000E9407108CE790E060E070E04EE550E017
:108AD0000E9407108CE790E060E070E04DE650E007
:108AE0000E9407106CE17AE186E090E00E94184451
:108AF0008CE790E060E070E04CE050E00E940710EE
:108B00008CE790E060E070E041E050E00E940710E8
:108B10008CE790E060E070E046E050E00E940710D3
:108B20006AE67AE080E090E00E9418440895CF93CE
:108B3000DF93CDB7DEB7A2970FB6F894DEBF0FBEB6
:108B4000CDBFDE015296EAE5F5E081E101900D929C
:108B50008150E1F7DE011196EBE6F5E081E101904D
:108B60000D928150E1F70E944245CE0142960E944B
:108B7000F44482E00E940F456AE67AE080E090E0EB
:108B80000E941844CE0101960E94F44460E17EEAFE
:108B900088E290E00E94184480E00E94214560E154
:108BA0007EEA88E290E00E94184481E00E9421451C
:108BB000A2960FB6F894DEBF0FBECDBFDF91CF9166
:108BC0000895E6E4F1E080812081908130818295F2
:108BD00086958695837022952F70822B832B929594
:108BE0009F70892B0895DF92EF92FF920F931F934E
:108BF000CF93DF9300D0CDB7DEB780E06CE046E0E6
:108C00000E948F4989E18093C4001092C50082E0E0
:108C10008093C00080E00E94314A0E94BB4884B724
:108C200084B784B784B784B7E6E3FDE222E432E494
:108C3000318320833A968DB79EB70A97E817F907D4
:108C4000B8F300D000D08FE29DE0ADB7BEB712966A
:108C50009C938E9311978CE795E014969C938E933A
:108C600013970E9418750F900F900F900F900E940D
:108C7000B6580E947E388FE295E060E070E00E9476
:108C800030390E947E3CE091C705F091C8050995F6
:108C90000E94E14590E00E94F358CE0101960E94A7
:108CA000ED47882359F000D08AE49DE0EDB7FEB788
:108CB000928381830E9418750F900F90CE010196C8
:108CC0000E94E7360E94F7478C010E94FC47BC01D6
:108CD000C801AE014F5F5F4F0E942B4D0E945A4763
:108CE0000E94104D0E9401480E94AC4E00D08AE6BE
:108CF0009DE0ADB7BEB712969C938E9311970E94DC
:108D0000187500D0EDB7FEB7319607E71DE0ADB797
:108D1000BEB712961C930E9311978A818283138299
:108D20000E941875EDB7FEB73196ADB7BEB7129673
:108D30001C930E9311978981828313820E94187568
:108D40000F900F908BE79DE0EDB7FEB79283818384
:108D50000E9418750F900F900E94F958E0914A06F2
:108D6000F0914B060995E0913106F0913206099594
:108D7000E091F305F091F405099500912F0610910B
:108D80003006E0904806F09049060E940D4DD82E1E
:108D90000E94B44E2DB73EB72A5030400FB6F8941B
:108DA0003EBF0FBE2DBFEDB7FEB731962DE73DE0BC
:108DB000ADB7BEB712963C932E93119713830283DF
:108DC000F582E482D6821782808711860E94187508
:108DD000E0915406F09155062DB73EB7265F3F4F00
:108DE0000FB6F8943EBF0FBE2DBF3097D1F0099556
:108DF000BC0100D000D088E99DE0ADB7BEB71296A7
:108E00009C938E93119780E890E00E943471EDB7A7
:108E1000FEB7748363830E9418750F900F900F90B4
:108E20000F9000D08BEA9DE0ADB7BEB712969C9331
:108E30008E9311970E9418750F900F9083E796E01C
:108E400060E070E00E94303985E594E00E94AF5701
:108E500000D08DEA9DE0EDB7FEB7928381830E943A
:108E600018750F900F900F900F90DF91CF911F9179
:108E70000F91FF90EF90DF90089500D000D000D0C8
:108E8000EDB7FEB7319625EB3DE0ADB7BEB7129614
:108E90003C932E93119793838283758364830E94FE
:108EA00018758DB79EB706960FB6F8949EBF0FBE85
:108EB0008DBF08950F931F93CF93DF93CDB7DEB788
:108EC000A0970FB6F894DEBF0FBECDBF82E290E050
:108ED0000E945876082F282F2B50203108F0982F09
:108EE0009095891709F46DC000D08BED9DE0ADB76A
:108EF000BEB712969C938E9311970E9418758E019F
:108F00000F5F1F4F0F900F90D80180E090E0FC01A1
:108F1000ED52F24FE491ED93019688309105B9F747
:108F2000F894CE0101966EE370E048E050E00E94B4
:108F30005E76D80180E090E0FC01EB53F24FE491C3
:108F4000ED9301968E309105B9F7CE01019660E35D
:108F500070E04EE050E00E945E7680E090E0FC0120
:108F6000E554F24FE491D801ED938D0101968A30DA
:108F70009105A9F7CE01019666E270E04AE050E063
:108F80000E945E7680E290E06DEC7BEA0E9476764D
:108F90008EE190E060E070E00E9476768DE190E0F6
:108FA00060E00E94687684E290E060E070E00E94F9
:108FB00076760AE182E290E06AE175EE0E947676CA
:108FC0007894802FA0960FB6F894DEBF0FBECDBF69
:108FD000DF91CF911F910F910895F8946EE370E0A7
:108FE00042E050E00E944076789480E0089580E26C
:108FF00090E00E94587608958EE190E00E945876A5
:1090000008958DE190E00E94507608954091C42427
:109010005091C5246091C6247091C72490E0A0E0CF
:10902000B0E0480F591F6A1F7B1F4093C424509320
:10903000C5246093C6247093C7244091C0245091E6
:10904000C1246091C2247091C324480F591F6A1F24
:109050007B1F4093C0245093C1246093C22470931B
:10906000C324209164262223A1F04091BC24509176
:10907000BD246091BE247091BF24480F591F6A1F00
:109080007B1F4093BC245093BD246093BE247093F7
:10909000BF2408951F920F920FB60F920BB60F9236
:1090A00011242F933F934F935F936F937F938F93ED
:1090B0009F93AF93BF93EF93FF938091B60F9091DF
:1090C000B70F01969093B70F8093B60F8091B50FAD
:1090D0008F5F8093B50F8038A9F41092B50F8091FF
:1090E000C4249091C524A091C624B091C7240196B0
:1090F000A11DB11D8093C4249093C524A093C624C0
:10910000B093C724809164268823E1F08091B40F46
:109110008F5F8093B40F8038A9F41092B40F8091C0
:10912000BC249091BD24A091BE24B091BF2401968F
:10913000A11DB11D8093BC249093BD24A093BE2497
:10914000B093BF240E94D53B009711F00E94DC3AF7
:10915000FF91EF91BF91AF919F918F917F916F910F
:109160005F914F913F912F910F900BBE0F900FBECB
:109170000F901F901895F8941092B60016BC83EFCC
:1091800087BD82E084BD94E095BD95B395BB809387
:109190006E00789408958091B60F9091B70F20914A
:1091A000B60F3091B70F82179307A9F7089507C03C
:1091B00022E330E0000021503040E1F701970097B2
:1091C000B9F708950F931F93CF93DF938C010E94FB
:1091D000CB48EC010E94CB488C1B9D0B801791075C
:1091E000C8F3DF91CF911F910F91089508950F93C8
:1091F0001F930091C4241091C5242091C62430915E
:10920000C7248091C4249091C524A091C624B09114
:10921000C724081719072A073B0759F7B801C901DE
:109220001F910F9108951F920F920FB60F92112464
:10923000109292050F900FBE0F901F9018951F92DD
:109240000F920FB60F920BB60F9211242F933F93EC
:109250004F935F936F937F938F939F93AF93BF933E
:10926000EF93FF93E0918805F09189058081E0916B
:109270009305F0919405309709F00995FF91EF91CE
:10928000BF91AF919F918F917F916F915F914F911E
:109290003F912F910F900BBE0F900FBE0F901F901C
:1092A00018951F920F920FB60F92112410929F05DE
:1092B0000F900FBE0F901F9018951F920F920FB630
:1092C0000F920BB60F9211242F933F934F935F93FE
:1092D0006F937F938F939F93AF93BF93EF93FF937E
:1092E000E0919505F09196058081E091A005F091BF
:1092F000A105309709F00995FF91EF91BF91AF91CA
:109300009F918F917F916F915F914F913F912F919D
:109310000F900BBE0F900FBE0F901F90189590E00E
:109320002DE030E0829FF001839FF00D929FF00DC1
:109330001124E857FA4FA281B3811C92A481B58110
:109340006C93A681B78188ED8C93A085B1854C93F1
:10935000128614861386089590E02DE030E0829FF7
:10936000F001839FF00D929FF00D1124E857FA4F02
:1093700081E08287A081B1816C933A9680818823B5
:10938000E9F70895CF93C82F8A3031F48091F80F10
:109390006DE00E94AC4902C08D3029F08091F80F39
:1093A0006C2F0E94AC4980E090E0CF9108951F930C
:1093B000CF93DF93182FEB010CC08A3021F4812F5B
:1093C0006DE00E94AC4969916D3019F0812F0E94C7
:1093D000AC498881882389F7DF91CF911F91089547
:1093E0000F931F93CF93DF93CDB7DEB79E01265F18
:1093F0003F4F08EB1FE0C80160E470E048855985E5
:109400000E94AA758F81B8010E94D749DF91CF9140
:109410001F910F9108951F93CF93DF93182FEB01A6
:1094200004C0812F0E94AC492196FE0164916623FD
:10943000C1F7DF91CF911F91089590E02DE030E0CA
:10944000829FF001839FF00D929FF00D1124E85749
:10945000FA4F748763870895682F80E00E94AC49B3
:1094600008958093F80F82EA95E09093312D8093D0
:10947000302D089584B7877F84BF88E10FB6F894B4
:1094800080936000109260000FBE08952FE088E185
:1094900090E00FB6F894A895809360000FBE2093DB
:1094A00060000895A895089588E10FB6F894809318
:1094B0006000109260000FBE0895F89428E088E1E3
:1094C00090E00FB6F894A895809360000FBE2093AB
:1094D0006000FFCF8091CF248091CF2490E0089549
:1094E0008091390181FD10C081E491E06FE140E09D
:1094F0000E944B50813059F021E030E0813111F071
:1095000020E030E0C901089580E090E0089581E016
:1095100090E0089581E491E06FE140E00E944B50BB
:109520000895E9E3F1E0808180818D7F80838DE083
:1095300090E00197F1F782E491E06FE140E023E0F1
:109540000E94555083E090E00197F1F708959091C3
:10955000390191FD0AC0282F803108F02FE085E401
:1095600091E06FE040E00E945550089580913901EC
:1095700081FD13C081E491E06FE140E00E944B5017
:10958000982F8151823038F09F3129F0913019F0B5
:1095900081E0923019F480E0089581E008950E94FE
:1095A000B64A8823E1F30895CF93DF93C82F88301C
:1095B00049F0863039F0893029F0863119F0893147
:1095C00009F045C08091390181FD44C00E94CF4A15
:1095D0000E948A4AD82FC817B9F1C83019F40E94DE
:1095E000914A2BC0C93141F48631A9F482E491E05B
:1095F0006FE140E029E009C0C63169F4893159F4CE
:1096000082E491E06FE140E026E00E945550E3E003
:10961000F0E03197F1F782E491E06FE140E02C2F28
:109620000E945550D83029F489E691E00197F1F76E
:1096300004C0E3E0F0E03197F1F70E948A4A8C170A
:1096400019F083E490E008C080E490E005C082E473
:1096500090E002C084E490E0DF91CF910895809182
:109660009400909195009093FD268093FC2621E034
:109670002093E9268091390181FF15C0209363264C
:1096800080919400909195009093F9268093F8260C
:109690002093E726809139018D7F80933901809155
:1096A00063268823E1F786E10E94D44A81E0809313
:1096B0006426089580916426882351F48091FA0FDE
:1096C000882321F081E080937C1002C00E942F4B00
:1096D00081E090E008950E94CF4A109264260E9493
:1096E000914A809139018260809339018091E72607
:1096F0008823E9F180919400909195002091F826BB
:109700003091F92682179307A0F48091C426909196
:10971000C526A091C626B091C7268C57914EAF4F53
:10972000BF4F8093C4269093C526A093C626B093BE
:10973000C7268091940090919500821B930BA0E026
:10974000B0E04091C4265091C5266091C626709124
:10975000C726840F951FA61FB71F8093C42690931A
:10976000C526A093C626B093C7261092E7268091FF
:10977000E9268823E9F18091940090919500209149
:10978000FC263091FD2682179307A0F48091CC2609
:109790009091CD26A091CE26B091CF268C57914E98
:1097A000AF4FBF4F8093CC269093CD26A093CE266B
:1097B000B093CF268091940090919500821B930BDB
:1097C000A0E0B0E04091CC265091CD266091CE260D
:1097D0007091CF26840F951FA61FB71F8093CC26AC
:1097E0009093CD26A093CE26B093CF261092E92653
:1097F000089580917C10882321F00E942F4B1092B5
:109800007C1080917D10882321F00E946B4B109278
:109810007D101092FA0F08950F931F93CF93DF934B
:10982000F82FE92FAB0181E08093FA0F0091A82671
:109830001091A9262091AA263091AB260F5F1F4FC9
:109840002F4F3F4F0093A8261093A9262093AA26B6
:109850003093AB26862F8E5F87FF0CC080916126E8
:109860009091622601969093622680936126CFEFB5
:10987000DFEF09C02BEF3FE0C9016F2F7E2F0E9461
:109880008774C0E0D0E00E94F94BCE01DF91CF9108
:109890001F910F91089580916426882399F08091FB
:1098A000FA0F882321F40E94B64A882331F481E01C
:1098B00080937D1081E090E008950E946B4B80E0E2
:1098C00090E0089580E090E008951F93CF93DF9398
:1098D0000F92CDB7DEB78FB789838091FA0F8823B7
:1098E00031F5F89480916426882351F080913901F4
:1098F00081FD1BC00E94B64A8823B9F080E003C0F6
:109900000E945A4B81E0909147019E3010F010E088
:1099100001C01FEF882311F00E944B4C16FF05C0B9
:1099200089818FBF81E090E004C089818FBF80E092
:1099300090E00F90DF91CF911F9108958093F90FE0
:1099400008950E948A4A8250813130F4E82FF0E075
:10995000E552FA4F8081089581E0089508958FEFD0
:1099600080934E018CE691E060EF44E022E00E949B
:1099700055508CE290E06EE041E025E00E945550A9
:1099800080E880936F018091460180936D0184E4AB
:1099900091E060E245E021E00E9455500895CF93A8
:1099A000DF93CDEFD3E0CE010197F1F70E94415054
:1099B0001092D82410925A251092DC251092D724A8
:1099C0001092D624E9E3F1E080818E7F808380814C
:1099D0008D7F80838DE090E00197F1F78081816039
:1099E000808382E491E06FE140E023E00E945550E3
:1099F0002197F1F780915D0180915E010E94AF4C4B
:109A00008DEB95E060E070E00E9430390E942F4BB2
:109A100081E090E0DF91CF91089580917E100895CC
:109A2000CF93DF930F92CDB7DEB789830E94CF4AE1
:109A3000298120937E1088E491E06FE140E00E944C
:109A400055500F90DF91CF9108950E94104D86E000
:109A50000E94D44A0895FA018093620190936301B1
:109A600060936001709361013097C1F080818093B1
:109A70006B01818180936A01828180936901838176
:109A8000809368018481809367018581809366015A
:109A900086818093650187818093640108958DEBB1
:109AA00095E00E94523981E08093CF248091D024A8
:109AB0009091D12401969093D1248093D02481E079
:109AC00090E00895CF93DF935091D724252F30E075
:109AD000F901EE0FFF1F3695322F22273795279574
:109AE000E20FF31FE852FB4D4081442309F4F4C018
:109AF0002091390121FDF0C020916426222309F430
:109B0000EBC047FF23C0852F90E0FC01EE0FFF1F45
:109B10009695982F882797958795E80FF91FE85213
:109B2000FB4D10828091982690919926A0919A26BB
:109B3000B0919B260196A11DB11D8093982690930C
:109B40009926A0939A26B0939B26C6C0433018F559
:109B5000852F90E0FC01EE0FFF1F9695982F882728
:109B600097958795E80FF91FE852FB4D1082809179
:109B7000942690919526A0919626B09197260196CD
:109B8000A11DB11D8093942690939526A0939626AF
:109B9000B0939726A1C0C42FD0E022976C177D0701
:109BA00018F5852F90E0FC01EE0FFF1F9695982F7A
:109BB000882797958795E80FF91FE852FB4D10828B
:109BC0008091902690919126A0919226B091932613
:109BD0000196A11DB11D8093902690939126A0938C
:109BE0009226B093932678C0252F30E0B901660FF6
:109BF000771F3695322F222737952795620F731FCF
:109C000067527B4D50E00E9487742091D724822FA9
:109C100090E0FC01EE0FFF1F9695982F88279795EF
:109C20008795E80FF91FE85AFA4D80818093C82480
:109C3000822F90E0FC01EE0FFF1F9695982F88274A
:109C400097958795E80FF91FE852FB4D10822F5F1B
:109C50002093D724233010F01092D7248091D7245A
:109C600090E0FC01EE0FFF1F9695982F882797959F
:109C70008795E80FF91FE852FB4D8081882311F08A
:109C80000E944F4D609147016093C9248091CE247A
:109C9000882311F0681710F46093CE2484E070E0FC
:109CA0000E94A3406091C82483E070E00E94A3401A
:109CB0008091AC269091AD26A091AE26B091AF26B2
:109CC0000196A11DB11D8093AC269093AD26A09363
:109CD000AE26B093AF2602C0C0E0D0E0CE01DF9147
:109CE000CF910895CF93DF93EC01888199810097FC
:109CF00029F024E08B3F920739F505C08BEF94E003
:109D00009983888325C0623819F51092CF240E9468
:109D100029400E948A3F60E870E00E94624D181658
:109D2000190644F40E94853FE0914E06F0914F06DB
:109D30000995E4CF8091CC249091CD240196909305
:109D4000CD248093CC24DACF1982188283E001C01D
:109D500081E0DF91CF91089591E09093FA0F0E94F6
:109D6000A74A0E94F94B08958091390181FD07C0EF
:109D700085E491E06FE040E00E944B50089580E15F
:109D800008950F931F93CF93DF93C82F21E0209363
:109D9000FA0FD09164268091390181FF16C080911D
:109DA0009400909195009093F9268093F826209343
:109DB000E72620936326809139018D7F80933901B6
:109DC000809163268823E1F7D0E00E94CF4A8091FA
:109DD0006426882309F441C08091E9268823E9F1AB
:109DE00080919400909195002091FC263091FD2661
:109DF00082179307A0F48091CC269091CD26A09154
:109E0000CE26B091CF268C57914EAF4FBF4F809347
:109E1000CC269093CD26A093CE26B093CF268091CA
:109E2000940090919500821B930BA0E0B0E04091CC
:109E3000CC265091CD266091CE267091CF26840FEE
:109E4000951FA61FB71F8093CC269093CD26A09375
:109E5000CE26B093CF261092E92689E10E94D44AFB
:109E600086E00E94AE40009751F00E94B44E082F49
:109E700086E00E94AE4081500E94A74A02C000E0E6
:109E800010E080919400909195009093FB26809330
:109E9000FA2681E08093E826F89480913901826067
:109EA00080933901809139018D7F809339016C2F26
:109EB0006E5F8BEF9FE00E948650789480915E26C3
:109EC00090915F26019690935F2680935E260E9474
:109ED000CF4A82E491E060EE45E00E944B50C82FEB
:109EE00086E00E94AE40009719F0802F0E94A74A9A
:109EF000DD2319F00E942F4B02C00E946B4B809112
:109F0000E8268823E9F180919400909195002091B2
:109F1000FA263091FB2682179307A0F48091C82679
:109F20009091C926A091CA26B091CB268C57914E0C
:109F3000AF4FBF4F8093C8269093C926A093CA26DF
:109F4000B093CB268091940090919500821B930B47
:109F5000A0E0B0E04091C8265091C9266091CA2681
:109F60007091CB26840F951FA61FB71F8093C8261C
:109F70009093C926A093CA26B093CB261092E826C8
:109F800080916426882361F08091940090919500DF
:109F90009093FD268093FC2681E08093E92607C0FC
:109FA00082E491E06FE140E023E00E9455500E947E
:109FB000F94BC130E1F0C330A9F48091A026909113
:109FC000A126A091A226B091A3260196A11DB11DA4
:109FD0008093A0269093A126A093A226B093A326B7
:109FE000C2E00AC0C53029F0C73031F404C0C0E077
:109FF00003C0C3E001C0C1E08C2F90E0DF91CF919E
:10A000001F910F910895CF93DF93EB010E940C4CA9
:10A01000009729F4CE010E94C14E009751F0209183
:10A020006126309162262F5F3F4F30936226209346
:10A030006126DF91CF910895CF93DF9380916426BD
:10A04000882321F40E945A4BC1E001C0C0E00E9465
:10A050008A4A863111F0813119F4D091470109C043
:10A0600086E491E06FE140E00E944B50D82FDD0F75
:10A07000D80FCC2311F00E944B4C8D2FDF91CF9144
:10A0800008951092801010927F10EFE6F0E080812A
:10A09000806280830895FC018081862390E002C065
:10A0A000959587954A95E2F70895F894FC0190817B
:10A0B000862F8095892330E002C0220F331F4A95F6
:10A0C000E2F72623282B208378940895CF93DF93FB
:10A0D000EC012196E0917B01DC01EC932E2FA0E8AE
:10A0E000B1E03D9139932150E1F7E150F0E0E058C3
:10A0F000FE4F2181FC01E058FF4F20838F579F4F77
:10A1000021E0FC012083DF91CF910895FC01609351
:10A110008001A1E8B1E0615881918D936A17E1F760
:10A1200008951F920F920FB60F920BB60F92112443
:10A130002F933F934F935F936F937F938F939F934F
:10A14000AF93BF93EF93FF93809147018093C9240E
:10A150002091D62430E0C901880F991F3695322FFF
:10A16000222737952795820F931F88529B4D0E9477
:10A1700066508091D6248F5F8093D624833010F070
:10A180001092D6240E944F4DFF91EF91BF91AF9155
:10A190009F918F917F916F915F914F913F912F91FF
:10A1A0000F900BBE0F900FBE0F901F9018951F922F
:10A1B0000F920FB60F9211240F900FBE0F901F90A9
:10A1C00018951F920F920FB60F9211240F900FBE89
:10A1D0000F901F9018951F920F920FB60F92112497
:10A1E0000F900FBE0F901F9018951F920F920FB6F1
:10A1F0000F921124109263260F900FBE0F901F90A4
:10A2000018951F920F920FB60F9211241092632689
:10A210000F900FBE0F901F9018951F920F920FB6C0
:10A220000F9211248F9381E08093CF248F910F9010
:10A230000FBE0F901F9018951F920F920FB60F929E
:10A240001124109263260F900FBE0F901F90189547
:10A250001F920F920FB60F9211248F939F938091AC
:10A260007F109091801001969093801080937F10C2
:10A270009F918F910F900FBE0F901F9018950F9385
:10A280001F93CF93DF9380916C2690916D26A091C0
:10A290006E26B0916F260196A11DB11D80936C268C
:10A2A00090936D26A0936E26B0936F260E94D7538D
:10A2B0008C0181E890E10E94FA3908C0EA81FB81B3
:10A2C000309709F00995CE010E94A03AEC01009761
:10A2D000A9F70115110519F0C8010E946837DF912F
:10A2E000CF911F910F9108950E94F9580E94294023
:10A2F0000E94F0518FE296E0909367268093662645
:10A300000E94D45382E090E060E074E040E05EE1BF
:10A310002FEF31E00E9495530895CF92DF92EF9294
:10A32000FF920F931F93CF93DF936C018B017A0100
:10A3300081E890E10E94FA3909C0EC81FD813097F3
:10A3400011F0C8010995CE010E94A03AEC010097D6
:10A35000A1F7C601B801A7010E947237DF91CF9122
:10A360001F910F91FF90EF90DF90CF900895BC0167
:10A3700081E890E10E94693A0895BC0181E890E18A
:10A380000E94343A0895CF93DF93EC0180916826C0
:10A3900090916926A0916A26B0916B260196A11D25
:10A3A000B11D8093682690936926A0936A26B09386
:10A3B0006B26CE010E94EA53009769F00E94A43FE9
:10A3C000E0913306F09134068DE891E5BE010995E0
:10A3D00081E090E002C080E090E0DF91CF910895AD
:10A3E00083E890E10E94F63908950F93CF93DF93AD
:10A3F000EC017B836A8318865F834E8383E890E158
:10A40000BE010E94693AE0918510F0918610309764
:10A4100049F04C815D818A819B81688520E030E034
:10A4200001E00995DF91CF910F910895BC0183E878
:10A4300090E10E94343A08950F93DC0118961C9223
:10A440001897E0918510F0918610309759F0129688
:10A450008D919C91139760E040E050E020E030E067
:10A4600000E009950F9108950F93DC01AB0114965C
:10A470002D913C91159781E018968C93189715961D
:10A480007C936E931497E0918510F091861030972D
:10A4900039F012968D919C91139761E000E0099537
:10A4A0000F9108950F93DC01E0918510F0918610D3
:10A4B000309769F014962D913C91159712968D91D5
:10A4C0009C91139718966C91A90101E009950F9141
:10A4D0000895E0918710F0918810309709F0099560
:10A4E0000895909388108093871008959093861014
:10A4F00080938510089583E890E10E94FA390895C9
:10A50000EF92FF920F931F93CF93DF938C01EB0198
:10A510007A0183E890E10E94FA3915C0DC011296B5
:10A520002D913C9113972C173D0759F41696ED91F8
:10A53000FC911797309749F0B801AE019701099542
:10A5400004C00E94A03A009749F7DF91CF911F9174
:10A550000F91FF90EF9008950895AF92BF92CF9220
:10A56000DF92EF92FF920F931F93CF93DF9300D070
:10A57000CDB7DEB75B010E948A3FFC01E080F1802D
:10A58000FA82E982FCE0EF16F10418F400E010E032
:10A590002DC000D000D087EF95E0EDB7FEB79283D5
:10A5A0008183F482E3820E9406750F900F900F90D2
:10A5B0000F901FC00E948A3FF801EE0FFF1FEE0FA1
:10A5C000FF1FE80FF91FC280D3800E948A3F0F5FF0
:10A5D0001F4FF801EE0FFF1FEE0FFF1FE80FF91FCF
:10A5E00040815181C501B6010E9480520E151F05A0
:10A5F00009F70F900F90DF91CF911F910F91FF906E
:10A60000EF90DF90CF90BF90AF900895CF93DF93FE
:10A61000C4EAD0E16091BA107091BB10CE0149E25A
:10A6200053E520E030E00E948B3C0E94F658609198
:10A63000BA107091BB100E943471BC01CE014097DA
:10A640004DE453E520E030E00E948B3CDF91CF9158
:10A6500008958091BA109091BB102091B81030915C
:10A66000B910880F991F2817390708F4C90190936A
:10A67000BB108093BA100E94065308950F930130C7
:10A6800051F48091B4109091B5109093BB108093C9
:10A69000BA100E9406530F910895CF93DF930E9442
:10A6A00029400E948A3FEC01198218820E947B5245
:10A6B00020C012962D913C911397FC01EE0FFF1FC5
:10A6C000EE0FFF1FEC0FFD1F3383228314962D9195
:10A6D0003C9115970196FC01EE0FFF1FEE0FFF1F37
:10A6E000EC0FFD1F3183208399838883CD010E9465
:10A6F000A03ADC0188819981109729F018962C9155
:10A7000018972223B1F6880F991F880F991F029678
:10A710000E94853F88819981009721F089E890E126
:10A720000E943B37DF91CF910895EF92FF920F93F4
:10A730001F93CF93DF93FC018B017A01E90189E834
:10A7400090E1BF0144E156E00E941D371093B5101F
:10A750000093B410F092B710E092B610D093B910F5
:10A76000C093B8108EE393E50E947652DF91CF91AB
:10A770001F910F91FF90EF900895CF93DF93C4EA5C
:10A78000D0E1CE010E94123DCE0140970E94123DC1
:10A79000CE014B970E943837DF91CF910895809179
:10A7A000BA109091BB1008950E947E370895CF9300
:10A7B000DF93E0911806F09119060995EC010097D6
:10A7C00029F06A817B8181E00E94A340CE01DF9164
:10A7D000CF9108950F931F93CF93DF93EC01E091F6
:10A7E0001A06F0911B0609958C016A817B8181E034
:10A7F0000E94A34081E090E00115110511F480E072
:10A8000090E0DF91CF911F910F910895E0911C0688
:10A81000F0911D06099508959C0180E090E005C027
:10A82000F90131974081840F911D2E5F3F4FF9014F
:10A83000329740814423A1F70895FC01308120E044
:10A84000818190E0822B932B02C0880F991F6A951B
:10A85000E2F7892F9927FA01E25EF94F208130E073
:10A860008223932328E030E0241B350B02C0969509
:10A8700087952A95E2F708956F927F928F929F9223
:10A88000AF92BF92CF92DF92EF92FF920F931F93FE
:10A89000CF93DF935C013B018A01690128303105C8
:10A8A00044F4CB01BA01A9010E941D54F501808333
:10A8B0004EC0790173E0F594E7947A95E1F741157C
:10A8C000510521F04501C0E0D0E005C0F301D501FC
:10A8D00080E090E021C0C3018C0F9D1FB80148E0CB
:10A8E00050E00E941D54F40181934F012196CE1532
:10A8F000DF058CF3C701F7FE02C080E090E0A601FF
:10A90000477050704115510511F1E501C80FD91F6D
:10A91000860D971DB80118C021912D9301968E15B3
:10A920009F05D4F3C701F7FE02C080E090E0A601C6
:10A93000477050704115510551F0E501C80FD91FFE
:10A94000860D971D60E070E00E941D548883DF91A2
:10A95000CF911F910F91FF90EF90DF90CF90BF901C
:10A96000AF909F908F907F906F9008958F929F925D
:10A97000AF92BF92CF92DF92EF92FF920F931F930D
:10A98000CF93DF9300D000D0CDB7DEB70E948A3FCF
:10A990008C0182E090E00E94673F009709F45FC05D
:10A9A000F801918180E02081820F911D0E949237F1
:10A9B0007C01009709F455C00E948A3F4C01F701C1
:10A9C0008681482F46954695469550E090E08770E1
:10A9D000907021E030E0009711F420E030E0CA01EF
:10A9E000820F931F0E94673F0097C9F1F70104810E
:10A9F0001581CC24DD242EC0F801A180BB24B60132
:10AA0000A3E075956795AA95E1F7680D791DA601F4
:10AA100047705070883168F0CE01039695010E940E
:10AA20003C54F8018081BE016D5F7F4F0E94B740AA
:10AA30000DC01A821982CE01019695010E943C54E4
:10AA400069817A81F80180810E94A340CA0CDB1CD5
:10AA50000E5F1F4FF8018081882371F602C0EE243B
:10AA6000FF24C7010F900F900F900F90DF91CF91AF
:10AA70001F910F91FF90EF90DF90CF90BF90AF901C
:10AA80009F908F900895FC0150E080E190E0861B3C
:10AA9000970B821B930B02C0440F551F8A95E2F758
:10AAA0008081852B80838181842B818308956F929F
:10AAB0007F928F929F92AF92BF92CF92DF92EF924E
:10AAC000FF920F931F93CF93DF933C016B015A01C9
:10AAD00079012830310524F4C301FA01408159C0BD
:10AAE0008901B3E015950795BA95E1F761157105F0
:10AAF00021F04A01C0E0D0E005C0FA01D30180E0B6
:10AB000090E023C0F40141914F01C3018C0F9D1FC0
:10AB1000B60128E030E00E9443552196C017D107C6
:10AB20008CF3980117FF02C020E030E0D701A77036
:10AB3000B070109781F1F501E20FF31F408150E0F2
:10AB4000C6018A1B9B0B089619C021912D93019673
:10AB500080179107D4F3980117FF02C020E030E07E
:10AB6000D701A770B0701097B1F0F501E20FF31F95
:10AB7000408150E088E090E08A1B9B0B02C0559515
:10AB800047958A95E2F7C301820F931F60E070E05A
:10AB90009D010E944355DF91CF911F910F91FF902E
:10ABA000EF90DF90CF90BF90AF909F908F907F906D
:10ABB0006F9008956F927F928F929F92AF92BF9203
:10ABC000CF92DF92EF92FF920F931F93CF93DF9379
:10ABD00000D0CDB7DEB77C01DC0116968C911697BC
:10ABE000282F26952695269530E090E08770907066
:10ABF00001E010E0009711F400E010E0020F131FD5
:10AC0000C80102960E94EF3F009709F451C00E94CC
:10AC1000913FFC01D70112968C9112978083139675
:10AC20008C9181830E94913F32E0632E712C680EDB
:10AC3000791EC30160E070E0A8010E949074F701E2
:10AC4000E480F580CC24DD242CC0D7011196AC9093
:10AC50001197BB24860193E0159507959A95E1F726
:10AC6000060D171D27E0822E912C8C209D20883107
:10AC700030F00E94C140AC01C801B40109C00E947B
:10AC8000AE409A838983C801B401AE014F5F5F4F24
:10AC900095010E945755CA0CDB1CE2E0F0E0EE0E75
:10ACA000FF1ED7018C91882381F681E090E002C0DD
:10ACB00080E090E00F900F90DF91CF911F910F9166
:10ACC000FF90EF90DF90CF90BF90AF909F908F90CC
:10ACD0007F906F900895E0914C06F0914D06099594
:10ACE0000895E091F505F091F60509950895E09134
:10ACF0005006F091510609950895E0915206F091A1
:10AD000053060995089580E090E008950895E09134
:10AD1000D705F091D8050995089580E090E0089551
:10AD20000F931F93CF93DF93CDB7DEB7E0970FB6A6
:10AD3000F894DEBF0FBECDBF0E94DA3F8C010E94A7
:10AD40008A3F602FAE014F5F5F4F0E94865E88236F
:10AD500009F446C088A99801281B3109C9010E943D
:10AD6000673F0097E9F12E81222379F18A859B853F
:10AD70003BEA8D3C930721F03FEF8F3F930781F52E
:10AD8000223069F088E090E00197E1E0F0E0EC0F1C
:10AD9000FD1FE80FF91F23852F3F21F007C082E038
:10ADA00090E0F2CF181619067CF30FC089E1BE01BE
:10ADB000645F7F4F0E94B74089E10E94C14065E710
:10ADC00074E20E94D536009759F088E1BE016A5EB0
:10ADD0007F4F0E94B740E0913506F0913606099505
:10ADE000E0960FB6F894DEBF0FBECDBFDF91CF91D6
:10ADF0001F910F910895AF92BF92CF92DF92EF9281
:10AE0000FF920F931F93CF93DF93CDB7DEB7E097F9
:10AE10000FB6F894DEBF0FBECDBF5C016B01FE0123
:10AE2000319680E3DF011D928A95E9F781E08983FD
:10AE30008CE00E94AE408C831D821F828091BE10E8
:10AE400089878F5F8093BE1003E008878DEC9BEAB3
:10AE50009B878A8789E10E94C14067E175E00E9473
:10AE6000D536009731F082E08E838FEF8C878D8707
:10AE700009C089E10E94C140BC01CE010C960E942C
:10AE8000CC360E838DEC9BEA9D8B8C8BCE01469647
:10AE900065E774E20E94CC360E948A3F9FA78EA786
:10AEA0000E94DA3F88ABCE0101960E94975D082F81
:10AEB00090E00E94EF3F009749F10E94913FBC0152
:10AEC000CE010196402F0E94B55D0091CD051091F5
:10AED000CE050E94913F7C010E94E43FBC01C70166
:10AEE000F8010995A114B10489F0009721F081308F
:10AEF000910561F404C0C60160E070E003C0C601C2
:10AF000064E070E041E050E0F5010995E0960FB68D
:10AF1000F894DEBF0FBECDBFDF91CF911F910F918F
:10AF2000FF90EF90DF90CF90BF90AF9008950E9478
:10AF3000F6588093BE10E091D705F091D805099599
:10AF40000895009731F0E091D705F091D805099563
:10AF50000895E091D905F091DA0509950895CF9308
:10AF6000DF93EC0104C060E070E00E943039899109
:10AF700099910097C1F7DF91CF910895CF93DF9317
:10AF8000EC0102C00E947738899199910097D1F71E
:10AF9000DF91CF910895CF93DF93EC017B836A8398
:10AFA0000E94CB4899838883DF91CF910895FC015B
:10AFB0008081918122813381820F931F91838083CD
:10AFC0000895CF93DF93EC010E94CB489983888347
:10AFD000DF91CF910895CF93DF93EC010E94CB488E
:10AFE00028813981AC01421B530B9A012F5F3F4FDF
:10AFF00081E090E04A815B814217530710F080E0C6
:10B0000090E0DF91CF910895CF93DF93FC01C2814F
:10B01000D38180819181C80FD91F0E94CB489E01A6
:10B02000281B390BC901DF91CF910895CF93DF938E
:10B03000EEEEF6E2C0EBD6E2A2EEB6E2119211928B
:10B0400019921992199219921D9287E2E630F80727
:10B05000A9F7DF91CF9108950F931F93CF93DF93BB
:10B06000FC01EE51F94D20818C01000F111F000FE2
:10B07000111F222311F12091940030919500E801D5
:10B08000C055D94DFC01EE0FFF1FE251F94D8081F3
:10B090009181A901481B590BCA01A0E0B0E0488189
:10B0A00059816A817B81840F951FA61FB71F8883F2
:10B0B0009983AA83BB8331832083F801E055F94D3E
:10B0C0006081718182819381DF91CF911F910F9176
:10B0D000089560E070E080E090E00895FC01EE0FDC
:10B0E000FF1FEE0FFF1FE055F94D40835183628330
:10B0F00073830895EF92FF920F931F93CF93DF9383
:10B10000B2EEEB2EB6E2FB2EE0EBF6E2CEEED6E2AE
:10B1100020E030E0D7018D917D018823C9F00091B6
:10B1200094001091950088819981A801481B590BC2
:10B1300060E070E080819181A281B381840F951FCE
:10B14000A61FB71F80839183A283B38319830883CB
:10B150002F5F3F4F349622962C303105D9F6DF9180
:10B16000CF911F910F91FF90EF9008950E94195D6C
:10B1700008950F931F93FC018091BF109091C01010
:10B18000338322831583048371836083F093C0101B
:10B19000E093BF10009719F4CB010E94335D80E06B
:10B1A00090E01F910F9108958091BF109091C01071
:10B1B0000097C1F01092C0101092BF10DC011496DD
:10B1C0006D917C9115971296ED91FC9113970995CD
:10B1D000E091BF10F091C010309721F080819181F3
:10B1E0000E94335D08950E94297208950E9424727E
:10B1F000089586E596E00E9468398EE596E00E9403
:10B2000068390895CF93DF930E94973F0097A9F084
:10B210008EE596E00E948739EC01009729F10E94A3
:10B22000DA3F998388830E94D53F9B838A83CE012E
:10B2300004960E94113F8CAB17C086E596E00E94F1
:10B240008739EC01009771F002960E94233F9983A1
:10B250008883BE016E547F4FCE018E579F4F0E9450
:10B26000814002C0C0E0D0E0CE01DF91CF910895CF
:10B27000BC016E547F4F8E579F4F0E9481400895AE
:10B28000CF93DF93EC0186E596E0BE010E94D839AA
:10B29000009719F086E596E009C08EE596E0BE01BC
:10B2A0000E94D839009729F08EE596E0BE010E94F1
:10B2B000B239DF91CF910895CF93DF93EC0186E50A
:10B2C00096E0BE010E94D839009779F068817981B3
:10B2D000CE0102960E945240BE016E547F4FCE01B5
:10B2E0008E579F4F0E9492401CC08EE596E0BE0193
:10B2F0000E94D8390097A9F00E942940688179817D
:10B300008A819B810E9452408CA990E00E94EF3F6D
:10B310000E94913F4CA9BE016C5F7F4F50E00E949C
:10B320008774DF91CF910895CF93DF93EC0186E589
:10B3300096E0BE010E94D839009719F0CE0102961E
:10B340000CC08EE596E0BE010E94D839009719F036
:10B350008A819B8102C080E090E0DF91CF910895C7
:10B36000FC0180819181089570E06F5B7F4F660FD3
:10B37000771F680F791FCB010895E62FF0E0EF5B90
:10B38000FF4FEE0FFF1FE80FF91F80819181089595
:10B3900008958AE197E10E94BD3B009721F08AE180
:10B3A00097E10E94A83B0895E0910517F0910617D8
:10B3B000309711F00995089580E00895EF92FF927B
:10B3C0000F931F93CF93DF937C018A01FC0180814F
:10B3D0009181009731F0F3E08C309F0709F0FFC0B6
:10B3E0002BC080E0E82FF0E0EE0FFF1FEE0FFF1FF5
:10B3F000E85FF84E118210828F5F843098F380935B
:10B4000007178091440E9091450EE8E0F7E1918B8B
:10B41000808B0E947038809306278AE197E160E470
:10B4200070E00E94923B0E94FB5F8CE093E0F7018A
:10B430009183808381E0D7C0623009F4B2C0633069
:10B4400030F4662309F482C0613079F795C067381B
:10B4500019F0683851F73AC010922217C8E0D7E1C6
:10B4600013C08A819B818017910741F4888199815B
:10B470000E943161198218821B821A82249680915F
:10B4800022178F5F8093221780912217843048F310
:10B49000E6E1FCE2848D958D8017910719F4158EF5
:10B4A000148E118EB0962CE2E639F20798F3ECEA8E
:10B4B000FCE2818592858017910711F41582148230
:10B4C0003D968DE2EE32F807A0F3AFCFE7E14A31C7
:10B4D0005E0709F0AACFCA010E94BD3B009709F49C
:10B4E000A4CF109222172DC0F0E035E0EE0FFF1F21
:10B4F0003A95E1F7EA5EF34D818D8823E9F08AE120
:10B5000097E10E94A83B8091221790E025E0880FE8
:10B51000991F2A95E1F78A5E934D9093152C80939D
:10B52000142C82E00E946561809107279091082782
:10B53000009711F00E94D459809122178F5F809359
:10B540002217E0912217E43078F26FCF41155105B0
:10B5500009F46BCF5093152C4093142C83E00E9478
:10B5600065618091072790910827009711F00E944C
:10B57000D4590E94C95959CF4115510509F455CFE5
:10B580005093112C4093102C85E00E9465618091AE
:10B59000072790910827009709F447CF0E94D459B4
:10B5A00044CF8091072790910827009709F43DCF59
:10B5B00080911827863031F48091302781FF02C0B6
:10B5C0000E94C95981E00E9465618091072790918E
:10B5D0000827009709F429CF0E94015C26CFF701C4
:10B5E0001182108283E0DF91CF911F910F91FF9024
:10B5F000EF900895909306178093051708959C0186
:10B600004091440E5091450E60E0E8E0F7E114C02F
:10B61000808191818217930769F4828193818417D5
:10B62000950741F46093231711821082C9010E948B
:10B630003161089534966F5F643050F3609323173F
:10B64000089540E0E8E0F7E116C0542F5F5F2081E5
:10B6500031812115310569F440932417918380834A
:10B660002091440E3091450E338322830E944B611A
:10B6700008953496452F443040F34093241708959D
:10B68000FC018091440E9091450E958F848F778FA9
:10B69000668F0895FC018091440E9091450E92872B
:10B6A0008187748763870895CF93DF93EA010E94AF
:10B6B000BD60009749F02091440E3091450EFC0189
:10B6C00032872187D487C387DF91CF9108950F9365
:10B6D0001F93CF93DF9300D000D0CDB7DEB78C019E
:10B6E000AB018FEF89838A838B838C83CE01019694
:10B6F000B8010E94545B009719F0FC011583048384
:10B700000F900F900F900F90DF91CF911F910F919D
:10B71000089583E796E062E040E050E00E9421391E
:10B7200010920827109207270895AC0183E796E04E
:10B7300061E00E94FE380895AC0183E796E060E086
:10B740000E94FE3808950F931F93CF93DF938A01D1
:10B750000E943160EC01009759F08091440E909165
:10B76000450E9D8F8C8F1F8F0E8FCE010E949C5B8C
:10B77000CE01DF91CF911F910F910895CF93DF9369
:10B78000A091142CB091152C109719F0ED016C9626
:10B7900005C0C091102CD091112C299680910F2CAE
:10B7A00086FF22C01092251740E0E8E0F7E116C0BE
:10B7B0008081918114962D913C9115978217930762
:10B7C00059F482819381009739F04093251799832A
:10B7D00088831B821A8206C034964F5F443040F340
:10B7E000409325170E94C95988819981009731F0AB
:10B7F0004A815B81609106270E942139DF91CF91B8
:10B8000008950F931F93CF93DF938091182786306D
:10B8100009F074C0809107279091082725E08030B7
:10B82000920709F06BC0C4E9D2E0D0930827C09317
:10B83000072702E00093112714E9109312271092B2
:10B840003427109233270E94F35F80959095909350
:10B8500034278093332710921A27109219270E94B9
:10B86000E25F8095909590931A27809319270E9404
:10B87000D459D0930827C09307270093112710931A
:10B8800012279091122C8091132CE92FF82FDF01B1
:10B89000A459BD4F8CE692E00D9001920197E1F71B
:10B8A00087E297E26CE672E00E949F5F80910B272F
:10B8B0008093272780910C278093282780910D273C
:10B8C0008093292780910E2780932A27109234276E
:10B8D000109233270E94F35F8095909590933427C0
:10B8E0008093332710921A27109219270E94E25F43
:10B8F0008095909590931A27809319270E94D45988
:10B90000DF91CF911F910F910895FC0120E030E06D
:10B9100080E0A8E111C0419198E0542F5827B52F3D
:10B92000B17050FD8A278695B13009F4806846953C
:10B93000915099F72F5F3F4F2617370761F708950A
:10B940001F920F920FB60F920BB60F9211242F93E6
:10B950003F934F935F936F937F938F939F93AF9397
:10B96000BF93EF93FF9380919400909195009093F3
:10B97000F3268093F22681E08093E4268091710083
:10B98000807D809371000E94D4588091E4268823A2
:10B99000E9F180919400909195002091F2263091E8
:10B9A000F32682179307A0F48091B8269091B926C8
:10B9B000A091BA26B091BB268C57914EAF4FBF4F86
:10B9C0008093B8269093B926A093BA26B093BB264D
:10B9D0008091940090919500821B930BA0E0B0E0C1
:10B9E0004091B8265091B9266091BA267091BB2635
:10B9F000840F951FA61FB71F8093B8269093B92672
:10BA0000A093BA26B093BB261092E426FF91EF9143
:10BA1000BF91AF919F918F917F916F915F914F9166
:10BA20003F912F910F900BBE0F900FBE0F901F9064
:10BA300018959FB7F894E1E7F0E08081807D8083DE
:10BA400088B38F6288BB10929000E1E9F0E0108229
:10BA5000109292001092950010929400808185605F
:10BA600080839FBF08952FB7F89490939900809397
:10BA7000980088B38F6288BBE1E7F0E08081826044
:10BA800080832FBF0895CF93DF93FC01DB0185E016
:10BA9000EB0119928A95E9F7858190E083709070A7
:10BAA000009711F082E08C93878190E08370907012
:10BAB000009721F082E012968C931297858190E096
:10BAC00083709070009799F0878190E083709070F8
:10BAD000009769F023893489818592852817390771
:10BAE00031F481E0848312961C92129701C0148273
:10BAF000C581C370C250C23028F4D0E0C358D94FBA
:10BB0000888101C080E011968C931197E781E370E2
:10BB1000E250E23028F4F0E0E358F94F808101C0B0
:10BB200080E013968C931397DF91CF910895CF9374
:10BB3000DF9300D000D00F92CDB7DEB7BE016F5FAC
:10BB40007F4F0E94435D89819A81890F8D5F9B8120
:10BB5000890F9C81890F9D81890F0F900F900F9005
:10BB60000F900F90DF91CF910895DF92EF92FF92A7
:10BB70000F931F93CF93DF9300D000D000D0CDB7A9
:10BB8000DEB78C017B01BE016F5F7F4F4E830E9449
:10BB9000435D79816A81AB81BC81872F90E00396F8
:10BBA000860F911D8A0F911D8B0F911D2D81820F84
:10BBB000911D4E8150E0481759070CF498C0F801C8
:10BBC000218130E02170307083E0220F331F8A958D
:10BBD000E1F7828190E08170907034E0880F991FC6
:10BBE0003A95E1F7822B90819770892B438150E041
:10BBF0004170507095E0440F551F9A95E1F7842BE2
:10BC0000448150E04170507026E0440F551F2A9542
:10BC1000E1F7842BF7018083F801258130E0237060
:10BC20003070220F331F220F331F868190E0837004
:10BC3000907054E0880F991F5A95E1F7822B9781F5
:10BC40009295990F990F907C982BF7019183F801A9
:10BC50008085F7018283723051F4F8018185F70104
:10BC60008383F8018285F701848355E001C053E0A6
:10BC700040E080E090E09801260F311D09C0F901F5
:10BC8000E80FF91FD384F701E70FF11DD0824F5F52
:10BC9000742F750F0197461791F7972FA23089F4EB
:10BCA0009701270F311DF8018389F9018083872FC0
:10BCB0008F5F9701280F311DF8018489F901808376
:10BCC0009E5F40E020E030E00B0F111D09C0F8013D
:10BCD000E20FF31F5589F701E80FF11D50834F5F05
:10BCE000842F890F215030404B1789F701C080E025
:10BCF00026960FB6F894DEBF0FBECDBFDF91CF9171
:10BD00001F910F91FF90EF90DF900895BF92CF9217
:10BD1000DF92EF92FF920F931F93CF93DF937C01FB
:10BD2000B62EEA0182E0861708F0AEC0F7018081E6
:10BD3000D82ED294D694D69463E0D622F1E0DF22B6
:10BD4000F7019181292F269526952370C92EC2943B
:10BD5000C694C69473E0C722382F37703883382FC3
:10BD600036953695369531703983382F3295317046
:10BD70003A838295869581708B83DC822D83892F0F
:10BD8000829583708E83CF8282818887222369F196
:10BD90003381948180E0830F911D9A8789872230B7
:10BDA00079F4CA010B9667E175E00E94CC36F70181
:10BDB00086818B8785818C878701095F1F4F20C013
:10BDC00087010B5F1F4F2330D9F4F7013D96DA014D
:10BDD00080E092911B969C931B978F5F1196883001
:10BDE000C1F78701035F1F4F0BC087010D5F1F4F16
:10BDF000CA010B9667E175E00E94CC361A86198657
:10BE0000CC2089F1DD2059F4F8012081918180E076
:10BE1000820F911D9C8B8B8B0E5F1F4F04C08985F9
:10BE20009A859C8B8B8BF2E0CF1671F4CE014596F0
:10BE300067E175E00E94CC36F80181818D8B8081AD
:10BE40008E8B0E5F1F4F17C0F3E0CF16A1F4085F73
:10BE50001F4FD801FE0180E09E91958B8F5F319638
:10BE60008830D1F708C0CE01459667E175E00E94A1
:10BE7000CC361C8A1B8A802F8E199B2D981B9FA75E
:10BE80001EA70DA7B81608F480E0DF91CF911F918F
:10BE90000F91FF90EF90DF90CF90BF9008959C019D
:10BEA00041505040460F571FFB010EC0B081A0E02B
:10BEB0008181BD01680F711D260F371F26173707B7
:10BEC00010F42F5F3F4F3296E417F50778F3E4172D
:10BED000F50749F4908180E0280F391F28173907AA
:10BEE00010F42F5F3F4FC9010895CF93DF93C091A6
:10BEF0001227D0E064973091112720E0C20FD31FA2
:10BF00009E01280F311DC9016BE177E248E050E046
:10BF10000E944F5F63E277E2AE010E944F5F00979D
:10BF200021F098278927982702C08FEF9FEFDF9194
:10BF3000CF91089590932D1780932C170895FC01AD
:10BF40004381460F40930E27872F99272281280F80
:10BF500020930D27A181A0930C27508150930B278C
:10BF600030E02817390748F48A2F8F5F80930C2719
:10BF7000882319F45F5F50930B27842F90E0707033
:10BF80008617970798F480910D278F5F80930D2770
:10BF9000882361F480910C278F5F80930C2788237E
:10BFA00029F480910B278F5F80930B2708959C01C4
:10BFB000AB0180E090E0B9010E944F5F982789278C
:10BFC0009827089580E090E06FE077E244E150E048
:10BFD0000E944F5F009721F098278927982708959E
:10BFE0008FEF9FEF089586E00E94755F089581E1CD
:10BFF0000E94755F089580E0E82FF0E0EE0FFF1FCC
:10C00000EA56F34D118210828F5F8430A8F380E0EE
:10C01000E82FF0E035E0EE0FFF1F3A95E1F7EA5E1A
:10C02000F34D118E8F5F843098F380E094E090930D
:10C03000301780932F1740E08DE090E0242F30E000
:10C04000289FF001299FF00D389FF00D1124E45531
:10C05000F34D158214824F5F4A3080F340932E17C0
:10C060000895CF93DF93EC0120912F173091301773
:10C070002F5F3F4F8DE72030380710F020E030E190
:10C08000522F432FA0E012C0EA2FF0E0B5E0EE0FF0
:10C09000FF1FBA95E1F7EA5EF34D818D882329F001
:10C0A000848195818417950719F3AF5FA43061F7F8
:10C0B0003093301720932F1710922E1780E0E0E076
:10C0C000F0E01EC0A82FB0E055E0AA0FBB1F5A95A4
:10C0D000E1F7AA5EB34D59969C915997992321F4A3
:10C0E00080932E17FD0110C0973049F4309731F03E
:10C0F0005A962C915A97928D921708F4FD018F5FF2
:10C10000843000F380932E17309799F182E0818F6D
:10C1100080913117848780913217858780913317FA
:10C12000868780913417878788ED94E0938B828B84
:10C13000958B848B81E090E0918B808B138E81E0D6
:10C14000828F83E0808F168A80E1878B80912F1702
:10C150009091301798278927982795838483778330
:10C16000668388819981AA81BB8180839183A28320
:10C17000B383CF01DF91CF9108950F931F93CF9396
:10C18000DF93EC018B0120912F17309130176DE078
:10C1900070E02F5F3F4F8DE72030380710F020E030
:10C1A00030E1522F432FA0E011C08A2F90E0869FEC
:10C1B000F001879FF00D969FF00D1124E455F34D8B
:10C1C00084819581AF5F8417950719F3AA3069F7C9
:10C1D0003093301720932F1740E02DE030E018C047
:10C1E000542F5F5F842F90E0829FF001839FF00DBA
:10C1F000929FF00D1124E455F34D848195810097B1
:10C2000031F440932E179F01309749F424C0452FF5
:10C210004A3030F340932E1720E030E01CC080916C
:10C220002F17909130179827892798279583848313
:10C2300017830683209729F41082118212821382B9
:10C2400008C088819981AA81BB8180839183A28360
:10C25000B38380E48087C901DF91CF911F910F9153
:10C26000089540E013C0E42FF0E0542F5F5FEE0F1D
:10C27000FF1FEA56F34D208131812817390729F431
:10C2800040932E17118210820895452F443058F3A1
:10C2900040932E17089540E013C0E42FF0E0542F90
:10C2A0005F5FEE0FFF1FEA56F34D208131812115AC
:10C2B000310529F440932E17918380830895452FEB
:10C2C000443058F340932E170895AF92BF92CF9207
:10C2D000DF92EF92FF920F931F93CF93DF93C09162
:10C2E000142CD091152C843009F4F1C127E337E2E6
:10C2F0003093132C2093122C30930A272093092774
:10C30000833071F4898D90E08F7090708330910547
:10C3100009F074C088899989009709F031C78DC0E8
:10C32000823009F08EC0809134178F5F809334176C
:10C33000882399F4809133178F5F80933317882374
:10C3400061F4809132178F5F80933217882329F42C
:10C35000809131178F5F80933117109208271092C8
:10C3600007271092AB2C1092AA2C898D873011F0E0
:10C37000853041F48A8D8F5F8A8F843109F000C740
:10C38000198EFEC6882309F4FBC628893989211530
:10C39000310509F44EC09A8D292F21502A8F9923F7
:10C3A00009F0EEC69B8D983031F0282F21502230B5
:10C3B00048F4953039F4198E80E880930F2C0E9450
:10C3C000BE5B94C5953048F423E030E0092E02C0EE
:10C3D000220F331F0A94E2F701C020E32A8F9F5FE8
:10C3E0009B8F90E08F70907083309105E1F08430E6
:10C3F00091054CF48130910509F469C382309105AF
:10C4000009F0BEC60DC08630910509F47EC588309E
:10C41000910509F47AC58430910509F0B1C675C556
:10C420001092302757C384E080930F2C0E94BE5B8C
:10C4300092C58F70833009F0A3C688E080930F2CDB
:10C440004AC5853019F5E091102CF091112C8481AA
:10C450009581009709F494C61092152C1092142C13
:10C460002C5030403093132C2093122C30930A27F9
:10C47000209309271092AB2C1092AA2C1092082717
:10C480001092072788E080930F2C1FC180910F27FF
:10C49000853409F075C61091112700E080911227AC
:10C4A000080F111D80910727909108278017910789
:10C4B00008F466C610930827009307278091152774
:10C4C00090E08F739070009709F05AC680911627FC
:10C4D000882309F055C64091A62C5091A72CA09016
:10C4E0007F06B09080064A155B0559F48091A82C10
:10C4F0009091A92C20918106309182068217930792
:10C50000A1F080911F27909120278417950709F0AB
:10C5100037C620912127309122278091A82C909115
:10C52000A92C2817390709F02BC60E94E25F2FEFCC
:10C530008F3F920709F024C680911827863009F4AE
:10C540002EC18131D1F1813009F01AC680912327A3
:10C55000883009F015C610922327809125279091E5
:10C5600026272FEF873F920710F0099601C0089603
:10C570009093262780932527EFE0F7E280911B27F1
:10C5800090911C27A0911D27B0911E2780931F27F3
:10C5900090932027A0932127B09322278091A62C47
:10C5A0009091A72CA091A82CB091A92C8487958755
:10C5B000A687B78780E48087C0C50C5110401093D0
:10C5C0000827009307278BE297E29093132C809320
:10C5D000122C8091292790912A27009739F00E94E8
:10C5E000F75F2FEF8F3F920709F0CAC540912527CB
:10C5F000509126274115510509F4C2C58CEA9CE2E9
:10C600009093112C8093102C6091232770912427F4
:10C61000A0918106B0918206C0918306D0918406D4
:10C620000091850610918606E0901B27F0901C274C
:10C63000C0901D27D0901E272EC084819581009721
:10C6400021F14817590709F586819781009719F05C
:10C6500068177907D1F4208131812A153B0529F427
:10C66000828193818A179B07F9F02C173D0729F4E3
:10C670008281938180179107B9F0E216F30629F4BD
:10C6800082819381C816D90679F0CF010D969093D7
:10C69000112C8093102CE091102CF091112C8DE234
:10C6A000EE32F80750F26CC51092152C1092142C33
:10C6B00082E080930F2C8BE297E290930A2780937D
:10C6C00009271092AB2C1092AA2C0E94BE5B80917D
:10C6D000AA2C9091AB2C009709F452C59C01245EC2
:10C6E0003F4F30930827209307273093112720933B
:10C6F0001227E091102CF091112C20852093172700
:10C7000021E1209318270896982789279827909346
:10C7100028278093272710922A271092292784817F
:10C7200095819093242780932327868197819093E6
:10C730002627809325278091A62C9091A72CA09145
:10C74000A82CB091A92C80931B2790931C27A09311
:10C750001D27B0931E2780819181A281B381809390
:10C760001F2790932027A0932127B093222787E3A8
:10C7700097E29093132C8093122C0E94F75F809580
:10C78000909590932A2780932927009709F0D5C484
:10C790008FEF9FEF90932A2780932927CEC40E9482
:10C7A000F35F2FEF8F3F920709F0EAC4209125270E
:10C7B000309126272115310509F4E2C44091232741
:10C7C000509124274115510509F4DAC4E0911B2743
:10C7D000F0911C27A0911D27B0911E27C6E1DCE235
:10C7E000698D6623A9F08C819D812817390781F412
:10C7F0008E819F814817590759F488819981E817DC
:10C80000F90731F48A819B81A817B90709F47AC125
:10C81000A0968CE2C637D80719F310F38091302721
:10C820008F738230B9F4309336172093351740E078
:10C830000DC0E42FF0E0EE0FFF1FEA56F34D8081AC
:10C8400091814F5F2817390709F47DC0443088F380
:10C8500040932E178091302782FD92C484E180930B
:10C86000302788E290E0909308278093072780E59F
:10C8700080932F2780912A2790912E2790932A2703
:10C880003091292790912D279093292730932D2798
:10C890002091282790912C279093282720932C27AC
:10C8A0009091272790932E1740912B27409327276D
:10C8B00090932B278F5F80932E27882379F4832FE3
:10C8C0008F5F80932D27882349F4822F8F5F809379
:10C8D0002C27882319F49F5F90932B27809123277F
:10C8E0009091242790933617809335172091252710
:10C8F00030912627309324272093232790932627AF
:10C900008093252780911B2790911C27A0911D279C
:10C91000B0911E2780931F2790932027A093212753
:10C92000B09322278091A62C9091A72CA091A82C9F
:10C93000B091A92C80931B2790931C27A0931D27AF
:10C94000B0931E27DFC310922E1780E0C0E0D0E026
:10C9500022C0E82FF0E075E0EE0FFF1F7A95E1F7B7
:10C96000EA5EF34D918D992321F480932E17EF0108
:10C9700016C0973079F4209721F0228D9A8D921766
:10C9800048F4C82FD0E065E0CC0FDD1F6A95E1F7D1
:10C99000CA5ED34D8F5F8430E0F280932E172097CC
:10C9A00009F4EEC3D093152CC093142C83E08A8F26
:10C9B000888F1E8A84E08F8B1B8E80912527909113
:10C9C00026279D838C8380912327909124279F8302
:10C9D0008E8380911B2790911C27A0911D27B091D9
:10C9E0001E2788839983AA83BB8381E0898F8091E6
:10C9F00031178C87809132178D87809133178E87FE
:10CA0000809134178F8781E090E0998B888B80919B
:10CA10002A278B87809129278A87809128278987D1
:10CA200080912727888781E090E00E94FC698091AF
:10CA30002F27282F30E0207F3070213531050CF46E
:10CA400046C082958F7090E00597880F991F880FD8
:10CA5000991F3091371720E031C0E15FF84D30A5C4
:10CA6000332329F420932E171092371730C031301A
:10CA700011F42F5F23C03230E9F441A54430D1F4E2
:10CA800020932E173093371792A580E023A530E02E
:10CA9000282B392B3093361720933517C90124E002
:10CAA000893D920710F088ED94E09B8B8A8B9D8BDB
:10CAB0008C8B0DC041A5442331F0240FE22FF0E010
:10CAC000E817F90754F220932E173093371780E1B7
:10CAD000809330278091302782608093302782E0D6
:10CAE0008093372784E0809338278093392788ED17
:10CAF00080933A278CE290E0909308278093072751
:10CB000080E6ADC2D093152CC093142C10920F2C3C
:10CB10004091302750E042FF03C0198E80E248C2A6
:10CB200080912F2782958F70880F880F80932E1702
:10CB30009801281B31092451304030930827209355
:10CB40000727862F90E08F7090708230910539F41E
:10CB5000CA018F7390708231910551F429C08130E0
:10CB6000910531F4CA018F7390708230910501F103
:10CB70002115310529F4CA01837090700097C1F026
:10CB8000909127278885981709F05FC290912827F0
:10CB90008985981709F059C2909129278A85981795
:10CBA00009F053C290912A278B85981709F04DC23E
:10CBB00044FF4AC0688979896115710509F444C048
:10CBC000CE010C960E949F5F30912B2780910B27FE
:10CBD0003817D1F520912C2780910C272817A1F523
:10CBE00090912D2780910D27981771F580912E2710
:10CBF00040910E27841741F53C872D879E878F87AC
:10CC00008B8D8823D1F42E89888D9A8D891B922F44
:10CC1000969596959695891B280F2E8B87FD819565
:10CC20009F89392F36953695931B980F9F8B822FAE
:10CC3000869586958695890F888F81E080930F2C45
:10CC4000888D8A8F198A188A498D50E0CA018F70A1
:10CC500090708430910509F4B0C18530910564F479
:10CC600082309105C9F1833091050CF0B6C0813056
:10CC7000910509F085C211C08630910509F4DDC126
:10CC8000863091050CF4B9C18730910509F4DDC1F6
:10CC90008830910509F074C285C180910F2C80FF06
:10CCA00014C083E0898F80E480930F2C198A188A3E
:10CCB0008091072790910827009709F408C122E482
:10CCC00020930F2C0E94FC6902C1809130278F7342
:10CCD000823009F055C2FBCE80910F2C80FF72C0CC
:10CCE000809130278F73823109F06CC080912F279B
:10CCF000282F30E0207F3070213531050CF446C0FC
:10CD000082958F7090E00597880F991F880F991F63
:10CD10003091371720E031C0E15FF84D30A5332363
:10CD200029F420932E171092371730C0313011F4A8
:10CD30002F5F23C03230E9F441A54430D1F4209371
:10CD40002E173093371792A580E023A530E0282BCB
:10CD5000392B3093361720933517C90124E0893DCC
:10CD6000920710F088ED94E09B8B8A8B9D8B8C8BC7
:10CD70000DC041A5442331F0240FE22FF0E0E81765
:10CD8000F90754F220932E173093371783E0898FD9
:10CD90008091272788878091282789878091292754
:10CDA0008A8780912A278B8781E090E00E94FC6926
:10CDB00082E480930F2C198A188A10920827109207
:10CDC000072785C080E280930F2C0E94BE5BE09114
:10CDD000142CF091152C118E3DCD8091302780FFC1
:10CDE00025C044FD23C088899989009709F0C8C1EE
:10CDF000809107279091082701960E94FC69209155
:10CE00000F2C822F806180930F2C809107279091A7
:10CE10000827009719F0226120930F2C0E94BE5B17
:10CE200081E090E0998B888B88E06DC085FF1CC005
:10CE30009091352780E02091362730E0282B392B40
:10CE40008091122C9091132C820F931F9093132C8E
:10CE50008093122C8091072790910827821B930BB7
:10CE600090930827809307278091072790910827A0
:10CE7000009749F044FD07C020910F2C22602093B9
:10CE80000F2C0E94FC699091312780E0209132277D
:10CE9000820F911D90933617809335172C893D8909
:10CEA0002817390710F0009721F430933617209394
:10CEB000351780913517909136179B8B8A8B80910F
:10CEC0000F2C90E083709070009709F459C1109274
:10CED000AB2C1092AA2C0E94BE5B20910F2C25FF38
:10CEE00007C01092AB2C1092AA2C198E84E1AEC010
:10CEF00024FF0DC01092AB2C1092AA2C81E090E080
:10CF0000998B888B84E0898F1B8E81E19FC08091F3
:10CF1000AA2C9091AB2C0097E9F020FF02C0198A4F
:10CF2000188A288939892115310581F42A893B8994
:10CF30002817390720F43093AB2C2093AA2C80912A
:10CF4000AA2C9091AB2C998B888B04C03093AB2C7E
:10CF50002093AA2C1B8E8091092790910A279093E9
:10CF6000132C8093122C8091AA2C9091AB2C0097BB
:10CF700059F088899989009739F088969093082705
:10CF80008093072788E10BC080910F2C81FFF8C0A8
:10CF900088E290E0909308278093072780E18093B0
:10CFA00030275CC080910F2C80FFEAC0198E80E191
:10CFB00080930F2C0E94BE5BE3C080910727909165
:10CFC0000827009711F00E94FC699091302780910A
:10CFD0000F2C90FF0BC080FF06C087E0898F1A8E50
:10CFE000198A188A19C086E0898F16C080FF1EC072
:10CFF00085E0898F198A188AC3C08091072790918C
:10D000000827009711F00E94FC698091302780FF6B
:10D010000DC087E0898F1A8E81E090E00E94FC6944
:10D0200080E180930F2C0E94BE5B0FC08091072788
:10D0300090910827009749F4A3C080910F2C80FF9E
:10D040009FC087E0898F1A8E9BC080E18093302734
:10D0500088E290E0909308278093072780E58093EB
:10D060002F27888580932B27898580932C278A8575
:10D0700080932D278B8580932E278C85809327275F
:10D080008D85809328278E85809329278F8580938F
:10D090002A2786E0809318278C819D8190932427EE
:10D0A000809323278E819F81909326278093252725
:10D0B0008091A62C9091A72CA091A82CB091A92C7E
:10D0C00080931B2790931C27A0931D27B0931E27A6
:10D0D00088819981AA81BB8180931F279093202703
:10D0E000A0932127B0932227898D84FF05C0109239
:10D0F00032271092312706C084E08093312788EDD3
:10D100008093322780E4809317278091072790919E
:10D110000827909311278093122710923627109298
:10D12000352710923427109233270E94F35F8095A1
:10D130009095909334278093332785E480930F272D
:10D1400010921027109216271092152780912C17F5
:10D1500090912D17019690932D1780932C179093F3
:10D1600013278093142710921A27109219270E94D0
:10D17000E25F8095909590931A278093192704C0B9
:10D18000109208271092072710920F2CDF91CF9151
:10D190001F910F91FF90EF90DF90CF90BF90AF90D5
:10D1A000089598278927982708950F931F93DC01E6
:10D1B000CB011A2F0B2F20E030E0982789279827E2
:10D1C000A0E0B0E0DC0199278827082B192B2A2B37
:10D1D0003B2BB801C9011F910F910895FC012091CB
:10D1E000092730910A278FE09CE2821B930BAB0149
:10D1F000861797070CF4AC01141615065CF44093DF
:10D20000AA2C5093AB2CE217F30721F0C901BF0100
:10D210000E9487740895CF92DF92EF92FF920F934E
:10D22000CF93DF93CDB7DEB760970FB6F894DEBF2C
:10D230000FBECDBF002309F45AC029873A874B8718
:10D240005C876D877E878F87988B80E2801B4985FE
:10D250005A856B857C851816B4F019821A821B8258
:10D260001C82992787FD9095909581959F4F04C0CA
:10D27000440F551F661F771F8A95D2F74D835E8333
:10D280006F8378872CC06A017B01002E04C0CC0C10
:10D29000DD1CEE1CFF1C0A94D2F7C982DA82EB82F5
:10D2A000FC826A017B0104C0F694E794D794C7948A
:10D2B0008A95D2F7D701C6014D855E856F8578893D
:10D2C00004C0440F551F661F771F0A95D2F7842BA1
:10D2D000952BA62BB72B8D839E83AF83B88729818F
:10D2E0003A814B815C816D817E818F8198856096CA
:10D2F0000FB6F894DEBF0FBECDBFDF91CF910F9177
:10D30000FF90EF90DF90CF900895A0E1B0E0EBE8C0
:10D31000F9E60C94A07129873A874B875C876D8763
:10D320007E878F87988BA982BA82CB82DC82ED823E
:10D33000FE820F8318874D855E856F8578898D8184
:10D340009E81AF81B885481759076A077B07C8F0E7
:10D3500084179507A607B70790F049855A856B850E
:10D360007C8589819A81AB81BC81481759076A07FE
:10D370007B0738F084179507A607B70720F482E0EB
:10D3800003C080E001C081E06096EAE00C94BC71CB
:10D3900080E880936100109261000E94F3450E9432
:10D3A0008E380E94524A8091B6249091B7240097FB
:10D3B00029F001979093B7248093B624C090B824A5
:10D3C000D090B924E090BA24F090BB240E94F74892
:10D3D000DC01CB01C816D906EA06FB0601F30E9460
:10D3E000F748DC01CB018093B8249093B924A09333
:10D3F000BA24B093BB24D3CFBC018091142C90915C
:10D40000152C08960E949F5FE091142CF091152C2A
:10D4100080910B27808780910C27818780910D2731
:10D42000828780910E27838708952F923F924F9293
:10D430005F926F927F928F929F92AF92BF92CF92A4
:10D44000DF92EF92FF920F931F93CF93DF93CDB7AD
:10D45000DEB765970FB6F894DEBF0FBECDBF4C01A7
:10D460007F876E87FC0117821682838181FD04C04D
:10D4700076C34C855D8504C01E010894211C311CB7
:10D48000F4019381EE85FF8593FD859193FF819152
:10D49000FF87EE87882309F45EC3853241F493FD4C
:10D4A000859193FF8191FF87EE87853259F490E053
:10D4B000B4014C8B5D8B0E94DA744C895D895D8769
:10D4C0004C87D7CFFF24DD2410E01032B0F48B322C
:10D4D00069F08C3228F4803251F0833271F40BC041
:10D4E0008D3239F0803349F411602CC01260146021
:10D4F00029C0186027C0106125C017FD2EC0282F35
:10D5000020532A3098F416FF08C08F2D880FF82E6C
:10D51000FF0CFF0CF80EF20E15C08D2D880FD82EC3
:10D52000DD0CDD0CD80ED20E10620CC08E3221F450
:10D5300016FD11C3106406C08C3611F4106802C0C9
:10D54000883659F4EE85FF8593FD859193FF81918F
:10D55000FF87EE87882309F0B8CF982F9554933032
:10D5600018F41061805E06C0982F9556933008F02D
:10D57000A2C11F7E16FD02C0E6E0FE2E1F73853697
:10D5800011F4106406C0863611F4106802C0F11060
:10D59000FA9417FF07C0FBE3FF1548F0EF2CE39464
:10D5A00027E00DC027E02F1530F02F2D07C027E012
:10D5B0007CE3E72E04C027E067E0F62EEE24CA01E4
:10D5C00004969D878C87FA016081718182819381A5
:10D5D000A1010E2D0E9497735C01C9802C2D30E0B3
:10D5E000398B288BC0FE03C0388933FF06C011FD7C
:10D5F00006C012FF06C000E205C00DE203C00BE248
:10D6000001C000E0888999898C709070009709F4B6
:10D610003CC0002311F084E001C083E08D1558F474
:10D62000D81A13FD09C080E290E0B4010E94DA74B8
:10D63000DA94C9F701C0DD24002329F0802F90E09F
:10D64000B4010E94DA74888983FD05C03CE0E32EB2
:10D650003EE0F32E11C028E0E22E2EE0F22E0CC0A8
:10D660000115110509F0805290E0B4010E94DA74AE
:10D670000894E11CF11C04C0012F10E0007110702F
:10D68000F7018491882361F763C217FF0EC0EA0C8B
:10D69000F889F4FF04C08A81813309F4EA941E14E6
:10D6A0004CF528E02E1548F12CC016FD2AC08F2D10
:10D6B00090E08A159B0544F03CEFA3163FEFB306BC
:10D6C0001CF0106801C0FA94FF2049F0E2E0F0E09D
:10D6D000EC0FFD1FEF0DF11D80818033A1F317FFCB
:10D6E00010C0EF2CE3948F2D90E0A816B90644F4F7
:10D6F000FA1807C0EE24E39404C098E0E92E01C0B4
:10D70000FF2417FF07C01A141B043CF495012F5F78
:10D710003F4F05C025E030E002C021E030E00023AB
:10D7200011F02F5F3F4FFF2029F08F2D90E00196E1
:10D73000280F391F8D2D90E02817390714F4D21ABD
:10D7400001C0DD24612E7724C30189709070009799
:10D7500049F406C080E290E0B4010E94DA74DA94E1
:10D76000DD20C1F7002329F0802F90E0B4010E9452
:10D77000DA7463FC09C006C080E390E0B4010E9443
:10D78000DA74DA94DD20C1F717FF48C08501B7FECF
:10D7900002C000E010E04424552495012E193109FF
:10D7A0003B8B2A8B3501601A710A620C731C6F2D3A
:10D7B00070E0EE24FF24E61AF70A3FEF0F3F13074D
:10D7C00029F48EE290E0B4010E94DA74A016B1064A
:10D7D00054F02A893B89201731072CF4F301E40D1A
:10D7E000F51D818101C080E3015010400894411C67
:10D7F000511C0E151F052CF090E0B4010E94DA7444
:10D80000DCCF0A151B0541F49A81963320F4953339
:10D8100019F4388934FF81E390E049C08A8181336B
:10D8200011F09FEEC92290E0B4010E94DA74FF204B
:10D8300089F08EE290E0B4010E94DA7412E0F10106
:10D84000E10FF11D1F5F808190E0B4010E94DA7446
:10D85000FA94A9F764FE03C085E490E002C085E66F
:10D8600090E0B4010E94DA74B7FC05C0A114B104C1
:10D8700041F4C4FE06C0B094A194B108B3948DE203
:10D8800001C08BE290E0B4010E94DA7480E305C02D
:10D890008F5FE6EFFFEFAE0EBF1EFAE0AF16B104EA
:10D8A000BCF790E0B4010E94DA74C501C096B401DF
:10D8B0000E94DA744DC1833631F0833789F08335A5
:10D8C00009F059C022C09A012E5F3F4F3D872C8737
:10D8D000FA018081898381E0E82EF12C510113C087
:10D8E0009A012E5F3F4F3D872C87FA01A080B180BF
:10D8F00016FF03C06F2D70E002C06FEF7FEFC50110
:10D900000E94A0747C011F7714C09A012E5F3F4FC4
:10D910003D872C87FA01A080B18016FF03C06F2DD0
:10D9200070E002C06FEF7FEFC5010E9477747C0149
:10D93000106813FD1CC006C080E290E0B4010E9494
:10D94000DA74DA948D2D90E0E816F906A8F30FC08A
:10D95000F50117FD859117FF81915F0190E0B401FA
:10D960000E94DA74D110DA940894E108F108E11405
:10D97000F10471F7EDC0843611F0893671F59A0122
:10D9800017FF0AC02C5F3F4F3D872C87FA0180812B
:10D990009181A281B3810BC02E5F3F4F3D872C87C1
:10D9A000FA0180819181AA2797FDA095BA2F012FB6
:10D9B0000F76B7FF08C0B095A095909581959F4FC1
:10D9C000AF4FBF4F0068BC01CD01A1012AE030E09C
:10D9D0000E94E275E82EE21841C0853721F41F7ECF
:10D9E0002AE030E020C0197F8F36A9F0803720F47C
:10D9F000883509F0B0C00BC0803721F0883709F0B6
:10DA0000AAC001C0106114FF09C0146007C014FF50
:10DA100008C0166006C028E030E005C020E130E014
:10DA200002C020E132E0CA0117FF09C004969D87B9
:10DA30008C87FA01608171818281938108C002968E
:10DA40009D878C87FA016081718180E090E0A1015F
:10DA50000E94E275E82EE218012F0F7706FF09C039
:10DA60000E7FEF1430F404FF06C002FD04C00F7EE9
:10DA700002C01E2D01C01F2D802F90E004FF0CC09E
:10DA8000FE01EE0DF11D2081203311F4097E09C045
:10DA900002FF06C01E5F05C086789070009709F0EF
:10DAA0001F5FA02EBB2403FD12C000FF0DC0FE2C83
:10DAB0001D1550F4FD0CF11A1D2D06C080E290E0FA
:10DAC000B4010E94DA741F5F1D15C0F304C01D1558
:10DAD00010F4D11A01C0DD24A4FE0FC080E390E051
:10DAE000B4010E94DA74A2FE1FC0A1FE03C088E543
:10DAF00090E010C088E790E00DC0C5018678907076
:10DB0000009791F0A1FC02C080E201C08BE207FD0A
:10DB10008DE290E0B4010E94DA7406C080E390E0E8
:10DB2000B4010E94DA74FA94EF14C0F3EA94F1019C
:10DB3000EE0DF11D808190E0B4010E94DA74EE20B8
:10DB4000A9F706C080E290E0B4010E94DA74DA948A
:10DB5000DD20C1F78ECCF4018681978102C08FEF62
:10DB60009FEF65960FB6F894DEBF0FBECDBFDF9175
:10DB7000CF911F910F91FF90EF90DF90CF90BF90CA
:10DB8000AF909F908F907F906F905F904F903F905D
:10DB90002F9008955058BB27AA270ED044C135D1E5
:10DBA00030F03AD120F031F49F3F11F41EF42AC135
:10DBB0000EF4E095E7FB20C1E92F46D180F3BA17B8
:10DBC000620773078407950718F071F49EF55EC12C
:10DBD0000EF4E0950B2EBA2FA02D0B01B901900188
:10DBE0000C01CA01A0011124FF27591B99F0593FCC
:10DBF00050F4503E68F11A16F040A22F232F342F14
:10DC00004427585FF3CF469537952795A795F04061
:10DC10005395C9F77EF41F16BA0B620B730B840B76
:10DC2000BAF09150A1F0FF0FBB1F661F771F881F2E
:10DC3000C2F70EC0BA0F621F731F841F48F4879586
:10DC400077956795B795F7959E3F08F0B3CF939575
:10DC5000880F08F09927EE0F979587950895A8D01B
:10DC600008F481E008950CD0DEC0D6D040F0CDD0CD
:10DC700030F021F45F3F19F0BFC0511108C1C2C09C
:10DC8000E3D098F39923C9F35523B1F3951B550BB2
:10DC9000BB27AA2762177307840738F09F5F5F4F7F
:10DCA000220F331F441FAA1FA9F333D00E2E3AF0C0
:10DCB000E0E830D091505040E695001CCAF729D0DA
:10DCC000FE2F27D0660F771F881FBB1F2617370729
:10DCD0004807AB07B0E809F0BB0B802DBF01FF2759
:10DCE00093585F4F2AF09E3F510568F085C0CFC022
:10DCF0005F3FECF3983EDCF3869577956795B79593
:10DD0000F7959F5FC9F7880F911D9695879597F9AD
:10DD10000895E1E0660F771F881FBB1F6217730726
:10DD20008407BA0720F0621B730B840BBA0BEE1F3B
:10DD300088F7E0950895E89409C097FB3EF4909524
:10DD40008095709561957F4F8F4F9F4F9923A9F0D4
:10DD5000F92F96E9BB279395F69587957795679563
:10DD6000B795F111F8CFFAF4BB0F11F460FF1BC0A7
:10DD70006F5F7F4F8F4F9F4F16C0882311F096E93A
:10DD800011C0772321F09EE8872F762F05C06623E8
:10DD900071F096E8862F70E060E02AF09A95660FA1
:10DDA000771F881FDAF7880F9695879597F908955A
:10DDB000990F0008550FAA0BE0E8FEEF161617069C
:10DDC000E807F907C0F012161306E407F50798F004
:10DDD000621B730B840B950B39F40A2661F0232B1D
:10DDE000242B252B21F408950A2609F4A140A69599
:10DDF0008FEF811D811D089597F99F6780E870E07E
:10DE000060E008959FEF80EC089500240A941616B0
:10DE1000170618060906089500240A941216130618
:10DE2000140605060895092E0394000C11F48823A6
:10DE300052F0BB0F40F4BF2B11F460FF04C06F5FC2
:10DE40007F4F8F4F9F4F089557FD9058440F551F98
:10DE500059F05F3F71F04795880F97FB991F61F06C
:10DE60009F3F79F087950895121613061406551FE3
:10DE7000F2CF4695F1DF08C0161617061806991F4F
:10DE8000F1CF86957105610508940895E894BB2744
:10DE900066277727CB0197F908950BD0C4CFB5DF5C
:10DEA00028F0BADF18F0952309F0A6CFABCF1124E4
:10DEB000EECFCADFA0F3959FD1F3950F50E0551F29
:10DEC000629FF001729FBB27F00DB11D639FAA27CF
:10DED000F00DB11DAA1F649F6627B00DA11D661F1E
:10DEE000829F2227B00DA11D621F739FB00DA11D3F
:10DEF000621F839FA00D611D221F749F3327A00DF9
:10DF0000611D231F849F600D211D822F762F6A2F94
:10DF100011249F5750408AF0E1F088234AF0EE0F19
:10DF2000FF1FBB1F661F771F881F91505040A9F726
:10DF30009E3F510570F060CFAACF5F3FECF3983E53
:10DF4000DCF3869577956795B795F795E7959F5F8D
:10DF5000C1F7FE2B880F911D9695879597F9089527
:10DF6000FA01EE0FFF1F30962105310599F1611579
:10DF7000710561F48038BFE39B0749F168949038DC
:10DF8000810561F08038BFEF9B0741F0992342F58E
:10DF9000FF3FE1053105210511F1E8940894E7956B
:10DFA000D901AA2329F4AB2FBE2FF85FD0F310C0FC
:10DFB000FF5F70F4A695E0F7F73950F019F0FF3ADB
:10DFC00038F49F779F930CD00F9007FC90580895DA
:10DFD0003EF018CF60E070E080E89FE308954FE7DF
:10DFE0009F775F934F933F932F939ED02F913F91B5
:10DFF0004F915F9152DF05C019F40EF0FDCE46CF70
:10E0000001CF2ADFC8F39638C0F707F80F92E894DB
:10E010002BE33AEA48EB5FE74EDF0F920F920F9245
:10E020004DB75EB70F92C0D0E0E2F1E016D04F914D
:10E030005F91EF91FF91E595EE1FFF1F49F0FE57AD
:10E04000E0684427EE0F441FFA95E1F74195550B20
:10E0500032D00F9007FE26C00895DF93CF931F9311
:10E060000F93FF92EF92DF927B018C01689405C0C1
:10E07000DA2EEF011EDFFE01E894A591259135917E
:10E0800045915591AEF3EF0197DDFE019701A8018F
:10E09000DA9479F7DF90EF90FF900F911F91CF9175
:10E0A000DF9108959B01AC0160E070E080E89FE3A0
:10E0B000DACDA2CEACC0D0DEE8F39923D9F3940F29
:10E0C000511DBBF39150504094F059F0882332F029
:10E0D000660F771F881F91505040C1F79E3F510532
:10E0E00044F7880F911D9695879597F908955F3F9E
:10E0F000ACF0983E9CF0BB27869577956795B795D1
:10E1000008F4B1609395C1F7BB0F58F711F460FFA5
:10E11000E8CF6F5F7F4F8F4F9F4FE3CFB8CE0EF0AA
:10E1200076C070CE689468CE97DEC8F39923D1F399
:10E13000C6F3DF93CF931F930F93FF92C92FDD2771
:10E1400088232AF02197660F771F881FDAF720E0CF
:10E1500030E040E85FEB9FE3883920F0803E30F00C
:10E1600021968F7718DDE8E4F1E003C014DDE5E7E0
:10E17000F1E073DF8B01BE01EC01FB2E6F577109DB
:10E180007595771F880B990BD8DD28E132E741E3BD
:10E190005FE38FDEAF2D9801AE01FF900F911F91CD
:10E1A000CF91DF9109DD3FCEFA01DC01AA0FBB1F41
:10E1B0009B01AC01BF5728F422273327442750780E
:10E1C0001FC0B75188F4AB2F00244695379527958B
:10E1D000011CA395D2F3002069F0220F331F441FC6
:10E1E000B395DAF30DD0D6CC61307105A0E88A077B
:10E1F000B94630F49B01AC016627772788279078D1
:10E20000309621F0208331834283538308959F3FCA
:10E2100031F0915020F4879577956795B795880FE1
:10E22000911D9695879597F90895629FD001739FE8
:10E23000F001829FE00DF11D649FE00DF11D929FA2
:10E24000F00D839FF00D749FF00D659FF00D9927E1
:10E25000729FB00DE11DF91F639FB00DE11DF91F05
:10E26000BD01CF0111240895AA1BBB1B51E107C0BA
:10E27000AA1FBB1FA617B70710F0A61BB70B881F56
:10E28000991F5A95A9F780959095BC01CD010895E5
:10E2900097FB092E07260AD077FD04D0E5DF06D0CC
:10E2A00000201AF4709561957F4F0895F6F79095C8
:10E2B00081959F4F0895A1E21A2EAA1BBB1BFD0159
:10E2C0000DC0AA1FBB1FEE1FFF1FA217B307E40755
:10E2D000F50720F0A21BB30BE40BF50B661F771FAD
:10E2E000881F991F1A9469F760957095809590958D
:10E2F0009B01AC01BD01CF01089597FB092E0526B6
:10E300000ED057FD04D0D7DF0AD0001C38F450954A
:10E310004095309521953F4F4F4F5F4F0895F6F749
:10E3200090958095709561957F4F8F4F9F4F089581
:10E330002F923F924F925F926F927F928F929F9215
:10E34000AF92BF92CF92DF92EF92FF920F931F9303
:10E35000CF93DF93CDB7DEB7CA1BDB0B0FB6F894B4
:10E36000DEBF0FBECDBF09942A88398848885F84F4
:10E370006E847D848C849B84AA84B984C884DF8065
:10E38000EE80FD800C811B81AA81B981CE0FD11D49
:10E390000FB6F894DEBF0FBECDBFED0108958F928A
:10E3A0009F92AF92BF92CF92DF92EF92FF92CF9364
:10E3B000DF93EC0188819981AA81BB810097A10537
:10E3C000B10521F484E299EDABE5B7E0BC01CD01E4
:10E3D0002DE133EF41E050E00E947D7149015A0187
:10E3E00027EA31E440E050E00E9415716B017C01A6
:10E3F000C501B4012CEE34EF4FEF5FEF0E941571B1
:10E40000DC01CB01C80ED91EEA1EFB1EF7FE08C0B8
:10E410008FEF9FEFAFEFBFE7C80ED91EEA1EFB1EBE
:10E42000C882D982EA82FB82C6019F77DF91CF91B1
:10E43000FF90EF90DF90CF90BF90AF909F908F9024
:10E4400008950E94CF71089587E896E00E94CF71E9
:10E450000895A0E0B0E08093870690938806A0938B
:10E460008906B0938A0608953F924F925F926F9209
:10E470007F928F929F92AF92BF92CF92DF92EF9254
:10E48000FF920F931F93CF93DF9300D000D0CDB7AF
:10E49000DEB72B017A016115710529F0DB018C9340
:10E4A00011969C931197E114F10439F097012250D1
:10E4B00030402332310508F0FCC06C01860108941D
:10E4C000C11CD11CF80130803601832D90E00E94E0
:10E4D0006F74009799F7FDE23F1661F4D801119629
:10E4E0003C90119792E0692E712C600E711ECC2425
:10E4F000C3940BC0BBE23B1639F4F801318082E0D3
:10E50000682E712C600E711ECC24E114F10421F0F0
:10E51000F0E1EF16F104F9F480E3381691F4D30139
:10E520008C91883711F0883561F4F301318082E0F5
:10E5300090E0680E791E92E0C92AB0E1EB2EF12C32
:10E540000AC0E114F10439F4A0E33A16D1F0AAE0CC
:10E55000EA2EF12C30C0BAE0EB16F10461F1E0E1F3
:10E56000EE16F10429F0F8E0EF16F104B1F409C059
:10E57000FFEF8F2EFFEF9F2EFFEFAF2EFFE0BF2E9E
:10E5800022C078E0E72EF12CEFEF8E2EEFEF9E2EDB
:10E59000EFEFAE2EEFE1BE2E16C09701442737FDF8
:10E5A0004095542F6FEF7FEF8FEF9FEF0E945B71CD
:10E5B00049015A0108C069E9862E69E9962E69E980
:10E5C000A62E69E1B62E40E000E010E020E030E049
:10E5D000C701AA2797FDA095BA2F89839A83AB8399
:10E5E000BC8350EDD52ED30C99E09D1570F4832D8E
:10E5F00081548A3118F499ECD92E06C0832D8156A6
:10E600008A3168F589EAD82ED30C8D2D90E08E15CD
:10E610009F052CF54F3FF9F080169106A206B30630
:10E62000B8F0C901B80129813A814B815C810E940F
:10E6300015718B019C018D2D90E0A0E0B0E0080FDA
:10E64000191F2A1F3B1F081719072A073B0710F439
:10E650004FEF01C041E0D3013D903D01C2CF4114D5
:10E66000510489F0442339F0089461087108F201DB
:10E670007182608208C0C1FE06C0C3010297D20148
:10E6800011969C938E93C0FE07C0309520951095EF
:10E6900001951F4F2F4F3F4F47FF0FC082E290E081
:10E6A0009093352D8093342D0FEF1FEF2FEF3FEF19
:10E6B00004C000E010E020E030E0B801C9010F9094
:10E6C0000F900F900F90DF91CF911F910F91FF90BE
:10E6D000EF90DF90CF90BF90AF909F908F907F9002
:10E6E0006F905F904F903F900895662777270C9426
:10E6F0007B76FC0188279927E89421912032E9F361
:10E70000293010F02E30C8F32B3241F02D3239F47D
:10E71000689404C00E94D274820F911D21912053ED
:10E720002A30C0F31EF4909581959F4F08952830AC
:10E7300008F027E03327DA01990F311D87FD91603A
:10E7400000966105710539F432602E5F3D9330E328
:10E750002A95E1F708959F3F30F0803871056105F3
:10E7600009F03C5F3C5F3D93913008F08068911D5B
:10E77000DF93CF931F930F93FF92EF92192F987F00
:10E780009695E92F96959695E90FFF27E659F14F53
:10E7900099273327EE24FF24A701E7010590089469
:10E7A000079428F4360FE71EF81E491F511D660F07
:10E7B000771F881F991F0694A1F70590079428F4E6
:10E7C000E70EF81E491F561FC11D770F881F991F9E
:10E7D000661F0694A1F70590079428F4F80E491FC8
:10E7E000561FC71FD11D880F991F661F771F0694DC
:10E7F000A1F70590079420F4490F561FC71FD81F93
:10E80000990F661F771F881F0694A9F784911095AA
:10E81000177041F0D695C79557954795F794E794AB
:10E820001A95C1F7E0E1FEE06894159015913591D5
:10E830006591959105907FE27395E118F10A430B7C
:10E84000560BC90BD009C0F7E10CF11E431F561F30
:10E85000C91FD01D7EF4703311F48A95E6CFE89479
:10E86000015030F0080F0AF40027021708F4202F97
:10E870002395022F7A3328F079E37D932A95E9F7DF
:10E8800010C07D932A9589F60694979567953795DC
:10E8900017951794E118F10A430B560BC90BD009D1
:10E8A00098F023957E9173957A3308F070E37C930A
:10E8B0002013B8F77E9170617D9330F0839571E3FA
:10E8C0007D9370E32A95E1F71124EF90FF900F916B
:10E8D0001F91CF91DF91992787FD90950895911110
:10E8E00089C3803219F089508550D0F70895FC0112
:10E8F0000590615070400110D8F7809590958E0F6B
:10E900009F1F089548E357E10E94AB740895FB01EF
:10E91000DC0102C001900D9241505040D8F708959B
:10E92000DC0101C06D9341505040E0F70895FB01B8
:10E93000DC018D91019080190110D9F3990B089594
:10E94000FC016150704001900110D8F780959095BE
:10E950008E0F9F1F0895FA01A191B081009719F4BD
:10E960001097E1F0CD01DC01CD010D90002011F4F4
:10E97000C00113C0FB012191222319F02015D9F702
:10E98000F3CFFB012191201519F41E92119606C0B8
:10E990002223C1F70D900020A1F7D001FA01A19325
:10E9A000B08308957AE0979F902D879F802D910DD9
:10E9B000112408950F931F93CF93DF938C01EB01E4
:10E9C0008B8181FF1BC082FF0DC02E813F818C8116
:10E9D0009D812817390764F4E881F9810193F9834F
:10E9E000E88306C0E885F985802F0995009731F402
:10E9F0008E819F8101969F838E8302C00FEF1FEF50
:10EA0000C801DF91CF911F910F910895CF93DF93AC
:10EA1000CDB7DEB7FE013596619171918091302DB1
:10EA20009091312DAF010E94156ADF91CF91089529
:10EA3000CF93DF93CDB7DEB7FE013596619171912B
:10EA40008091302D9091312DDC0113962C911397EC
:10EA5000286013962C93AF010E94156AE091302D27
:10EA6000F091312D2381277F2383DF91CF9108956A
:10EA70006091302D7091312D0E94DA7408950F93BA
:10EA80001F93CF93DF938C01E091302DF091312DC6
:10EA9000838181FF1AC0C0E0D0E005C009950097CE
:10EAA00011F0CFEFDFEFF80181918F016091302DF0
:10EAB0007091312DDB011896ED91FC911997882307
:10EAC00069F78AE00995009711F0CFEFDFEFCE01EB
:10EAD000DF91CF911F910F9108950F931F93CF93C3
:10EAE000DF93CDB7DEB72E970FB6F894DEBF0FBE1B
:10EAF000CDBF0D891E898F89988D26E02C831A83BE
:10EB0000098397FF02C080E090E801979E838D8380
:10EB1000AE01455E5F4FCE010196698D7A8D0E94F0
:10EB2000156A4D815E8157FD0AC02F8138854217D5
:10EB300053070CF49A01020F131FF80110822E964E
:10EB40000FB6F894DEBF0FBECDBFDF91CF911F91FE
:10EB50000F9108950F931F93CF93DF93CDB7DEB737
:10EB60002E970FB6F894DEBF0FBECDBF8C0186E0A6
:10EB70008C831A83098377FF02C060E070E86150DC
:10EB800070407E836D83CE010196BA01A9010E9477
:10EB9000156A4D815E8157FD0AC02F813885421765
:10EBA00053070CF49A01020F131FF80110822E96DE
:10EBB0000FB6F894DEBF0FBECDBFDF91CF911F918E
:10EBC0000F910895FA01AA27283051F1203181F1DF
:10EBD000E8946F936E7F6E5F7F4F8F4F9F4FAF4F65
:10EBE000B1E03ED0B4E03CD0670F781F891F9A1F78
:10EBF000A11D680F791F8A1F911DA11D6A0F711D2C
:10EC0000811D911DA11D20D009F468943F912AE037
:10EC1000269F11243019305D3193DEF6CF0108951F
:10EC2000462F4770405D4193B3E00FD0C9F7F6CF50
:10EC3000462F4F70405D4A3318F0495D31FD405218
:10EC4000419302D0A9F7EACFB4E0A69597958795AE
:10EC500077956795BA95C9F700976105710508958D
:10EC60009B01AC010A2E0694579547953795279539
:10EC7000BA95C9F7620F731F841F951FA01D0895D1
:10EC8000DC01CB01FC01F999FECF06C0F2BDE1BD6C
:10EC9000F89A319600B40D9241505040B8F708955B
:10ECA000F999FECF92BD81BDF89A992780B5089554
:10ECB000A8E1B0E042E050E00C944276DC01CB01E8
:10ECC00003C02D910E94697641505040D0F70895BD
:10ECD000262FF999FECF1FBA92BD81BD20BD0FB678
:10ECE000F894FA9AF99A0FBE019608950E946876F0
:10ECF000272F0C9469766F927F928F929F92AF929A
:10ED0000BF92CF92DF92EF92FF920F931F93CF9318
:10ED1000DF935B016115710521F0DB018C93119686
:10ED20009C937C01E7010894E11CF11C08816701B8
:10ED3000802F90E00E946F740097A1F70D3241F48C
:10ED4000098142E0C42ED12CCC0EDD1E11E009C099
:10ED50000B3231F4098132E0C32ED12CCC0EDD1EF2
:10ED600010E0E6012197CE016AE07FE043E050E049
:10ED70000E94FD770097D1F4E6012296CE016DE066
:10ED80007FE045E050E00E94FD77009711F4E60136
:10ED90002796A114B10419F0F501D183C08330E0A6
:10EDA00020E090E8112309F40DC107C1CE0162E112
:10EDB0007FE043E050E00E94FD77009759F4A114F2
:10EDC000B10409F4FCC0C6010296D50111969C93CA
:10EDD0008E93F5C040E050E060E070E08824992414
:10EDE00000530A3090F51260212F30E0C90188707D
:10EDF000907012FF06C0009769F50894811C911C61
:10EE000029C0009719F0089481089108DB01CA0114
:10EE1000D2E0880F991FAA1FBB1FDA95D1F7480FC0
:10EE2000591F6A1F7B1F440F551F661F771F400F16
:10EE3000511D611D711D4839B9E95B07B9E96B07BF
:10EE4000B9E17B0738F0146005C00E3F39F413FDBB
:10EE500043C01860F60101916F01C2CF053311F074
:10EE60000531D1F5D601EC91ED3211F4106108C0F5
:10EE7000EB3229F0C601019621E030E008C0D6014E
:10EE80001196EC911197C601029622E030E0E05312
:10EE9000EA3020F06C01C21AD30A1EC0DC0120E067
:10EEA00030E0FCE020383F075CF4C901880F991F6F
:10EEB000880F991F280F391F220F331F2E0F311D66
:10EEC000ED91E0536D01EA3060F314FF03C030951B
:10EED00021953F4F820E931EC12FD0E011FF08C035
:10EEE000A114B10429F0C6010197D5018D939C931B
:10EEF000CB01BA010E949B6E6B017C01CE01837035
:10EF000090708330910521F4F7FAF094F7F8F094BB
:10EF1000C701B60120E030E040E050E00E942F6ED3
:10EF2000882309F445C097FE07C090948194910806
:10EF30009394C1E4DFE002C0C9E2DFE098EE692EFD
:10EF40009FEF792E6C0E7D1E20E2A22EB12C0FC0F9
:10EF5000FE010591159125913491C701B601A901D2
:10EF600098010E944D6F6B017C018A189B088A14DE
:10EF70009B0474F72497B594A794C615D705B9F7E1
:10EF8000C601D7012A2F220F2B2F221F2F3F51F00E
:10EF9000BC01CD0120E030E040E050E00E942F6E47
:10EFA000882331F482E290E09093352D8093342DC4
:10EFB0003C2D2D2D9E2D8F2D06C08FEF04C030E0EF
:10EFC00020E090EC8FE7B901AC01872F922FA52F9D
:10EFD000B42FBC01CD01DF91CF911F910F91FF9014
:10EFE000EF90DF90CF90BF90AF909F908F907F90E9
:10EFF0006F900895992788270895FB01DC014150FF
:10F00000504088F08D9181341CF08B350CF4805E7B
:10F01000659161341CF06B350CF4605E861B6111E8
:0EF0200071F3990B0895881BFCCFF894FFCF75
:10F02E00263A202573205B414444523D252D642E03
:10F03E00252D64205345513D252D642052535349AF
:10F04E003D252D75204C51493D252D75204452509E
:10F05E003D252D642E253032645D0A00523D252D4E
:10F06E0075204C3D252D7520533D252D64200054D3
:10F07E00696D656F757420414444523D252D642E93
:10F08E00252D64205345513D252D6420525353495F
:10F09E003D252D75204C51493D252D750A002845DD
:10F0AE007874507772290000413A20256420256437
:10F0BE00202564200A00433A20256420256420255B
:10F0CE0064200A007374617475733D307825303294
:10F0DE00780A2000312E30204669726D7761726594
:10F0EE00205665722E20332E3420323031322D319F
:10F0FE00322D323700656570726F6D006F6E006F66
:10F10E00666600666F7263655F69646C6500646550
:10F11E006570004F6E006131007265736574006139
:10F12E003200765F696E00310032003300340061C8
:10F13E0075746F00666C75736800414444523D25CA
:10F14E002D642E252D64205345513D252D642052CE
:10F15E005353493D252D75204C51493D252D750A9A
:10F16E0000707772733D25730A007472696D0043E7
:10F17E00683D252D642054785077723D252D640A04
:10F18E00004572726F72205458204C656E67746819
:10F19E003D25640A0049443D002530327800205058
:10F1AE00533D25640020543D252D362E3266002019
:10F1BE0054313D252D362E32660020545F4D435579
:10F1CE003D252D352E31660020565F4D43553D258C
:10F1DE002D342E3266002050303D252D6C580020E7
:10F1EE0050305F543D252D372E3366002050313D73
:10F1FE00252D6C58002050315F543D252D372E3370
:10F20E0066002055503D252D6C58002052483D2556
:10F21E002D342E31660020565F494E3D252D352E5C
:10F22E0032660020565F41313D252D352E32660067
:10F23E0020565F41323D252D352E32660020503D41
:10F24E00252D6C64002050413D252D372E32660051
:10F25E00263A2025730A00545820706B74206C6572
:10F26E006E203D2025640A0025303258006C656EF4
:10F27E003D25640A00D404BE04A60472048A040068
:10F28E0000506572696F6469632070726F63657395
:10F29E00730000006104071500000000536C6565E3
:10F2AE00702070726F636573730000007C04370FFB
:10F2BE000000000062726F6164636173742070728B
:10F2CE006F636573730000009404DE2F000000006E
:10F2DE00737464696E2070726F63657373000000DF
:10F2EE00B004490E00000000636D642070726F63FD
:10F2FE00657373000000C8041D2F000000000A0093
:10F30E003C00130A6162636465666768696A6B6CC8
:10F31E006D6E6F7020090D00F4041A22FFCC3B2293
:10F32E00FFCC3BED478A3C010010001D004000C29F
:10F33E00060207DF0700000000F936ED3618100050
:10F34E000000004576656E742074696D657200006C
:10F35E00002305E13A000000004374696D657220D8
:10F36E0070726F636573730000003905173C0000FF
:10F37E000000020306070A0B0E0F28432920323025
:10F38E003132204865726A756C6600557476656315
:10F39E006B6C696E6720202020202000436F6E74F6
:10F3AE00696B6920322E3500C600C500C400C1004D
:10F3BE00C200000000CE00CD00CC00C900CA000083
:10F3CE0000000000000200000000C2490000000022
:10F3DE00524632333020647269766572000000B096
:10F3EE0005724E00000000CF4C0C4CC14E03506213
:10F3FE004D654C704A6A4A5A4B4B4C000101010153
:10F40E0001010101010101010101010052696D6556
:10F41E0000EC0574513F5161646174612E6E756D1F
:10F42E0020776179206F75742074686572653A2053
:10F43E0025640A00AD52AC52B654DA550C54008015
:10F44E00C0E0F0F8FCFEFF6E756C6C6D616300271A
:10F45E000686566B56715677567D5683567369637C
:10F46E00736C6F776D6163003D069757FB56905630
:10F47E008756A1578D56BA000800C110C910350025
:10F48E00020099169B165443502F495020737461F5
:10F49E00636B0000006606DE5900000000020800E3
:0CF4AE00000000FFFFFFFF010000000055
:00000001FF
